:100000000C94FA2A0C942CC00C9401C00C94D6BF0A
:100010000C94ABBF0C9480BF0C9455BF0C942ABFBA
:100020000C94FFBE0C942B2B0C942B2B0C942B2B91
:100030000C942B2B0D94950A0C942B2B0C942B2B9E
:100040000C942B2B0C94B8DD0C942B2B0C942B2B99
:100050000C942B2B0C942B2B0C94119A0C94B8C150
:100060000C942B2B0D945F150D94FC150C942B2BDD
:100070000C942B2B0C942B2B0C942B2B0C942B2BA8
:100080000C942B2B0C942B2B0C942B2B0C942B2B98
:100090000C942B2B0C942B2B0C942B2B0C942B2B88
:1000A0000C942B2B0C942B2B0C942B2B0C942B2B78
:1000B0000C942B2B0C942B2B0C942B2B0C942B2B68
:1000C0000C942B2B0C942B2B0C942B2B0C942B2B58
:1000D0000C942B2B0C942B2B0C942B2B0C942B2B48
:1000E0000C942B2B9EB19EB1A5B1A5B1A5B1ACB11D
:1000F000ACB1ACB1B9B1B3B1B3B1B3B166BB69BB6B
:1001000058BB5CBB62BBA0BB6DBB71BB77BB7BBB91
:100110007FBB85BB89BB8DBBA0BB93BB97BB9BBB88
:10012000D4C0D9C0DEC0E8C0F2C06BC1FCC004C1FD
:100130000CC116C120C12AC139C143C16BC14DC117
:1001400057C161C1E000EC00D600EA00E600E4001F
:10015000DC00E400DA00D800E400E200084AD73B03
:100160003BCE016E84BCBFFDC12F3D6C74319ABD86
:1001700056833DDA3D00C77F11BED9E4BB4C3E91AA
:100180006BAAAABE000000803F05A84CCDB2D44E99
:10019000B93836A9020C50B9918688083CA6AAAA9B
:1001A0002ABE000000803F000D9490090D94AC150C
:1001B0000D94CB150D94C7150D94C3150D94880E91
:1001C0000D9495150D94D1150D94D4150D94BF155E
:1001D0000D94B5080D94B7150D949B154E414E49DD
:1001E0004E495459494E46CDCCCC3D0AD7233C17F5
:1001F000B7D13877CC2B329595E6241FB14F0A0042
:100200000020410000C84200401C4620BCBE4CCA31
:100210001B0E5AAEC59D74434F4D4D554E4943413B
:1002200054494F4E0044525952554E004552524F78
:10023000525300494E464F004543484F0020746FCB
:100240006F206C6F6E6720657874727573696F6E5E
:100250002070726576656E7465640A0020636F6C49
:100260006420657874727573696F6E20707265763C
:10027000656E7465640A0047322F473320626164FB
:1002800020706172616D65746572730A00205A3A5C
:10029000200020593A200042656420583A20004C42
:1002A000756C7A426F742054415A20362072656111
:1002B00064792E00526573756D696E67207072697E
:1002C0006E7400436C69636B20746F207265737584
:1002D0006D652E2E2E004E6F206D6F76652E0045BB
:1002E0006E642066696C65206C6973740A004265EF
:1002F00067696E2066696C65206C6973740A004DCD
:10030000313235005344207072696E74696E672013
:100310006279746520004E6F7420534420707269B6
:100320006E74696E670A0046696C652064656C6569
:100330007465643A0044656C6574696F6E2066612B
:10034000696C65642C2046696C653A20006F7065A5
:100350006E206661696C65642C2046696C653A2084
:10036000002569730025696D20256973002569687A
:100370002025696D20256973002569642025696839
:100380002025696D20256973002569792025696418
:10039000202569682025696D2025697300507269E0
:1003A0006E742074696D653A2000000125301D0CC3
:1003B0001824311C0B17232F1B0A1E1604030806D2
:1003C0000202222B1A4142033809FF362829452709
:1003D000444350726F7465637465642050696E0A9B
:1003E000004578747275646572202573004C756CD5
:1003F0007A426F742054415A2036207265616479C4
:100400002E00380233022C02250217026F666600A6
:1004100044454255473A006F6B00436F6F6C696EFD
:100420006720646F6E652E0048656174696E672091
:10043000646F6E652E0020573A00457874727564BB
:100440006572202573004C756C7A426F742054419C
:100450005A20362072656164792E004265642064FA
:100460006F6E652E0020573A004265642068656112
:1004700074696E672E0042656420636F6F6C696EED
:10048000672E004361703A454D455247454E4359EA
:100490005F5041525345523A310A004361703A432A
:1004A0004153455F4C494748545F4252494748547D
:1004B0004E4553533A300A004361703A544F474710
:1004C0004C455F4C49474854533A300A00436170E9
:1004D0003A534F4654574152455F504F5745523A51
:1004E000300A004361703A4C4556454C494E475FCF
:1004F000444154413A310A004361703A5A5F5052C4
:100500004F42453A310A004361703A4155544F4CCD
:100510004556454C3A310A004361703A5052494EB3
:10052000545F4A4F423A310A004361703A50524F89
:1005300047524553533A300A004361703A4155548B
:100540004F5245504F52545F54454D503A310A0076
:100550004361703A454550524F4D3A310A00464981
:10056000524D574152455F4E414D453A4D61726C77
:10057000696E20204649524D574152455F564552BB
:1005800053494F4E3A312E312E352E3735204558AE
:100590005452554445525F545950453A466C65781B
:1005A000797374727564657220534F555243455F79
:1005B000434F44455F55524C3A68747470733A2FF8
:1005C0002F636F64652E616C6570686F626A656326
:1005D00074732E636F6D2F646966667573696F6ED1
:1005E0002F4D41524C494E2050524F544F434F4C87
:1005F0005F56455253494F4E3A312E30204D4143BC
:1006000048494E455F545950453A4C756C7A426F93
:10061000742054415A20362045585452554445526E
:100620005F434F554E543A3120555549443A38347A
:100630003566303033632D616562642D3465353342
:100640002D613662392D3764303938346664653649
:1006500030390A002F2F20004D31343520533C69AA
:100660006E6465783E206F7574206F662072616ECF
:1006700067652028302D31290A00426564204C65C9
:1006800076656C696E6720004661696C65642074EC
:100690006F20656E61626C6520426564204C6576F2
:1006A000656C696E670A00426564204C6576656C0E
:1006B00020436F7272656374696F6E204D6174724E
:1006C00069783A004F666673657473206170706C68
:1006D000696564004572723A20546F6F20666172DA
:1006E0002100546F6F206661722066726F6D2072F8
:1006F00065666572656E636520706F696E740A0069
:100700003A20007A5F6D696E3A20202D32207A5FA0
:100710006D61783A202035005A204F666673657403
:1007200020004E6F2063617365206C696768740AEE
:1007300000416374697665204578747275646572EA
:100740003A2000556E6B6E6F776E20636F6D6D6132
:100750006E643A2022004D6F76652059004D6F7609
:1007600065205A004578747275646572004D6F7625
:100770006520302E316D6D004D6F766520316D6DC9
:10078000004D6F76652031306D6D004D6F766520C0
:1007900061786973004578747275646572004D6F95
:1007A0007665205A004D6F76652059004D6F76654D
:1007B0002058004578747275646572004D6F7665D7
:1007C000205A004D6F76652059004D6F7665205890
:1007D000004D6F76656D656E7400436F6F6C646F6E
:1007E000776E0046616E2073706565642031004647
:1007F000616E20737065656420310042656400425B
:100800006564004E6F7A7A6C65004E6F7A7A6C651B
:10081000004D61696E005654726176206D696E00FC
:100820005654726176206D696E005654726176205E
:100830006D696E00566D696E00566D696E00566D7D
:10084000696E00566D6178204500566D61782045CF
:1008500000566D6178204500566D6178205A00562B
:100860006D6178205A00566D6178205A00566D618E
:1008700078205900566D6178205900566D617820B6
:100880005900566D6178205800566D6178205800E7
:10089000566D61782058004D6F74696F6E00416D20
:1008A0006178204500416D6178204500416D617897
:1008B000205A00416D6178205A00416D61782059BD
:1008C00000416D6178205900416D617820580041E8
:1008D0006D6178205800412D74726176656C00411D
:1008E0002D74726176656C00412D7265747261635E
:1008F0007400412D726574726163740041636365B5
:100900006C00416363656C004D6F74696F6E0053DA
:100910006C6565702E2E2E005A2070726F626520F5
:100920006F75742E206265640A005A2070726F62BF
:1009300065206F75742E2062656400486F6D6520B8
:1009400058592066697273740A00486F6D652058A3
:10095000592066697273740020706F736974696FCF
:100960006E206F7574206F662072616E67652E0A47
:10097000003F50726F626520000A0A426564204C95
:100980006576656C20436F7272656374696F6E2063
:100990004D61747269783A00202B000A436F7272BD
:1009A000656374656420426564204865696768749E
:1009B0002076732E2042656420546F706F6C6F67D1
:1009C000793A0A00202B000A42656420486569676D
:1009D000687420546F706F6772617068793A0A208A
:1009E00020202B2D2D2D204241434B202D2D2B0A35
:1009F0002020207C20202020202020202020207C3F
:100A00000A204C207C20202020282B292020202058
:100A10007C20520A2045207C2020202020202020DD
:100A20002020207C20490A2046207C20282D2920B7
:100A30004E20282B29207C20470A2054207C20206F
:100A40002020202020202020207C20480A20202038
:100A50007C20202020282D29202020207C20540AA2
:100A60002020207C20202020202020202020207CCE
:100A70000A2020204F2D2D2046524F4E54202D2D40
:100A80002B0A2028302C30290A004D65616E206F1A
:100A9000662073616D706C656420706F696E74732D
:100AA0003A200020643A200020623A200045716E0E
:100AB00020636F656666696369656E74733A206169
:100AC0003A200052756E6E696E6720696E2044523E
:100AD000592D52554E206D6F64650A0047323920FA
:100AE0004175746F20426564204C6576656C696E53
:100AF000670A0028422961636B00284629726F6EDD
:100B000074002852296967687400284C2965667446
:100B1000003F4E756D626572206F662070726F6265
:100B20006520706F696E747320697320696D706CD5
:100B300061757369626C65202832206D696E696D1C
:100B4000756D292E0A003F2856296572626F7365FC
:100B5000206C6576656C20697320696D706C6175B9
:100B60007369626C652028302D34292E0A002575A2
:100B70003A2530327500253032753A25303275000D
:100B800025756420253032753A253032750000060F
:100B90000900FE000000000001090008FE00000539
:100BA000080806000040F0C88888987810050808F2
:100BB000060000C0F88888888888F80505050600C2
:100BC000012030F830200508080600002070F820C9
:100BD000202020E00509090600FF2070A8A8B88899
:100BE0008870200509090600FFE080C0B0A8283001
:100BF00028280509090600FFF8A88888888888A899
:100C0000F8050A0A0600FE205050505088A8A8880F
:100C10007003030306000340A04000060900FE071E
:100C20000192032120FFFF08FF07FF0000000600DC
:100C30000001070706020080808080800080030298
:100C400002060105A0A00507070600005050F85055
:100C5000F850500507070600002078A07028F02003
:100C6000050707060000C0C81020409818050707B0
:100C70000600006090A040A89068020303060104EB
:100C8000C04080030707060100204080808040208C
:100C9000030707060100804020202040800505054D
:100CA00006000120A870A8200505050600012020E7
:100CB000F820200203030602FFC040800501010660
:100CC0000003F8020202060200C0C0050505060086
:100CD00001081020408005070706000070888888FA
:100CE00088887003070706010040C040404040E08C
:100CF000050707060000708808708080F805070760
:100D0000060000F81020100808F00507070600008C
:100D100010305090F81010050707060000F880F01A
:100D200008088870050707060000708080F0888832
:100D300070050707060000F808102020202005078E
:100D4000070600007088887088887005070706000D
:100D50000070888878080870020505060200C0C087
:100D600000C0C00206060602FFC0C000C0408004EA
:100D700007070600001020408040201005030306EE
:100D80000002F800F8040707060100804020102048
:100D90004080050707060000708808102000200525
:100DA000070706000070880868A8A87005070706EE
:100DB0000000708888F8888888050707060000F01A
:100DC0008888F08888F00507070600007088808012
:100DD000808870050707060000F08888888888F0FA
:100DE000050707060000F88080F08080F8050707F7
:100DF000060000F88080F08080800507070600006C
:100E0000708880B888887005070706000088888881
:100E1000F88888880107070602008080808080802B
:100E200080050707060000381010101090600507B5
:100E3000070600008890A0C0A0908805070706005C
:100E400000808080808080F805070706000088D831
:100E5000A8888888880507070600008888C8A89899
:100E600088880507070600007088888888887005CC
:100E70000707060000F08888F080808005070706D5
:100E8000000070888888A89068050707060000F0B1
:100E90008888F0A090880507070600007880807099
:100EA0000808F0050707060000F820202020202071
:100EB0000507070600008888888888887005070766
:100EC00006000088888888885020050707060000EB
:100ED0008888888888A850050707060000888850F9
:100EE0002050888805070706000088888850202041
:100EF00020050707060000F80810204080F80307C7
:100F000007060100E08080808080E005050506007E
:100F1000018040201008030707060100E020202080
:100F20002020E00503030600042050880501010687
:100F30000000F802020206020580400505050600D1
:100F40000070087888780507070600008080B0C820
:100F50008888F00505050600007080808870050708
:100F600007060000080868988888780505050600C7
:100F7000007088F880700507070600003048E040E0
:100F80004040400506060600FF7088887808700516
:100F900007070600008080B0C88888880107070618
:100FA0000200800080808080800308080601FF2006
:100FB0000020202020A04004070706000080809029
:100FC000A0C0A090030707060100C0404040404079
:100FD000E0050505060000D0A8A8A8A80505050697
:100FE0000000B0C88888880505050600007088885C
:100FF00088700506060600FFF08888F080800506E8
:10100000060600FF788888780808050505060000B0
:10101000B0C880808005050506000070807008F06B
:101020000407070600004040E04040403005050549
:1010300006000088888898680505050600008888ED
:101040008850200505050600008888A8A8500505D9
:101050000506000088502050880506060600FF8817
:101060008888780870050505060000F8102040F80B
:101070000307070601002040408040402001070789
:1010800006020080808080808080030707060100C0
:101090008040402040408005020206000268900027
:1010A000000006000000000006000000000006002E
:1010B0000000000006000000000006000000000024
:1010C000060000000000060000000000060000000E
:1010D00000000600000000000600000000000600FE
:1010E00000000000060000000000060000000000F4
:1010F00006000000000006000000000006000000DE
:1011000000000600000000000600000000000600CD
:1011100000000000060000000000060000000000C3
:1011200006000000000006000000000006000000AD
:10113000000006000000000006000000000006009D
:101140000000000006000000000006000000000093
:10115000060000000000060000000000060000007D
:10116000000006000000000006000001070706025C
:1011700000800080808080800507070600002070C6
:10118000A8A0A87020050707060000304040E040F6
:1011900050A80505050600008870507088050707EF
:1011A000060000885020F820F820010707060200FA
:1011B000808080008080800508080600003048207C
:1011C0005050209060030101060107A005070706A3
:1011D0000000F888B8B8B888F8050707060001705D
:1011E0000878887800F80505050600012850A05009
:1011F00028050303060001F8080802020206020699
:101200004080050707060000F888A88898A8F80518
:101210000101060006F804040406000360909060D3
:101220000507070600002020F8202000F804050527
:1012300006000360902040F0030505060003E0204F
:10124000E020E002020206020640800508080600CF
:10125000FF8888888898E88080050707060000785E
:10126000989878181818020202060202C0C00202FA
:10127000020602FF408003050506000340C040400F
:10128000E0050707060001708888887000F80505EA
:1012900005060001A0502850A00507070600008899
:1012A00090A858B808080507070600008890B848B5
:1012B000982038050808060000C040C048D8380803
:1012C00008050707060000200020408088700508F8
:1012D000080600004020007088F888880508080685
:1012E00000001020007088F88888050808060000B3
:1012F0002050007088F8888805080806000068906B
:10130000007088F88888050808060000500070887A
:1013100088F888880508080600002050207088F8A2
:1013200088880507070600003860A0B8E0A0B80567
:1013300008080600FF708880808870206005080813
:10134000060000402000F880F080F805080806003C
:1013500000081000F880F080F8050808060000205A
:101360005000F880F080F80507070600005000F8EC
:1013700080F080F8030808060100804000E040404B
:1013800040E0030808060100204000E0404040E043
:1013900003080806010040A000E0404040E00307C9
:1013A00007060100A000E0404040E00507070600F6
:1013B00000704848E8484870050808060000689032
:1013C0000088C8A898880508080600004020708892
:1013D00088888870050808060000102070888888B2
:1013E0008870050808060000205000708888887002
:1013F0000508080600006890007088888870050855
:101400000806000050007088888888700505050669
:10141000000188502050880508080600FF1070A8B9
:10142000A8A8A87040050808060000402088888801
:101430008888700508080600001020888888888839
:10144000700508080600002050008888888870050C
:1014500008080600005000888888888870050808F9
:1014600006000010208850202020200509090600D1
:10147000FFC040704848704040E00408080601FF83
:10148000609090A09090E080050808060000402041
:1014900000700878887805080806000010200070A1
:1014A0000878887805080806000020500070087841
:1014B0008878050808060000689000700878887829
:1014C00005070706000050007008788878050808AE
:1014D000060000205020700878887805060606006F
:1014E00000D02878A0A8500506060600FF70808866
:1014F0007020600508080600004020007088F88011
:10150000700508080600001020007088F88070053B
:1015100008080600002050007088F8807005070752
:1015200006000050007088F880700308080601006B
:1015300080400040C04040E0030808060100204011
:101540000040C04040E003080806010040A0004001
:10155000C04040E0030707060100A00040C0404033
:10156000E0050707060000A040A010788870050875
:1015700008060000689000B0C8888888050808063A
:101580000000402000708888887005080806000068
:101590001020007088888870050808060000205018
:1015A0000070888888700508080600006890007040
:1015B00088888870050707060000500070888888B2
:1015C000700505050600012000F800200507070644
:1015D00000FF1070A8A8A870400508080600004089
:1015E00020008888889868050808060000102000F8
:1015F00088888898680508080600002050008888B8
:101600008898680507070600005000888888986851
:101610000509090600FF102000888888F808700472
:1016200007070601FFC04060506040E0050808065B
:1016300000FF50008888887808705A0059005800C8
:101640000920000000000000000000000000007FF2
:10165000FFE000000000000000000000000070003B
:10166000E000000000000000000000000061F860E1
:1016700000000000000000000000000041F8200011
:10168000000000000000000000000040F02000000A
:10169000000000000000000000004060200000008A
:1016A0000000000000000000005801A07F80000042
:1016B00000000000004104005C63A0FFC0000000C7
:1016C000000000002082005EF7A0FFC000000000C4
:1016D0000000002082005EF7A0FFC00000000000B4
:1016E00000004104005C63A07F8000000000000057
:1016F000008208005801A07F800000000000000167
:10170000041000406020FFC0000000000000010441
:10171000100040F020FFC000000000000000820820
:101720000041F820FFC0000000000000004104005C
:1017300061F8603F00000000000000000000007041
:1017400000E01E0000000000000001FFFF807FFF9E
:10175000E00C0000000000000001FFFF800000001E
:101760000000000000000000000000007FFFE0001B
:1017700000000000000000000000007000E0000019
:1017800000000000000000000000630C600000008A
:10179000000000000000000000470E2000000000D4
:1017A00000000000000000004F0F200000000000BB
:1017B000000000000000005F0FA00000000000001B
:1017C0000000000000005E07A07F80000000000015
:1017D0000000410400406020FFC000000000000045
:1017E0000020820040F020FFC00000000000000048
:1017F00020820040F020FFC00000000000000041F7
:1018000004004060207F800000000000000082088B
:10181000005E07A07F8000000000000001041000AF
:101820005F0FA0FFC0000000000000010410004F87
:101830000F20FFC000000000000000820800470EDB
:1018400020FFC000000000000000410400630C60A5
:101850003F00000000000000000000007000E01EDB
:101860000000000000000001FFFF807FFFE00C008F
:1018700000000000000001FFFF80000000205A3A35
:101880000020593A0020436F756E7420583A0020AA
:10189000453A00205A3A0020593A00583A00536518
:1018A0007474696E672054726176656C204163635D
:1018B000656C65726174696F6E3A2000536574746B
:1018C000696E672052657472616374204163636559
:1018D0006C65726174696F6E3A2000536574746947
:1018E0006E67205072696E7420416363656C657227
:1018F0006174696F6E3A200053657474696E672075
:101900005072696E7420616E642054726176656CE9
:1019100020416363656C65726174696F6E3A200083
:10192000205A00205900580020204D61783A2000AC
:10193000205A00205900580020204D696E3A20009E
:101940004F6E20004F666600536F667420656E64AC
:1019500073746F70733A200020643A0020693A0073
:1019600020703A0020643A0020693A0020703A0062
:1019700043290A0061626C656420286D696E2074D9
:10198000656D702000436F6C6420657874727564B7
:1019900065732061726520004B64200023646566D6
:1019A000696E65202044454641554C545F004B69A3
:1019B000200023646566696E6520204445464155D4
:1019C0004C545F004B70200023646566696E65208F
:1019D0002044454641554C545F00504944204175D0
:1019E000746F74756E652066696E697368656421CD
:1019F0002050757420746865206C617374204B707E
:101A00002C204B6920616E64204B6420636F6E73E1
:101A100074616E74732066726F6D2062656C6F778F
:101A200020696E746F20436F6E66696775726174AA
:101A3000696F6E2E680A00504944204175746F74B6
:101A4000756E65206661696C6564212074696D65D9
:101A50006F75740A00504944204175746F74756E37
:101A600065206661696C6564212054656D706572DE
:101A7000617475726520746F6F20686967680A0009
:101A8000204B643A2000204B693A2000204B703AEA
:101A900020000A20436C617373696320504944201D
:101AA0000A002054753A2000204B753A2000206D22
:101AB00061783A2000206D696E3A200020643A2057
:101AC0000020626961733A20001FFFFFFFFFFFFFE4
:101AD000600000000001FF400000000000FF8000E7
:101AE000000000007F83CF00000C303F87FF8000A4
:101AF0000C301F867980000C000F8C30C7838C302F
:101B0000E78C30CFC7CC31F38C30DCECEC33B98CC4
:101B100030D86C6C33198C30D06C0C33198C30D8B5
:101B20006C0C33198C30DC6C0E3B198C30CF7C077D
:101B30009F198C30C77C038F194000000000000201
:101B4000600000000000061FFFFFFFFFFFF82020DD
:101B5000506C616E6E65724275666665724279742C
:101B600065733A20002046726565204D656D6F7281
:101B7000793A2000436F6D70696C65643A204A6160
:101B80006E20333020323031380A00207C204175FD
:101B900074686F723A2028416C657068204F626AE1
:101BA0006563747320496E632E2C204C756C7A42E9
:101BB0006F7420476974205265706F7369746F7217
:101BC00079290A004A616E203330203230313830B2
:101BD000393A30363A333500204C617374205570F1
:101BE00064617465643A2000312E312E350A004D4F
:101BF00061726C696E0020536F6674776172652044
:101C000052657365740A00205761746368646F6776
:101C10002052657365740A002042726F776E206FE0
:101C200075742052657365740A0020457874657276
:101C30006E616C2052657365740A00506F7765722F
:101C400055700A0073746172740A006572726F7263
:101C50002077726974696E6720746F2066696C659D
:101C60000A00456E6473746F7073202563202563CA
:101C70002025632025630020503A00205A3A002096
:101C8000593A0020583A00656E6473746F7073207F
:101C90006869743A2000446F6E6520736176696EDE
:101CA000672066696C652E0A004D32390020746F1A
:101CB0006F206C6F6E6720657874727573696F6ED4
:101CC0002070726576656E7465640A0020636F6CBF
:101CD0006420657874727573696F6E2070726576B2
:101CE000656E7465640A007C3C3E5E2B3D3F2F5B55
:101CF0005D3B2C2A225C001000C90210012C01401F
:101D000001220170011801B0010E01F0010401501F
:101D100002FA00B002F0003003E600D003DC0090CD
:101D200004D2007005C800A006BE000008B400B0D0
:101D300009AA00D00BA000600E960060118C000074
:101D400015820020197800C01D6E00A0226400B02A
:101D5000275A00902C500000314600E0343C00101F
:101D6000383200903A2800603C1E00A03D140080EC
:101D70003E0A00203F000048656174696E67206676
:101D800061696C6564204245440048656174696E10
:101D900067206661696C65640048656174696E6797
:101DA000206661696C65640048656174696E6720CE
:101DB0006661696C6564204530001000AD03300138
:101DC0006A0150022B0170030A019004F500B0056E
:101DD000E500D006D800F007CE001009C500300A93
:101DE000BE00500BB700700CB100900DAB00B00EF0
:101DF000A600D00FA200F0109D0010129900301321
:101E000095005014920070158E0090168B00B0173C
:101E10008700D0188400F0198100101B7E00301C50
:101E20007B00501D7900701E7600901F7300B0205B
:101E30007000D0216E00F0226B0010246900302564
:101E40006600502663007027610090285E00B0296C
:101E50005C00D02A5900F02B5600102D5400302E73
:101E60005100502F4E0070304B0090314800B0327E
:101E70004500D0334200F0343E0010363B0030378E
:101E800037005038330070392E00903A2900B03BAB
:101E90002300D03C1B00F03D1100103F0100F03F3B
:101EA00000004572723A204D494E54454D50204233
:101EB0004544004D494E54454D5020747269676742
:101EC00065726564004572723A204D494E54454D25
:101ED00050204531004572723A204D494E54454DCF
:101EE00050204530004572723A204D415854454DBE
:101EF0005020424544004D415854454D5020747285
:101F000069676765726564004572723A204D415891
:101F100054454D50204531004572723A204D41588C
:101F200054454D50204530004572726F72207772D3
:101F30006974696E6720746F20454550524F4D217A
:101F40000A00290A002062797465733B206372637A
:101F5000200053657474696E67732053746F7265E3
:101F600064202800202863616C63756C617465646B
:101F700029210A0020213D2000454550524F4D2087
:101F8000435243206D69736D61746368202D20286E
:101F900073746F726564292000290A0020627974C5
:101FA00065733B2063726320002073746F726564F5
:101FB0002073657474696E677320726574726965E5
:101FC000766564202800204D61726C696E3D563440
:101FD00030290A0028454550524F4D3D0045455097
:101FE000524F4D2076657273696F6E206D69736D07
:101FF00061746368200048617264636F6465642083
:1020000044656661756C742053657474696E67739A
:10201000204C6F616465640A0028230000282300B7
:1020200000640000001027000000009643000096A6
:1020300043000040400000C8410000C9420000C900
:10204000420000C84400804F4420204D38353120E4
:102050005A005A2D50726F6265204F666673657420
:1020600020286D6D293A0A002044002049002020D4
:102070004D33303420500020440020490020204DB2
:102080003330312050005049442073657474696EB8
:1020900067733A0A002046002042002048002020B2
:1020A0004D3134352053004D6174657269616C2087
:1020B00068656174757020706172616D65746572B8
:1020C000733A0A0020204D34323020530041757499
:1020D0006F20426564204C6576656C696E673A0ACC
:1020E00000205A0020590020204D32303620580060
:1020F000486F6D65206F66667365743A0A00204507
:1021000000205A002059002058002042002054008E
:1021100020204D323035205300416476616E636576
:10212000643A20533C6D696E5F66656564726174E4
:10213000653E20543C6D696E5F74726176656C5FBC
:1021400066656564726174653E20423C6D696E5FD0
:102150007365676D656E745F74696D655F6D733E01
:1021600020583C6D61785F78795F6A65726B3E20BC
:102170005A3C6D61785F7A5F6A65726B3E20453CC0
:102180006D61785F655F6A65726B3E0A002054007E
:1021900020520020204D32303420500041636365CE
:1021A0006C65726174696F6E2028756E6974732F27
:1021B0007332293A20503C7072696E745F616363B8
:1021C000656C3E20523C726574726163745F61633A
:1021D00063656C3E20543C74726176656C5F61632C
:1021E00063656C3E0A00204500205A0020590020FB
:1021F000204D3230312058004D6178696D756D2069
:10220000416363656C65726174696F6E2028756ED9
:102210006974732F7332293A0A00204500205A004E
:1022200020590020204D3230332058004D6178690C
:102230006D756D20666565647261746573202875BF
:102240006E6974732F73293A0A00204500205A00E2
:1022500020590020204D3932205800537465707386
:102260002070657220756E69743A0A0020204D3224
:1022700030302044300A0020204D323030204400DD
:102280002044697361626C65640A0046696C616D23
:10229000656E742073657474696E67733A002020EC
:1022A0004D3134392043203B20556E6974732069C9
:1022B0006E2043656C736975730A002020473231C4
:1022C000202020203B20556E69747320696E206D9C
:1022D0006D0A0000000A0B02090C0D0E080703042A
:1022E00001000000000000000000000000000000ED
:1022F00000000000000000000000000000000012CC
:1023000011100000000000000000000000000000AC
:10231000000000000000000000486F6D652025737C
:102320002573257320666972737400206669727361
:10233000740A005A0059005800486F6D6520005318
:10234000442063617264206F6B0A006F70656E5287
:102350006F6F74206661696C65640A00766F6C75D6
:102360006D652E696E6974206661696C65640A002A
:10237000534420696E6974206661696C0A00617556
:10238000746F25692E67004D3234004D323320259D
:10239000730057726974696E6720746F2066696C88
:1023A000653A20006F70656E206661696C65642C0B
:1023B0002046696C653A20006F70656E2066616921
:1023C0006C65642C2046696C653A200046696C6532
:1023D0002073656C65637465640A002053697A65CF
:1023E0003A200046696C65206F70656E65643A201E
:1023F000006F70656E206661696C65642C204669AB
:102400006C653A20002066696C653A20004E6F7753
:1024100020002220706F73002220706172656E743C
:102420003A2200535542524F5554494E452043419C
:102430004C4C207461726765743A22004B494C4CD5
:1024400045442E2000747279696E6720746F206392
:10245000616C6C207375622D67636F6465206669BB
:102460006C6573207769746820746F6F206D616E7E
:1024700079206C6576656C732E204D4158206C6513
:1024800076656C2069733A004572726F723A004E3D
:102490006F204C696E65204E756D6265722077699C
:1024A000746820636865636B73756D2C204C617371
:1024B00074204C696E653A200053544F5050454487
:1024C0002E20005072696E7465722073746F707084
:1024D00065642064756520746F206572726F727315
:1024E0002E2046697820746865206572726F7220AC
:1024F000616E6420757365204D39393920746F2001
:10250000726573746172742E202854656D706572E3
:1025100061747572652069732072657365742E200D
:1025200053657420697420616674657220726573E6
:1025300074617274696E67290A004E6F2043686582
:10254000636B73756D2077697468206C696E6520A4
:102550006E756D6265722C204C617374204C696ECF
:10256000653A2000636865636B73756D206D6973F0
:102570006D617463682C204C617374204C696E65C6
:102580003A20004C696E65204E756D626572206957
:1025900073206E6F74204C617374204C696E6520DB
:1025A0004E756D6265722B312C204C617374204C1A
:1025B000696E653A20004D313130004D3331004DA8
:1025C000383420582059205A204500534420726541
:1025D0006164206572726F720A00446F6E652070CC
:1025E00072696E74696E672066696C650A002049BD
:1025F0006E76616C696420657874727564657220AA
:10260000000000D8C10000A0C10000000000009040
:10261000430000974300008743000020002300266A
:102620000029002C002F00320000010000030106E9
:1026300001090143616E6E6F74206F70656E2073C7
:10264000756264697220006563686F3A005448459A
:10265000524D414C2052554E41574159204245441C
:1026600000546865726D616C2052756E6177617996
:1026700000544845524D414C2052554E4157415906
:1026800020453100544845524D414C2052554E4151
:102690005741592045300000002200250028002B1A
:1026A000002E003100340002010000050108010B7A
:1026B0000100002100240027002A002D00300033F3
:1026C0000001010000040107010A010505050507D5
:1026D0000508080808020202020A0A08080404049D
:1026E00004010101010101010103030303030303C9
:1026F00003040707070C0C0C0C0C0C0C0C02020258
:102700000206060606060606060B0B0B0B0B0B0B4A
:102710000B010210202008081020401020408002E9
:102720000102010804020101020408102040808017
:10273000402010080402018004020180402010089B
:102740000402010804020101020408102040800173
:1027500002040810204080506C656173652072652A
:10276000736574005052494E5445522048414C54B0
:102770004544005072696E7465722068616C7465BE
:10278000642E206B696C6C28292063616C6C656415
:10279000210A00656E7175657565696E6720220096
:1027A0000000D8C10000974300000000000048422C
:1027B0000000484200004040000000005761726E77
:1027C000696E673A20486F6D696E672042756D705B
:1027D0002044697669736F72203C20310A0002023E
:1027E000040000A0400000A0400000004000809DC8
:1027F000430000A14300008743FF01FF4D36303006
:1028000020486F74656E6420746F6F20636F6C6412
:1028100020746F206368616E67652066696C616D06
:10282000656E740A0000060900FE06018902FE209A
:10283000FFFE07FE06FE0000000600070106060672
:102840000200808080800080030303060103A0A0B3
:10285000A00507070600FF5050F850F85050050932
:10286000090600FE2070A8A07028A870200608089D
:102870000600FF40A8481020485408050707060036
:10288000FF609090609890680103030602038080C7
:10289000800207070602FF40808080808040020798
:1028A000070602FF804040404040800505050600C5
:1028B000008850F850880505050600002020F82003
:1028C000200204040602FEC040408005010106000B
:1028D00002F8020202060200C0C004060606010059
:1028E0001010204080800406060601006090909041
:1028F000906003060606010040C0404040E0040628
:10290000060601006090102040F004060606010053
:10291000F020601010E00506060600001030509010
:10292000F810040606060100F080E01010E004062E
:10293000060601006080E090906004060606010033
:10294000F0101020404004060606010060906090E0
:102950009060040606060100609090701060020509
:1029600005060200C0C000C0C00207070602FEC084
:10297000C000C0404080050505060000186080606A
:1029800018050303060001F800F805050506000018
:10299000C0300830C0040707060100609010604096
:1029A00000400506060600007090A8B0807005067D
:1029B00006060000205088F88888050606060000F4
:1029C000F088F08888F00406060601006090808098
:1029D0009060040606060100E090909090E00406E6
:1029E00006060100F080E08080F004060606010083
:1029F000F080E0808080040606060100609080B0D0
:102A000090600406060601009090F09090900306F6
:102A100006060100E040404040E0050606060000D2
:102A200038101010906004060606010090A0C0A0A7
:102A300090900406060601008080808080F00506E4
:102A40000606000088D8A8A88888040606060100A3
:102A500090D0B09090900506060600007088888897
:102A60008870040606060100E09090E0808004076C
:102A7000070601FF609090D0B060100406060601C2
:102A800000E09090E09090040606060100609040FF
:102A9000209060050606060000F820202020200473
:102AA00006060601009090909090600406060601CC
:102AB00000909090F060600506060600008888A8E7
:102AC000A8D88805060606000088502020508805F2
:102AD000060606000088885020202004060606010D
:102AE00000F010204080F0030606060100E0808020
:102AF0008080E0040606060100808040201010035C
:102B00000606060100E020202020E0050303060061
:102B1000032050880501010600FEF80202020602A9
:102B200004804004040406010070909070040606BE
:102B30000601008080E09090E0040404060100702B
:102B400080807004060606010010107090907004DA
:102B5000040406010060B0C07004060606010020EF
:102B60005040E040400406060601FE609090701060
:102B7000600406060601008080E09090900306063F
:102B80000601004000C04040E00308080601FE20A6
:102B90000060202020A0400406060601008080A0DE
:102BA000C0A090030606060100C040404040E0057A
:102BB0000404060000D0A8A888040404060100E06C
:102BC0009090900404040601006090906004060652
:102BD0000601FEE09090E080800406060601FE708B
:102BE0009090701010040404060100A0D0808004AE
:102BF000040406010070C030E0040606060100402F
:102C000040E04050200404040601009090907004BD
:102C1000040406010090906060050404060000882A
:102C2000A8A8500404040601009060609004060601
:102C30000601FE909090709060040404060100F07C
:102C40002040F0030707060100204040804040205C
:102C50000107070602FF80808080808080030707CD
:102C6000060100804040204040800402020601032B
:102C700050A0FFFFFFFFFFFFFFFFFFFFFFFFFFFF72
:102C8000FFFFFFFFFFFFFFFFFFFFFFFFFFFFFFFF54
:102C9000FFFFFF0000000600070106060602008095
:102CA00000808080800406060601FF2070A0A070CE
:102CB000200507070600FF304840F04040F80505B2
:102CC00005060000A8508850A805060606000088E2
:102CD00050F820F8200107070602FF80808000805E
:102CE00080800407070601FF708060906010E00399
:102CF0000101060105A0060707060000788494A4D8
:102D000094847803050506010160A06000E00505D4
:102D1000050600002850A05028040303060100F017
:102D20001010040101060102F006070706000078F2
:102D300084B4A4A48478040101060105F00403030B
:102D40000601026090600507070600FF2020F820BA
:102D50002000F803050506010140A02040E003051E
:102D600005060101C0204020C00202020602044004
:102D7000800405050601FF9090B0D0800506060688
:102D8000000078E8E86828280101010602028002B4
:102D900002020602FE408003050506010140C04014
:102DA00040E003050506010140A04000E0050505DF
:102DB000060000A0502850A00508080600FF40C0EB
:102DC0004050703078100508080600FF40C04050A1
:102DD000680810380508080600FFC0204030F030B1
:102DE000781004070706010020002060809060052D
:102DF0000707060000402020507088880507070656
:102E00000000102020507088880507070600002069
:102E10005020507088880507070600002850205071
:102E200070888805070706000050002050708888C9
:102E30000507070600002050205070888805060608
:102E400006000078A0F0A0A0B80408080601FE6003
:102E5000908080906020400407070601004020F029
:102E600080E080F00407070601002040F080E08049
:102E7000F00407070601002050F080E080F004070E
:102E8000070601005000F080E080F003070706010C
:102E9000008040E0404040E003070706010020407A
:102EA000E0404040E003070706010040A0E040404A
:102EB00040E0030707060100A000E0404040E005B5
:102EC00006060600007048E8484870040707060137
:102ED0000050A090D0B09090040707060100402059
:102EE0006090909060040707060100204060909079
:102EF00090600407070601002050609090906004E5
:102F0000070706010050A060909090600407070634
:102F10000100500060909090600505050600008853
:102F2000502050880408080601FF1070B0B0D0D0BF
:102F3000E080040707060100402090909090600414
:102F40000707060100204090909090600407070654
:102F500001002050909090906004070706010050F7
:102F600000909090906005070706000010208850A0
:102F700020202004060606010080E09090E08004F6
:102F800006060601006090A0A090A00407070601B5
:102F90000040200070909070040707060100204058
:102FA0000070909070040707060100205000709098
:102FB000907004070706010050A000709090700404
:102FC0000606060100500070909070040707060185
:102FD000002050207090907005040406000070A836
:102FE000B0780406060601FE708080702040040759
:102FF0000706010040200060B0C07004070706010A
:103000000020400060B0C070040707060100205097
:103010000060B0C070040606060100500060B0C039
:1030200070030707060100804000C04040E003072E
:1030300007060100204000C04040E00307070601EA
:103040000040A000C04040E0030606060100A000CA
:10305000C04040E004070706010030601070909007
:103060006004070706010050A000E090909004075C
:1030700007060100402000609090600407070601E9
:103080000020400060909060040707060100205077
:10309000006090906004070706010050A000609057
:1030A00090600406060601005000609090600505DF
:1030B000050600002000F80020040404060100704A
:1030C000B0D0E00407070601004020009090907007
:1030D0000407070601002040009090907004070745
:1030E0000601002050009090907004060606010032
:1030F0005000909090700409090601FE2040009055
:1031000090907090600408080601FE8080E0909026
:10311000E080800408080601FE50009090907090B6
:10312000607A5F70726F62653A20007A5F6D6178D5
:103130003A20007A5F6D696E3A2000795F6D6178A0
:103140003A2000795F6D696E3A2000785F6D617892
:103150003A2000785F6D696E3A20005265706F7298
:1031600074696E6720656E6473746F702073746128
:103170007475730A0056652D6A65726B0056652D6D
:103180006A65726B0056652D6A65726B00567A2D02
:103190006A65726B00567A2D6A65726B0056792DDE
:1031A0006A65726B0056792D6A65726B0056792DCF
:1031B0006A65726B0056782D6A65726B0056782DC1
:1031C0006A65726B0056782D6A65726B004D6F747C
:1031D000696F6E004573746570732F6D6D00457374
:1031E000746570732F6D6D005A73746570732F6DF5
:1031F0006D005A73746570732F6D6D00597374652B
:1032000070732F6D6D005973746570732F6D6D0041
:103210005873746570732F6D6D0058737465707397
:103220002F6D6D004D6F74696F6E004F6666004FB5
:103230006E2000456E6473746F702061626F7274EB
:103240000053746570732F6D6D004A65726B004199
:103250006363656C65726174696F6E0056656C6F4F
:1032600063697479005A204F66667365740041641F
:1032700076616E6365642053657474696E6773006C
:1032800043616E6E6F7420656E7465722073756233
:103290006469723A2000022E2E004D61696E00248E
:1032A000F4D43050C38E20C2A24017828B7011120A
:1032B0007A910D816CD90AA861E108C75866076147
:1032C0005143061E4B5D05C145A7041A411104096F
:1032D0003D9803713931034036DB0265339102D4E6
:1032E000305402802E1D02632CEE01752AC501B0F8
:1032F00028A001102781018F2564012B244B01E0B8
:10330000223401AC211F018D200D01801FFC00849F
:103310001EED00971DDF00B81CD200E61BC6002082
:103320001BBC00641AB200B219A8000A19A0006AF6
:10333000189900D117910040178B00B51684003101
:10334000167E00B31579003A157300C7146F005844
:10335000146A00EE1366008813630025135E00C72D
:10336000125B006C12570015125400C1115100700D
:10337000114F0021114B00D61049008D1047004617
:1033800010440002104200C00F4000800F3E004277
:103390000F3C00060F3B00CB0E3800930E37005C4D
:1033A0000E3500270E3400F30D3200C10D310090B0
:1033B0000D3000600D2E00320D2D00050D2C00D9B2
:1033C0000C2B00AE0C2900850C29005C0C27003565
:1033D0000C27000E0C2600E80B2400C40B2400A0D0
:1033E0000B23007D0B23005A0B2100390B21001801
:1033F0000B2000F80A1F00D90A1E00BB0A1E009D00
:103400000A1D00800A1D00630A1C00470A1B002CCD
:103410000A1B00110A1A00F7091A00DD091900C475
:10342000091900AB091900920917007B09180063FC
:103430000917004C09160036091600200916000A63
:10344000091500F5081500E0081400CC081400B8B0
:10345000081400A4081400900813007D0812006BE3
:1034600008130058081200460812003408110023FF
:103470000811001208110001081100F0071000E007
:10348000071000D0071000C0071000B0070F00A100
:1034900007100091070E0083070F0074070F0065E7
:1034A000070E0057070E0049070E003B070D002EC0
:1034B000070E0020070D0013070D0006070D00F989
:1034C000060C00ED060D00E0060C00D4060C00C84A
:1034D000060C00BC060C00B0060C00A4060B0099FC
:1034E000060C008D060B0082060B0077060B006CA5
:1034F000060B0061060A0057060B004C060A004244
:10350000060A0038060A002E060A0024060A001AD7
:10351000060A001006090007060A00FD050900F466
:10352000050900EB050900E2050900D9050900D0ED
:10353000050900C7050900BE050900B5050800AD6D
:10354000050800A50509009C050800940508008CE5
:10355000050800840508007C050800740508006C57
:10356000050700650508005D050700560508004EC3
:10357000050700470507004005080038050700312A
:103580000507002A050700230507001C050600168D
:103590000507000F0507000805060002050700FBE8
:1035A000040600F5040700EE040600E8040600E245
:1035B000040700DB040600D5040600CF040600C99A
:1035C000040600C3040600BD040600B7040600B1EB
:1035D000040500AC040600A6040600A00405009B38
:1035E00004060095040500900406008A0405008581
:1035F000040500800406007A0405007504050070C7
:103600000405006B04050066040500610405005C08
:1036100004050057040500520405004D0405004848
:10362000040500430405003E0404003A0405003587
:10363000040500300404002C0405002704040023C2
:103640000405001E0404001A0404001604050011F9
:103650000404000D0404000904050004040400002F
:10366000040400FC030400F8030400F4030400F065
:10367000030400EC030400E8030400E4030400E096
:10368000030400DC030400D8030400D4030400D0C6
:10369000030400CC030400C8030300C50303002493
:1036A000F404D9201BC40C5C0E9804C4095F0265A5
:1036B000077101F405F900FB04B30048048700C159
:1036C0000369005803550003034500BE023A008415
:1036D00002310053022A002902250004022000E4DE
:1036E000011C00C8011900AF0117009801140084E3
:1036F000011300710110006101100051010E00431F
:10370000010D0036010B002B010B0020010B0015F1
:103710000109000C01090003010800FB000800F387
:10372000000800EB000700E4000600DE000600D8F9
:10373000000600D2000600CC000500C7000500C24C
:10374000000500BD000400B9000400B5000400B18C
:10375000000400AD000400A9000400A5000300A2BD
:103760000003009F0004009B0003009800030095E5
:1037700000020093000300900003008D0002008B04
:10378000000300880002008600020084000300811C
:103790000002007F0002007D0002007B0002007931
:1037A000000200770001007600020074000200723F
:1037B000000100710002006F0002006D0001006C4A
:1037C0000002006A00010069000200670001006653
:1037D0000001006500010064000200620001006158
:1037E000000100600001005F0002005D0001005C5C
:1037F0000001005B0001005A00010059000100585F
:10380000000100570001005600010055000100545E
:10381000000100530000005300010052000100515C
:10382000000100500001004F0001004E0000004E5A
:103830000001004D0001004C0001004B0000004B56
:103840000001004A00010049000100480000004852
:10385000000100470001004600000046000100454D
:103860000000004500010044000100430000004347
:103870000001004200000042000100410000004140
:10388000000100400001003F0000003F0001003E39
:103890000000003E0001003D0000003D0001003C32
:1038A0000000003C0000003C0001003B0000003B29
:1038B0000001003A0000003A000100390000003920
:1038C0000001003800000038000000380001003717
:1038D000000000370001003600000036000000360E
:1038E0000001003500000035000000350001003403
:1038F00000000034000000340001003300000033F9
:1039000000000033000100320000003200000032ED
:1039100000010031000000310000003100010030E2
:1039200000000030000000300001002F0000002FD8
:103930000000002F0000002F0001002E0000002ECC
:103940000000002E0001002D0000002D0000002DC1
:103950000000002D0001002C0000002C0000002CB5
:103960000000002C0001002B0000002B0000002BA9
:103970000000002B0001002A0000002A0000002A9D
:103980000000002A00010029000000290000002991
:103990000000002900000029000100280000002884
:1039A0000000002800000028000000280001002777
:1039B000000000270000002700000027000000276B
:1039C000000100260000002600000026000000265E
:1039D0000000002600010025000000250000002551
:1039E0000000002500000025000000250001002443
:1039F0000000002400000024000000240000002437
:103A00000001002300000023000000230000002329
:103A1000000000230000002300000023000100221A
:103A2000000000220000002200000022000000220E
:103A30000000002200010021000000210000002100
:103A400000000021000000210000002100000021F2
:103A500000010020000000200000002000000020E5
:103A600000000020000000200000002000000020D6
:103A70000001001F0000001F0000001F0000001FC9
:103A80000000001F0000001F0000001F0001001EBA
:103A90000000001E0000001E0000001E0000004D7F
:103AA000383420582059205A20450020204E6F7A63
:103AB0007A6C653A200020004261636B004D696EAC
:103AC000696D756D2054656D7020697320313230D9
:103AD0002E0048656174696E67206661696C656473
:103AE0000045787472756465206D6F72650052656B
:103AF00073756D65207072696E7400524553554D33
:103B000045204F5054494F4E533A0020204E6F7A73
:103B10007A6C653A20006368616E6765006F6620A5
:103B20007468652066696C616D656E7400576169C3
:103B30007420666F72207374617274005052494E23
:103B400054205041555345440020204E6F7A7A6CE2
:103B5000653A2000200066696C616D656E742075A1
:103B60006E6C6F6164005761697420666F720050FB
:103B700052494E54205041555345440020204E6F29
:103B80007A7A6C653A20002000506C65617365207C
:103B9000776169742E2E2E0048656174696E672006
:103BA0006E6F7A7A6C65005052494E5420504155E0
:103BB0005345440020204E6F7A7A6C653A200020ED
:103BC0000068656174206E6F7A7A6C652E005072A1
:103BD00065737320627574746F6E20746F00505239
:103BE000494E54205041555345440020204E6F7A91
:103BF0007A6C653A2000746F20636F6E74696E751D
:103C0000652E2E2E00616E642070726573732062C3
:103C10007574746F6E00496E736572742066696C9A
:103C2000616D656E74005052494E54205041555399
:103C300045440020204E6F7A7A6C653A20002000BF
:103C400066696C616D656E74206C6F6164005761AC
:103C5000697420666F72005052494E54205041558D
:103C60005345440020204E6F7A7A6C653A2000203C
:103C70000066696C616D656E742065787472756438
:103C800065005761697420666F72005052494E5446
:103C90002050415553454400746F20726573756D13
:103CA00065005761697420666F72207072696E7466
:103CB000005052494E5420504155534544004D6FD9
:103CC000766520617869730044697361626C652070
:103CD0007374657070657273004D383400426564AA
:103CE000204C6576656C696E6700473238205859FC
:103CF0000A4D31303920533137350A473238205A8E
:103D00000A4D31303920523134350A4731320A47B1
:103D100032390A4D313034205330004175746F20F0
:103D2000686F6D6500473238004D61696E004D3532
:103D300030320A4D353030004C6F61642073657449
:103D400074696E677300526573746F726520666183
:103D5000696C736166650053746F72652073657476
:103D600074696E677300416476616E6365642053A5
:103D7000657474696E6773004D61696E000A003B7B
:103D800020454550524F4D20496E6465783A2000D9
:103D90005570646174696E67207A6F6666736574C6
:103DA00020696E20454550524F4D3A2000060006CE
:103DB0000006000600060006000600060006003F9A
:103DC000C01F800F00060006000F001F803FC006C6
:103DD00000060006000600060006000600060006B3
:103DE0000007F8000C0C00100200200100600180A8
:103DF0004000804003E04001C0400080400000409F
:103E000000006000002000001000000C0C0007F80B
:103E10000001FE0003030004008008004018006059
:103E20001000207C0020380020100020000020001E
:103E3000002000006000004000008003030001FE3D
:103E400000FFFFFF7F80FFC0FFC0FFC07F807F803B
:103E5000FFC0FFC0FFC03F001E000C005A204F668D
:103E600066736574005A204F666673657400466C0D
:103E70006F7700466C6F770046616E2073706565E2
:103E80006420310046616E207370656564203100E6
:103E900042656400426564004E6F7A7A6C65004E3C
:103EA0006F7A7A6C65005370656564005370656560
:103EB00064004D61696E004D6F7665205800453194
:103EC0003A200045303A20005A3A2000593A200062
:103ED000583A20004D53312C4D53322050696E73A7
:103EE0000A006265640A002C2073797374656D2082
:103EF00073746F7070656421204865617465725FCA
:103F000049443A2000436172642072656D6F7665A2
:103F100064004361726420696E7365727465640045
:103F20005265776970696E670050726F62696E677B
:103F3000206661696C65640050726F62696E67200B
:103F40006661696C65640050524F424520464149A4
:103F50004C20434C45414E204E4F5A5A4C450A0086
:103F60005265776970696E670A0052657769706992
:103F70006E670050726F62696E67206661696C657A
:103F8000640050726F62696E67206661696C656477
:103F90000050524F4245204641494C20434C454138
:103FA0004E204E4F5A5A4C450A0052657769706947
:103FB0006E670A0050726F62696E67206661696C95
:103FC00065640A0050726F62696E67206661696C91
:103FD000656400205A3A200020593A200042656466
:103FE00020583A20000201050800FF060121023591
:103FF00020FFFF07FF06FF09005022165680808031
:10400000800080153353A0A0A00257575050F8509D
:10401000F850500257572070A07028702013355563
:1040200080A040A02002475740A0A040A0A050255B
:104030001353808080122656408080808040122654
:10404000568040404040800245559060F0609002AC
:1040500055552020F82020113353604080044151F1
:10406000F011335340E0400246561010204080804B
:1040700012365640A0A0A0A04012365640C0404084
:1040800040E00246566090106080F0024656F020F4
:10409000601090600246562060A0F0202002465634
:1040A000F080E01090600246566080E090906002E0
:1040B0004656F01020204040024656609060909096
:1040C00060024656609090701060122555C0C00086
:1040D000C0C01136566060006040801236562040E5
:1040E00080804020034353F000F012365680402079
:1040F00020408012365640A02040004001585830E1
:104100004898A8A8904030024656609090F0909051
:10411000024656E090E09090E00246566090808023
:104120009060024656E090909090E0024656F080F3
:10413000E08080F0024656F080E0808080024656A3
:10414000609080B090600246569090F090909012EF
:104150003656E040404040E002465670202020A005
:104160004002465690A0C0A0A09002465680808093
:104170008080F002465690F0F09090900246569063
:10418000D0F0B0B090024656609090909060024699
:1041900056E09090E08080014757609090D0B060EA
:1041A00010024656E09090E0909002465660904093
:1041B000209060123656E040404040400246569003
:1041C0009090909060024656909090906060024669
:1041D00056909090F0F090024656909060609090CB
:1041E000025656888850202020024656F010204063
:1041F00080F0123656E080808080E0024656808053
:1042000040201010123656E020202020E0163252B6
:1042100040A0014151F01622528040024454709057
:1042200090700246568080E09090E0123454608096
:10423000806002465610107090907002445460B036
:10424000C060024656205040E04040014555609015
:104250007010600246568080E09090901236564072
:1042600000C04040E01137572000202020A040022D
:104270004656808090E09090123656C040404040B4
:10428000E0025454D0A8A8A8024454E090909002B0
:10429000445460909060014555E090E08080014575
:1042A000557090701010024454A0D0808012345485
:1042B00060C020C00246564040E0405020024454B6
:1042C00090909070123454A0A0A04002545488A83A
:1042D000A8500244549060609001455590907090B1
:1042E00060024454F02040F0024757304020C02084
:1042F0004030221656808080808080024757C02040
:1043000040304020C006425250A0FFFFFFFFFFFF99
:10431000FFFFFFFFFFFFFFFFFFFFFFFFFFFFFFFFAD
:10432000FFFFFFFFFFFFFFFFFFFFFF090050221607
:10433000568000808080800146562070A0A07020AA
:104340000246562050E04050A002555588705070EB
:10435000880256568850F820F8202217578080800F
:10436000008080800247577080E0907010E0173125
:1043700051A002565670A8C8C8A87014355560A040
:104380006000E003435350A050123353E020201448
:104390003151E002565670E8D8E8D870173151E034
:1043A00015335340A04012355540E04000E014352D
:1043B0005540A02040E0143555C020C020C0162232
:1043C000524080014555909090E08002565678E822
:1043D000E868282824115180112252408014355554
:1043E00040C04040E014355540A04000E003435336
:1043F000A050A0024757808080A060F0200247575D
:104400008080A0D010207002475780408060A0F0CC
:104410002012365640004080A0400247574020609E
:1044200090F0909002475720406090F090900247A3
:104430005760906090F0909002475750A06090F0C5
:10444000909002475790006090F09090024757601C
:10445000906090F0909002465670A0A0F0A0B0013D
:104460004757609080809060400247574020F0801E
:10447000E080F00247572040F080E080F00247578C
:104480006090F080E080F00247579000F080E0807C
:10449000F01237578040E0404040E012375720404C
:1044A000E0404040E012375740A0E0404040E0127A
:1044B0003757A000E0404040E00256567048E848B8
:1044C000487002475750A090D0B090900247574094
:1044D00020609090906002475720406090909060DC
:1044E0000247576090609090906002475750A060DC
:1044F00090909060024757900060909090601233C7
:1045000053A040A002465670B0B0D0D0E00247574A
:10451000402090909090600247572040909090905B
:1045200060024757609090909090600247579000CB
:1045300090909090600257571020885020202002C1
:10454000465680E09090E0800246566090A0A09091
:10455000A0024757402000709090700247572040BB
:104560000070909070024757205000709090700239
:10457000475750A0007090907002465650007090BF
:10458000907002475760906070909070025454F0A1
:1045900068B07811355560808060400247574020F0
:1045A0000060B0C06002475720400060B0C06002A9
:1045B000475760900060B0C060024656500060B03F
:1045C000C060123757804000C04040E0123757208B
:1045D0004000C04040E012375740A000C04040E0DB
:1045E000123656A000C04040E0024757A040A0103D
:1045F00070906002475750A000E09090900247579B
:1046000040200060909060024757204000609090EA
:10461000600247576090006090906002475750A03A
:104620000060909060024656900060909060123555
:10463000554000E0004002445470B0D0E0024757BB
:10464000402000909090700247572040009090903A
:10465000700247576090009090907002465690000C
:1046600090909070014858204000909070906001A8
:1046700047578080E090E0808001475790009090FD
:1046800070906001050700FE0500FB01F220FFFEAF
:1046900005FE05FE02004002152580808000800591
:1046A0003242A0A002556550F850F85001465620FD
:1046B00070C030E0200255659010204048025565DA
:1046C00060806890680512228080022535408080D5
:1046D00080400225358040404080043343A040A004
:1046E00003334340E0400122324080043141E00284
:1046F00011218002556508102040800245556090C8
:10470000909060022535C040404040024555E01081
:104710006080F0024555E0106010E00245552060D1
:10472000A0F020024555F080E010E0024555608081
:10473000E09060024555F0102040400245556090E1
:1047400060906002455560907010600313238000F4
:104750008002142480008080023545204080402063
:10476000033343E000E002354580402040800245AD
:1047700055E0106000400255657088B8A870024589
:1047800055609090F090024555E090E090E0023541
:10479000456080808060024555E0909090E0023551
:1047A00045E080E080E0023545E080E08080024521
:1047B000557080B090700245559090F09090023501
:1047C00045E0404040E00245553010109060024501
:1047D0005590A0C0A09002354580808080E00255B1
:1047E0006588D8A8888802455590D0B09090024539
:1047F000556090909060024555E09090E0800146B1
:1048000056609090906010024555E09090E09002C4
:10481000455570806010E0023545E0404040400260
:10482000455590909090600245559090A0A0400210
:10483000556588A8A8A850024555909060909002B0
:1048400045559090701060023545E0204080E002B0
:104850002535C0808080C002556580402010080248
:104860002535C0404040C005324240A0024151F0D1
:104870000522328040024454709090700245558069
:10488000E09090E0023444608080600245551070F2
:1048900090907002445460B0C0600235452040E002
:1048A000404000465670909070106002455580E080
:1048B000909090021525800080808000273740006E
:1048C00040404040800245558090A0E09002152570
:1048D0008080808080025464F0A8A8A8024454E03C
:1048E00090909002445460909060004656E0909002
:1048F000E08080004656709090701010023444A002
:10490000C0808002445470C030E002354540E04031
:104910004020024454909090700244549090A040E3
:10492000025464A8A85050023444A04040A000465D
:1049300056909090701060024454F02040F0023580
:10494000456040804060021525808080808002356F
:1049500045C0402040C005425250A0FFFFFFFFFF6E
:10496000FFFFFFFFFFFFFFFFFFFFFFFFFFFFFFFF57
:10497000FFFFFFFFFFFFFFFFFFFFFFFF020040FF02
:10498000FFFFFFFFFFFFFFFFFFFFFFFFFFFFFFFF37
:10499000FFFFFFFFFFFFFFFFFFFFFFFFFFFFFFFF27
:1049A000FFFFFFFFFFFFFFFFFFFFFFFFFFFFFFFF17
:1049B000FFFFFFFFFFFFFFFFFFFFFFFFFFFFFFFF07
:1049C000FFFFFFFFFFFFFFFFFFFFFFFFFFFFFFFFF7
:1049D000FFFFFFFFFFFFFFFFFFFFFFFFFFFF0106DE
:1049E0000D00FE09016602D620FFFE0BFE0AFE0D39
:1049F0000060221969808080808080800080183368
:104A000063A0A0A00357675050F850F850500259C7
:104A1000692078A0A0702828F02002596948A85081
:104A200010204050A89002586840A0A040A0989044
:104A300068281363808080113B6B20404080808019
:104A40008080404020113B6B80404020202020206F
:104A500040408006556520A870A820045565202098
:104A6000F82020113363604080065161F8113363F0
:104A700040E0400259690808101020404080800240
:104A80005969205088888888885020025969206098
:104A9000A02020202020F802596970888808102062
:104AA0004080F8025969F8081020700808887002E0
:104AB0005969101030505090F81010025969F88060
:104AC00080B0C80808887002596970888080F088B2
:104AD000888870025969F808101020204040400270
:104AE00059697088888870888888700259697088C8
:104AF0008888780808887011386840E040000040D5
:104B0000E04011386840E040000060408002596990
:104B1000081020408040201008045464F80000F879
:104B200002596980402010081020408002596970A5
:104B3000888808102020002002596970888898A869
:104B4000A8B080780259692050888888F8888888B9
:104B5000025969F048484870484848F0025969705D
:104B60008880808080808870025969F04848484871
:104B7000484848F0025969F8808080F0808080F8C9
:104B8000025969F8808080F08080808002596970C5
:104B9000888080809888887002596988888888F819
:104BA00088888888123969E040404040404040E0B1
:104BB000025969381010101010109060025969885D
:104BC0008890A0C0A09088880259698080808080E9
:104BD000808080F80259698888D8A8A88888888841
:104BE00002596988C8C8A8A8989888880259697025
:104BF0008888888888888870025969F0888888F051
:104C000080808080015A6A70888888888888A87027
:104C100008025969F0888888F0A09088880259694C
:104C2000708880807008088870025969F8202020F8
:104C300020202020200259698888888888888888D0
:104C4000700259698888888850505020200259691C
:104C500088888888A8A8A8A85002596988885050D0
:104C60002050508888025969888850502020202080
:104C700020025969F808101020404080F8113B6B61
:104C8000E0808080808080808080E0025969808020
:104C900040402010100808113B6BE020202020200D
:104CA00020202020E0085363205088015161F82A19
:104CB00022628040025666700878889868025969B6
:104CC000808080F088888888F002566670888080AE
:104CD0008870025969080808788888888878025698
:104CE000667088F880887002596930484040F0400A
:104CF0004040400058687088888878088870025959
:104D000069808080B0C8888888881238684000C070
:104D100040404040E0004A6A1000301010101090EF
:104D2000906002596980808090A0C0A0908812395C
:104D300069C040404040404040E0025666D0A8A8CC
:104D4000A8A888025666B0C8888888880256667007
:104D50008888888870005868F0888888F08080800B
:104D60000058687888888878080808025666B0C8AD
:104D70008080808002566670886010887002586853
:104D80004040F04040404830025666888888889805
:104D9000680256668888885050200256668888A81F
:104DA000A8A850025666885020205088005868886D
:104DB00088889868088870025666F810204080F845
:104DC000015B6B1820202020C020202020182219F1
:104DD00069808080808080808080015B6BC0202023
:104DE00020201820202020C008536348A890FFFFEF
:104DF000FFFFFFFFFFFFFFFFFFFFFFFFFFFFFFFFC3
:104E0000FFFFFFFFFFFFFFFFFFFFFFFFFFFFFF0DA4
:104E10000060221969800080808080808080035833
:104E2000682070A8A0A0A8702002596930484040AE
:104E3000E0404048B0035666887050507088025970
:104E40006988885050F820F82020221969808080D5
:104E5000800080808080124A6A60908060909060BC
:104E60001090601A3262A0A00359697088A8D8C84F
:104E7000D8A88870045767700878887800F80356B7
:104E8000662850A0A05028045363F8080816316122
:104E9000E00359697088E8D8D8E8D888700A516169
:104EA000F8174464609090600357672020F8202032
:104EB00000F807356540A02040E007356540A04078
:104EC00020C02A226240800058688888888898E834
:104ED000808002596978E8E8E8E8682828282621CF
:104EE00061C0202262408007356540C04040E00438
:104EF0005767708888887000F8035666A050282885
:104F000050A0025A6A40C04040E008182838080201
:104F10005A6A40C04040E01028081038025A6A40DF
:104F2000A04020A0481828380802596920002020F5
:104F30004080888870025A6A40200020508888F893
:104F40008888025A6A10200020508888F8888802D1
:104F50005A6A30480020508888F88888025A6A289F
:104F6000500020508888F88888025A6A50500020E3
:104F7000508888F88888025A6A20502020508888F3
:104F8000F8888802596958A0A0A0B0E0A0A0B80095
:104F90005B6B7088808080808088702040025A6AB5
:104FA000402000F88080F08080F8025A6A102000CB
:104FB000F88080F08080F8025A6A304800F88080DB
:104FC000F08080F8025A6A505000F88080F08080AB
:104FD000F8123A6A804000E04040404040E0123A17
:104FE0006A204000E04040404040E0124A6A609041
:104FF00000E04040404040E0123A6AA0A000E0409B
:1050000040404040E0025969F0484848E848484874
:10501000F0025A6A2850008888C8A8988888025ADE
:105020006A40200070888888888870025A6A102038
:105030000070888888888870025A6A3048007088B2
:105040008888888870025A6A285000708888888802
:105050008870025A6A505000708888888888700367
:1050600055658850205088015B6B08709898A8A8F7
:10507000A8C8C87080025A6A40200088888888883A
:105080008870025A6A102000888888888888700290
:105090005A6A30480088888888888870025A6A501E
:1050A000500088888888888870025A6A1020008892
:1050B00088502020202002596980F0888888F0805C
:1050C0008080025969609090A0A0908888B00259B1
:1050D000694020007008788898680259691020009B
:1050E0007008788898680259693048007008788894
:1050F00098680259692850007008788898680259A1
:1051000069505000700878889868025A6A304830B0
:1051100000700878889868025666702870A0A850B9
:10512000005868708880808870204002596940204B
:10513000007088F88088700259691020007088F823
:105140008088700259693048007088F88088700241
:1051500059695050007088F8808870123969804011
:1051600000C040404040E0123969204000C040404B
:105170004040E0124969609000C040404040E01269
:105180003969A0A000C040404040E0025A6A502067
:105190006010708888888870025969285000B0C8EB
:1051A00088888888025969402000708888888870BB
:1051B0000259691020007088888888700259693007
:1051C0004800708888888870025969285000708863
:1051D0008888887002596950500070888888887063
:1051E000035767202000F8002020015868087098B5
:1051F000A8A8C870800259694020008888888898CB
:10520000680259691020008888888898680259695E
:10521000304800888888889868025969505000880A
:105220008888889868005B6B102000888888986858
:10523000088870005A6A8080B0C88888C8B08080AA
:10524000005B6B5050008888889868088870000060
:10525000000000000000000000000000000000004E
:10526000000000000000000000000000000000003E
:10527000000C000000000000000C00000000000016
:1052800000120000000000000023000000000000E9
:105290000021000000000000004C80000000000021
:1052A000005E80000000000000924000000000004E
:1052B00000A14000000000000121200000000000CB
:1052C000027F9000000000000200100000000000BB
:1052D00007FFF800000000000400080000000000C4
:1052E00008000400000000000800060000000000A4
:1052F0001000020000000000301E0100000000004D
:10530000207F81000000000041FFE08000000000DD
:1053100043FCF08000000000873B78400000000163
:105320008EDBFC60000000010FEBCC2000000002CF
:105330001FEDB610000000021FDEB61000000004D2
:1053400039CD7F080000000436E0FF0800000008A7
:105350007EC0BB84000000187F005D860000001046
:105360007FC0ED82000000203CC0730100000020DF
:105370003B337F01000000701BE77E03800000C804
:105380001DEEDE04C00000880FDEDC0440000124B6
:105390000FDF3C092000012607DBF819200002720C
:1053A00003E7F0139000025101FFE022900004890E
:1053B000007F802448000904801E004824000BFE62
:1053C000400000DFF40010004000008002001FFFDA
:1053D000FFFFFFFFFE0000000000000000000000D3
:1053E000000000000000000000000000000010228B
:1053F000103C3C0E1F001022100422110400102249
:10540000100822110400102210083C110400102280
:1054100010102211040010221020221104001E1C62
:105420001E3C3C0E040000000000000000000000D4
:10543000000000000000000000000000000000006C
:10544000000000000000000000000000000000005C
:10545000000000000000000000000000000000004C
:10546000000000000000000000000000000000003C
:10547000000000000000000000000000000000002C
:10548000000000000000000000000000526573658D
:105490006E643A20002042002050006F6B004B49A0
:1054A0004C4C45442E20004B494C4C206361757395
:1054B0006564206279204B494C4C20627574746F8E
:1054C0006E2F70696E0A004B494C4C45442E2000EB
:1054D0004B494C4C2063617573656420627920747C
:1054E0006F6F206D75636820696E6163746976659E
:1054F0002074696D65202D2063757272656E74204D
:10550000636F6D6D616E643A20004D36303020421D
:1055100030005072696E7420706175736564004D5F
:1055200031323500004D3234005072696E742061A2
:10553000626F72746564004E6F2053442063617221
:1055400064005072696E742066726F6D205344005F
:1055500053746F70207072696E7400526573756D4C
:1055600065207072696E7400506175736520707289
:10557000696E740041626F7574204669726D77615F
:105580007265004368616E67652066696C616D6570
:105590006E7400436F6E66696775726174696F6ED1
:1055A0000054656D7065726174757265004D6F763B
:1055B000656D656E740054756E6500496E666F208A
:1055C00073637265656E00202F002042403A002010
:1055D000403A004C756C7A426F742054415A203620
:1055E000204F66662E004B494C4C45442E2000004F
:1055F00013C27ACC11241FBECFEFD1E2DEBFCDBFE4
:1056000000E00CBF14E0A0E0B2E0ECE9F4E402E05A
:105610000BBF02C007900D92AE30B107D9F725E15C
:10562000AEE0B4E001C01D92AE32B207E1F71AE27B
:10563000C9EFDAE200E006C021970109802FFE01E0
:105640000F94CA21C83FD10780E00807A9F70E943C
:105650008D720D943D220C9400002F923F924F9238
:105660005F926F927F928F929F92AF92BF92CF92F2
:10567000DF92EF92FF920F931F93CF93DF93CDB7FB
:10568000DEB7C658D1090FB6F894DEBF0FBECDBF46
:1056900000917F0620E6029F8001112401501B4FDC
:1056A00080917B1480FF1AC0E7E4F6E284917F01C9
:1056B0003FEFE31AF30A811102C0780104C00F948E
:1056C0000214F701F3CFD7018D917D01882319F0E2
:1056D0000F940214F8CF8AE00F94021410922E0453
:1056E00010922D048FE38093420410924104109293
:1056F0004004109228041092290410922A04109257
:105700002B04F80180810F5F1F4F8032D1F38E345C
:10571000B1F4818190ED980F9A3020F08D3211F024
:105720008B3269F43296DF0131962C9120532A3066
:10573000D0F3CD01FC01019620812032D9F3F09302
:105740007214E09371147F01BFEFEB1AFB0A108112
:105750006AE270E0C7010F940E22009731F0FC015D
:10576000319780818032E1F311821D3429F01435A4
:1057700019F0173409F0CDC0F70180812FEFE21A3C
:10578000F20A8032C9F380538A3008F0C2C0109305
:10579000420420914004309141044AE03196429FF6
:1057A000C001439F900D1124DF0111972C9130E02F
:1057B00020533109280F391F808180538A3070F3BC
:1057C0003093410420934004DF0131968C91803264
:1057D000D9F31D3449F00091711440912D0450917A
:1057E0002E0461E070E058C02E31310591F03CF498
:1057F0002731310571F02C31310569F70AC02537A1
:1058000031054CF32737310524F0203A43E03407C3
:1058100011F7B0932E04A0932D047BC0813209F4BC
:1058200045C09FEBB92EB80E89E1A82EAB1408F441
:105830005EC0DF01FD01908111969032D9F3A0ED99
:10584000A90FAA3008F047C04F01EB2CF12C6701DB
:10585000A3E0D594C794AA95E1F7C601885D9B4F54
:105860006C018B2D8770DB0102C0AA0FBB1F8A95CC
:10587000E2F7CD01D6019C91892B8C938114910480
:10588000A1F1801AC701825F9B4FDC018C9280815D
:1058900081548A3188F5DF01FD0131968C918111A7
:1058A000BDCF50932E0440932D0433C01D3409F016
:1058B000B8CF2032310509F0B4CFF0932E04E09335
:1058C0002D0463E270E0CF010F940E22009709F1DE
:1058D000DC011C921EC0A3EDA90FA23008F4B4CFC6
:1058E0009B3211F00C94CE41AFCF812CCBCF411520
:1058F000510569F6AD01CBCFDF0131969C919053F4
:105900009A30D0F3CD01FC010196A081A032D9F3E9
:10591000C2CF809142048D3411F40C94C934843583
:1059200011F40C947041873411F00C94B1418091C2
:105930004004909141048A31910509F4F4C6BCF405
:105940008430910544F4823091050CF01FC197FF1B
:105950002BC00C94CB418430910509F4E0C60C9720
:1059600011F00C94CB410E943F5F0C94CB418E31DF
:10597000910509F47FC73CF48C31910509F464C7A3
:105980000CF4D8C666C78B35910509F4F9C78C3578
:10599000910509F4FAC78A35910511F00C94CB41B1
:1059A00010923F040C94CB4180917D02882311F426
:1059B0000C94CB410E94C6B984E39DE00F94AA0DDC
:1059C0000E9482BA80917B1483FD8FC0C090400DED
:1059D000D090410DE090420DF090430D20911707BB
:1059E000309118074091190750911A07C701B60165
:1059F0000F94A21A882309F478C08091B012811103
:105A000038C06091690270916A02072E000C880B01
:105A1000990B0F94A81A9B01AC016091AC12709184
:105A2000AD128091AE129091AF120F94A21A87FF1F
:105A300020C0C0921707D0921807E0921907F09281
:105A40001A07E7E4F6E284918F010F5F1F4F882366
:105A500021F00F940214F801F6CFECE5F2E0849106
:105A60008F010F5F1F4F882321F00F940214F8015C
:105A7000F6CFC090400DD090410DE090420DF090D7
:105A8000430D209117073091180740911907509145
:105A90001A07C701B6010F94DA1E20E030E048E48F
:105AA00053E40F940121181604F5C0921707D09201
:105AB0001807E0921907F0921A07E7E4F6E28491DA
:105AC0008F010F5F1F4F882321F00F940214F801FC
:105AD000F6CFEDE3F2E084918F010F5F1F4F882333
:105AE00021F00F940214F801F6CF2091340D30917B
:105AF000350D4091360D5091370D60910B07709127
:105B00000C0780910D0790910E070F94A21A811136
:105B10001DC02091380D3091390D40913A0D5091B2
:105B20003B0D60910F0770911007809111079091C4
:105B300012070F94A21A811109C060918702709117
:105B400088028091890290918A021AC060916F0246
:105B500070917002072E000C880B990B0F94A81AF5
:105B600020918702309188024091890250918A02E7
:105B70000F94071B2AE037ED43E25CE30F94071B09
:105B80000E9487B40E947DB40C94CB4120917D0289
:105B9000222311F40C94CB4111E0029709F010E09C
:105BA0000E94C6B982E50E94BAB9882309F45CC193
:105BB0000E9458B96B017C0140900B0750900C0774
:105BC00060900D0770900E0720910F07309110071D
:105BD000409111075091120763962CAF3DAF4EAF25
:105BE0005FAF63978091340D9091350DA091360D84
:105BF000B091370D67968CAF9DAFAEAFBFAF6797D3
:105C00002091380D3091390D40913A0D50913B0D56
:105C10006B962CAF3DAF4EAF5FAF6B9720E030E09F
:105C2000A901C701B6010F94A21A882309F45DC522
:105C3000A301920167966CAD7DAD8EAD9FAD679768
:105C40000F94A21A811111C063962CAD3DAD4EADDB
:105C50005FAD63976B966CAD7DAD8EAD9FAD6B9771
:105C60000F94A21A882309F440C520E030E0A9016E
:105C7000C701B6010F94A21A881F8827881F18131E
:105C80000BC080E090E0A0E8BFE3AB968CAF9DAF87
:105C9000AEAFBFAFAB970AC020E030E040E85FEBAB
:105CA000AB962CAF3DAF4EAF5FAFAB97A301920168
:105CB00067966CAD7DAD8EAD9FAD67970F94DA1E84
:105CC000A3966CAF7DAF8EAF9FAFA39763962CADBD
:105CD0003DAD4EAD5FAD63976B966CAD7DAD8EAD5A
:105CE0009FAD6B970F94DA1EA7966CAF7DAF8EAF0A
:105CF0009FAFA797A3962CAD3DAD4EAD5FADA397DB
:105D0000CA01B9010F94071B4B015C01A7962CAD8A
:105D10003DAD4EAD5FADA797CA01B9010F94071B0A
:105D20009B01AC01C501B4010F94DB1E0F94462109
:105D30006F966CAF7DAF8EAF9FAF6F9720E030E076
:105D400040E05FE30F94071B4B015C01A701960144
:105D5000C701B6010F94071B6B017C01A5019401DB
:105D6000C501B4010F94071B9B01AC01C701B6012B
:105D70000F94DA1E0F9446219B01AC01AB966CADDB
:105D80007DAD8EAD9FADAB970F94071B4B015C01B2
:105D900067962CAD3DAD4EAD5FAD6797C301B201C7
:105DA0000F94DB1E20E030E040E05FE30F94071B20
:105DB0006B017C01A7966CAD7DAD8EAD9FADA797B5
:105DC00090586F962CAD3DAD4EAD5FAD6F970F9473
:105DD000B71F9B01AC01C501B4010F94071B9B01C8
:105DE000AC01C701B6010F94DB1EA30192010F9411
:105DF000DA1E6B017C016B962CAD3DAD4EAD5FADF7
:105E00006B9763966CAD7DAD8EAD9FAD63970F9430
:105E1000DB1E20E030E040E05FE30F94071B2B0126
:105E20003C016F962CAD3DAD4EAD5FAD6F97A39627
:105E30006CAD7DAD8EAD9FADA3970F94B71F9B0149
:105E4000AC01C501B4010F94071B9B01AC01C30158
:105E5000B2010F94DB1E63962CAD3DAD4EAD5FAD30
:105E600063970F94DA1E14C089E40E94BAB988239C
:105E700029F00E9458B96B017C0103C0C12CD12CC0
:105E800076018AE40E94BAB98823F9F00E9458B9D1
:105E90006B966CAF7DAF8EAF9FAF6B9720E030E01D
:105EA000A901C701B6010F94A21A81111EC020E0FA
:105EB00030E0A9016B966CAD7DAD8EAD9FAD6B975B
:105EC0000F94A21A811111C010C420E030E0A90182
:105ED000C701B6010F94A21A882309F406C46B9671
:105EE0001CAE1DAE1EAE1FAE6B97D701C601B058DB
:105EF00063968CAF9DAFAEAFBFAF63976B962CAD83
:105F00003DAD4EAD5FAD6B97505867962CAF3DAF32
:105F10004EAF5FAF67979C01AD01BC01CD010F94FF
:105F2000071B4B015C0167962CAD3DAD4EAD5FADDF
:105F30006797CA01B9010F94071B9B01AC01C5010A
:105F4000B4010F94DB1E0F944621EB966CAF7DAF2E
:105F50008EAF9FAFEB9780910B0790910C07A091AC
:105F60000D07B0910E076F968CAF9DAFAEAFBFAF70
:105F70006F97A7019601BC01CD010F94DB1EAB9674
:105F80006CAF7DAF8EAF9FAFAB9720910F07309175
:105F900010074091110750911207A3962CAF3DAF07
:105FA0004EAF5FAFA3976B962CAD3DAD4EAD5FADE1
:105FB0006B97A3966CAD7DAD8EAD9FADA3970F94FF
:105FC000DB1EAF966CAF7DAF8EAF9FAFAF9780916A
:105FD000340D9091350DA091360DB091370DE396AB
:105FE0008CAF9DAFAEAFBFAFE397AB962CAD3DADE1
:105FF0004EAD5FADAB97BC01CD010F94DA1E6B01C6
:106000007C012091380D3091390D40913A0D50911D
:106010003B0DE7962CAF3DAF4EAF5FAFE797AF9626
:106020002CAD3DAD4EAD5FADAF97E7966CAD7DADA0
:106030008EAD9FADE7970F94DA1E4B015C01809106
:10604000130790911407A0911507B0911607C15836
:10605000DF4F88839983AA83BB83CF57D0409C01AD
:10606000AD0160913C0D70913D0D80913E0D909180
:106070003F0D0F94DA1EA7966CAF7DAF8EAF9FAF2A
:10608000A797209117073091180740911907509151
:106090001A07CD57DF4F288339834A835B83C35860
:1060A000D0406091400D7091410D8091420D9091D2
:1060B000430D0F94DA1EEF966CAF7DAF8EAF9FAF9E
:1060C000EF97A701960163966CAD7DAD8EAD9FAD48
:1060D00063970F94071B2B013C01A5019401679660
:1060E0006CAD7DAD8EAD9FAD67970F94071B9B0187
:1060F000AC01C301B2010F94DB1E2B013C01A501D1
:10610000940163966CAD7DAD8EAD9FAD63970F949A
:10611000071B4B015C01A701960167966CAD7DAD35
:106120008EAD9FAD67970F94071B9B01AC01C50116
:10613000B4010F94DA1EA30192010F944E1F6B015C
:106140007C0120E030E0A9010F94A21A87FF0AC069
:106150002BED3FE049EC50E4C701B6010F94DB1E84
:106160006B017C01112351F02BED3FE049EC50E431
:10617000C701B6010F94DA1E6B017C0120E030E00C
:10618000A901C701B6010F94A21A811128C0E39694
:106190002CAD3DAD4EAD5FADE3976F966CAD7DAD73
:1061A0008EAD9FAD6F970F94A21A811118C0E7961C
:1061B0002CAD3DAD4EAD5FADE797A3966CAD7DAD1B
:1061C0008EAD9FADA3970F94A21A811108C0EBED7D
:1061D000CE2EEFE0DE2EE9ECEE2EE0E4FE2EEB9686
:1061E0002CAD3DAD4EAD5FADEB97C701B6010F9441
:1061F000071B9B01AC010F94071B4B015C01A79689
:106200002CAD3DAD4EAD5FADA797CA01B9010F945E
:10621000071B9B01AC01C501B4010F94DB1E0F9459
:1062200046214B015C012FE632E143E85AE30F942B
:10623000A21A87FD56C2C501B4010F9450200F94D5
:106240002420A1967FAF6EAFA197672B31F421E098
:1062500030E0A1963FAF2EAFA197A196AEACBFACF8
:10626000A197B50180E090E00F94A61A4B015C0164
:106270009B01AC01C701B6010F94B71F6F966CAFBD
:106280007DAF8EAF9FAF6F97A5019401A7966CADC0
:106290007DAD8EAD9FADA7970F94B71FEB966CAFFA
:1062A0007DAF8EAF9FAFEB97A5019401EF966CADDC
:1062B0007DAD8EAD9FADEF970F94B71FEF966CAF8E
:1062C0007DAF8EAF9FAFEF976F962CAD3DAD4EADCE
:1062D0005FAD6F97CA01B9010F94071B20E030E052
:1062E00040E05FE30F94071B9B01AC0160E070E0AE
:1062F00080E89FE30F94DA1EA7966CAF7DAF8EAF58
:106300009FAFA797C158DF4F288139814A815B81B0
:10631000CF57D04029873A874B875C87CD57DF4FCF
:1063200088819981AA81BB81C358D0408D879E877F
:10633000AF87B88B60916F0270917002072E000CCE
:10634000880B990B0F94A81A20918702309188022C
:106350004091890250918A020F94071B2AE037ED81
:1063600043E25CE30F94071BE3966CAF7DAF8EAF07
:106370009FAFE3970E94ACC19B01AC0128533F4FF4
:106380004F4F5F4FE7962CAF3DAF4EAF5FAFE797F4
:1063900060964FAC609761965FAC619762966FAC08
:1063A000629763967FAC639722242394312C79E122
:1063B000D72EA196AEACBFACA1972A143B0409F42A
:1063C0004CC10E94289D0E94ACC1DC01CB01E79624
:1063D0002CAD3DAD4EAD5FADE797821B930BA40B8B
:1063E000B50BB7FD11C00E94ACC19B01AC01285395
:1063F0003F4F4F4F5F4FE7962CAF3DAF4EAF5FAF74
:10640000E79780E00F94360BDA94DD2009F44BC057
:10641000A7962CAD3DAD4EAD5FADA79767966CAD21
:106420007DAD8EAD9FAD67970F94071B4B015C014F
:106430006F962CAD3DAD4EAD5FAD6F97B201C30110
:106440000F94071BA50194010F94DB1E7B018C01A7
:10645000A7962CAD3DAD4EAD5FADA797B201C30180
:106460000F94071B4B015C016F962CAD3DAD4EADFB
:106470005FAD6F9767966CAD7DAD8EAD9FAD679745
:106480000F94071B9B01AC01C501B4010F94DA1EE8
:106490002B013C01C701D80167968CAF9DAFAEAF11
:1064A000BFAF67975BC0B10180E090E00F94A61A80
:1064B0006F962CAD3DAD4EAD5FAD6F970F94071B42
:1064C0004B015C010F94B41F6B017C01C501B40149
:1064D0000F943C214B015C01A701960163966CADC2
:1064E0007DAD8EAD9FAD63970F94071B2B013C01D3
:1064F000A50194016B966CAD7DAD8EAD9FAD6B9794
:106500000F94071B9B01AC01C301B2010F94DB1E6A
:106510002B013C01A501940163966CAD7DAD8EAD60
:106520009FAD63970F94071B4B015C01A701960178
:106530006B966CAD7DAD8EAD9FAD6B970F94071BC9
:106540009B01AC01C501B4010F94DA1E67966CAFD4
:106550007DAF8EAF9FAF679759E1D52E9201A30112
:10656000AB966CAD7DAD8EAD9FADAB970F94DB1E42
:1065700069837A838B839C8367962CAD3DAD4EAD4A
:106580005FAD6797AF966CAD7DAD8EAD9FADAF97AC
:106590000F94DB1E6D837E838F839887EB962CADE3
:1065A0003DAD4EAD5FADEB9769857A858B859C855A
:1065B0000F94DB1E69877A878B879C87EF962CADBB
:1065C0003DAD4EAD5FADEF976D857E858F8598892A
:1065D0000F94DB1E6D877E878F87988BCE01019687
:1065E0000F94AA0DC090391389819A81AB81BC8127
:1065F00088A399A3AAA3BBA38D819E81AF81B885EF
:106600008CA39DA3AEA3BFA389859A85AB85BC85CA
:1066100088A799A7AAA7BBA7AE01485D5F4FBE0197
:106620006C5D7F4FCE0180960E947C88E396ECAC37
:10663000FDAC0EAD1FADE3979E01235F3F4FAE0152
:10664000485D5F4FBE016C5D7F4FCE0180960E941A
:106650005D7A3FEF231A330AACCEC0903913809194
:10666000340D9091350DA091360DB091370D88A362
:1066700099A3AAA3BBA38091380D9091390DA09145
:106680003A0DB0913B0D8CA39DA3AEA3BFA3809107
:106690003C0D90913D0DA0913E0DB0913F0D88A70E
:1066A00099A7AAA7BBA7AE01485D5F4FBE016C5D6D
:1066B0007F4FCE0180960E947C88E396ECACFDACC7
:1066C0000EAD1FADE39720E43DE0AE01485D5F4FA6
:1066D000BE016C5D7F4FCE0180960E945D7A0E9464
:1066E0007DB40E9482BA0C94CB41E8E8F4E2849134
:1066F0008F010F5F1F4F882321F00F940214F801C0
:10670000F6CFE7E7F2E084918F010F5F1F4F8823F8
:1067100011F40C94CB410F940214F801F4CF0E94B1
:10672000915F0C94CB4181E080937D021092BF0970
:106730000C94CB410E94B8AF81110C94CB4180E501
:106740000E94BAB9882321F00E9428B9262F01C0DF
:1067500020E06091130770911407809115079091C4
:106760001607C12CD12C18E8E12E11ECF12EC982AC
:10677000DA82EB82FC82C12CD12C02E9E02E03E408
:10678000F02ECD82DE82EF82F886C12CD12C30EA49
:10679000E32E31E4F32EC986DA86EB86FC86C12C23
:1067A000D12C40ECE42E4FE7F42ECD86DE86EF862A
:1067B000F88A213071F1223021F518A219A21AA20B
:1067C0001BA220E030E040EA51E40F94DB1E6B0195
:1067D0007C0120E030E047E853E40F9401211816D3
:1067E00034F4C12CD12CB7E8EB2EB3E4FB2ECBAEA6
:1067F000DCAEEDAEFEAEBE01605E7F4FCE01CB964D
:1068000011C020E030E040EA51E40F94A21A87FF63
:106810000BC018A219A21AA21BA2BE01605E7F4F74
:10682000CE0109960E946CB418A219A21AA21BA24A
:10683000AE01405E5F4FBE016B5F7F4FCE010196A0
:106840000E9468B40C94CB4180E00E94975C0C9449
:10685000CB4181E08093D10424982C9A0898109A17
:106860000E946E4E1092D104249A2C98089A109887
:106870000C94CB4120E030E0A90160910B077091AE
:106880000C0780910D0790910E070F94DB1E6B0192
:106890007C0188E50E94BAB9882321F00E9458B98A
:1068A0006B017C01C8A2D9A2EAA2FBA220E030E0E1
:1068B000A90160910F0770911007809111079091C5
:1068C00012070F94DB1E6B017C0189E50E94BAB9A7
:1068D000882321F00E9458B96B017C01C982DA82B9
:1068E000EB82FC824090471350904813609049130C
:1068F00070904A13209143133091441340914513F3
:106900005091461368A179A18AA19BA10F94DA1E28
:106910004B015C012CE032E048ED51EC0F94012179
:1069200087FF02C00C94CB4121E230E040E953E400
:10693000C501B4010F94A21A181614F40C94CB419B
:10694000A3019201C701B6010F94DA1E6B017C010D
:106950002CE032E040EA51EC0F94012187FF02C0A5
:106960000C94CB4121E230E047E953E4C701B60182
:106970000F94A21A181614F40C94CB410C94D8411D
:1069800081E080933F040C94CB410F9447130C9407
:10699000CB4180914004909141048937910511F4D5
:1069A0000C94023D0CF0D8C08D34910509F4A9C5B2
:1069B0000CF053C08931910509F4EDC21CF5843106
:1069C000910509F469C27CF48131910509F459C239
:1069D0002CF4029708F4D1C10C94CB41429709F4EE
:1069E00033C70C94CB418631910509F49CC20CF459
:1069F00096C28731910509F49CC2489709F4ACC24C
:106A00000C94CB418F31910509F481C47CF48B3116
:106A1000910509F4DCC20CF4CCC28C31910509F467
:106A200012C34E9709F419C30C94CB418A329105D5
:106A300009F412C52CF4809709F41FC40C94CB41BF
:106A40008B34910509F45AC58C34910511F00C94DE
:106A5000CB410E94EEB00C94CB418B36910509F4EA
:106A6000D6C6C4F58535910509F4F1C6C4F482355E
:106A7000910509F4E2C64CF48135910511F00C94AE
:106A8000CB410F94B9110C94CB418335910509F496
:106A9000D7C68435910509F4D7C60C94CB41883606
:106AA000910509F431C54CF48C35910511F00C9425
:106AB000CB410E9467710C94CB418936910509F452
:106AC00038C68A36910511F00C94CB410F94CF1142
:106AD0000C94CB418337910509F4BCC6D4F48E36AF
:106AE000910509F45DC534F48D36910509F464C649
:106AF0000C94CB418F36910509F463C5823791051B
:106B000011F00C94CB410E94BEF80E94A8700C9426
:106B1000CB418637910509F42EC774F4853791056A
:106B200011F00C94CB4160E080912D0490912E04E3
:106B30000E9452D60C94CB418737910509F452C775
:106B40008837910511F00C94CB4181E08093D004FB
:106B50008093CF040C94CB41803321E0920711F451
:106B60000C94D43D0CF084C08D3C910509F4CCC745
:106B7000C4F58E3B910509F437C6C4F48C389105F1
:106B800009F4BDC54CF48D37910511F00C94CB413F
:106B90000E941E700C94CB418139910509F437C7CE
:106BA0008B39910509F4DFC50C94CB41893C9105E3
:106BB00009F4A4C74CF4883C910511F00C94CB4126
:106BC0000E94D16F0C94CB418B3C910509F499C77D
:106BD0008C3C910511F00C94CB410E94256F0C94D4
:106BE000CB41823E910509F4D9C72CF5833D91052F
:106BF00009F4C4C79CF48E3C910511F00C94CB4170
:106C0000E3E0AE2EE3E0BE2EFBE0CF2EF7E0DF2E7A
:106C1000A2EDEA2EA4E0FA2E10E079C78C3D910592
:106C200009F4AFC78D3D910511F00C94CB410E9442
:106C3000106E0C94CB418D3241E0940709F4B1C73A
:106C40004CF48C32914011F00C94CB410E94906D29
:106C50000C94CB418E32B1E09B0709F4A8C78F3268
:106C6000914011F00C94CB410E946C670C94CB4185
:106C7000853FF1E09F0711F40C94203F0CF041C0D8
:106C8000813931E0930709F495C7ECF48F3551E071
:106C9000950711F40C94F1403CF48E35914011F4B9
:106CA0000C94BC400C94CB418336E1E09E0711F478
:106CB0000C9445418039914011F00C94CB410E94D5
:106CC000BEF80C94CB41843A21E0920709F476C7D0
:106CD00054F48239914011F00C94CB4180E00E9431
:106CE00023B40C94CB418C3A51E0950709F4BAC710
:106CF000843F914011F00C94CB410E941E950C945E
:106D0000CB418335B3E09B0711F40C943F3FB4F4BF
:106D1000873FF1E09F0711F40C94263F14F40C9484
:106D2000233F8C3132E0930711F40C94343F8835C3
:106D3000924011F40C94723F0C94CB418C3853E088
:106D4000950711F40C94A24064F48B38934011F031
:106D50000C94CB4133E0E32E33E0F32E10E00C949F
:106D60007B40803AE3E09E0709F4C4C2873E93402B
:106D700011F40C945E410C94CB41A0902D04B09082
:106D80002E0480E50E94BAB9882359F00E9418B9F0
:106D90006B017C0111E0672B682B692B31F410E04B
:106DA00004C010E0C12CD12C760183E50E94BAB951
:106DB0008823F1F00E9458B920E030E04AE754E41B
:106DC0000F94071B0F9424206B017C01111112C03A
:106DD000672B682B692B71F4A114B10459F0D5010C
:106DE0008C91882339F061E0C5010E9452D607C01A
:106DF000112391F360E083EC92E00E9433D681E0AE
:106E0000809317130E94BEF80E9482BAC114D10465
:106E1000E104F104F1F08091731490917414A09145
:106E20007514B0917614C80ED91EEA1EFB1E0E947E
:106E3000ACC1DC01CB018C199D09AE09BF09B7FFBC
:106E40001CC0809117138823C1F080E00F94360B8B
:106E5000EECF80911713882321F080E00F94360B3A
:106E6000F8CF8091770A60E0882319F084EB92E0F4
:106E700002C08FE992E00E9433D6109217130C944F
:106E8000CB4160E086ED92E00E9433D617981698C9
:106E9000159814980C94CB41EEEEF2E084918F019A
:106EA0000F5F1F4F882321F00F940214F801F6CFD3
:106EB0001092230D40E050E0BA018FEC9AE00E945E
:106EC0003F8C8BE1EFECFAE0DE01159601900D921C
:106ED0008A95E1F78091CD0A9091CE0A9C838B83AD
:106EE00081E993E09A83898340E050E0BE016F5FBF
:106EF0007F4F8BEB93E00E94EEC6CE0101960E947D
:106F000097CCEFEDF2E084918F010F5F1F4F882344
:106F100011F40C94CB410F940214F801F4CF0E94A9
:106F200004AE0C94CB411092770A1092780A0C941C
:106F3000CB4180912D0490912E04FC0120812223CD
:106F400029F0203209F410823196F8CF40E061E058
:106F50000E94D5AA0C94CB4119821A821B821C82F2
:106F600018A219A21AA21BA28091550D882341F0E4
:106F700040E0BE016F5F7F4FCE0180960E9439CA0C
:106F80008091780A882319F081E08093770A0E9423
:106F90007EAF0C94CB411092770A0E94EEB08FEF37
:106FA00092E090933A09809339090E9455B50C9468
:106FB000CB418091780A882311F40C94CB4183E56E
:106FC0000E94BAB981110C942E420C94CB4180914D
:106FD000780A882351F1E4E0F3E084918F010F5F98
:106FE0001F4F882321F00F940214F801F6CF60910F
:106FF0001A0D70911B0D80911C0D90911D0D4AE092
:107000000F945B148FE20F9402146091160D70912F
:10701000170D8091180D9091190D4AE00F945B1493
:107020008AE00F9402140C94CB41E6E1F3E08491E2
:107030008F010F5F1F4F882311F40C94CB410F94E5
:107040000214F801F4CF40E060E080912D049091AB
:107050002E040E94D5AA0C94CB418091780A8823F3
:1070600011F40C94CB4189E69CE00E94418D89E6A5
:107070009CE00E94728D1092760A1092750AE09040
:107080002D04F0902E048091780A882311F40C943A
:10709000CB410E942CC51D8218861C821B8281E96F
:1070A00093E09A8389838BEC9AE09093EB0A809328
:1070B000EA0AF70180818F3209F068C06FE270E060
:1070C000C7010F940E228C010F5F1F4F9E012F5F8F
:1070D0003F4F49010115110509F45EC06FE270E0F0
:1070E000C8010F940E226C01009709F456C00817CE
:1070F000190708F052C05C01A01AB10AA501B80135
:10710000CE0180960F942E22E0E2F0E0EC0FFD1FFE
:10711000EA0DFB1D10828E01005E1F4FD8018D917C
:107120008D01882319F00F940214F8CF8AE00F9490
:1071300002146091EA0A7091EB0A6115710511F071
:107140006C5F7F4F21E0AE01405E5F4FCE01059640
:107150000E947D93811112C0BE01605E7F4F8DE45D
:1071600093E00E94D9778EE20F9402148AE00F9484
:107170000214C4010E9497CC0C94CB419092EB0A6C
:107180008092EA0A86010F5F1F4FA4CF8CEE9AE02F
:107190009093EB0A8093EA0A87016091EA0A709162
:1071A000EB0A6115710511F06C5F7F4F18A21BA2ED
:1071B00022E0A801CE0180960E947D93811102C039
:1071C000F12C14C0CE0180960E949AC48823C1F38A
:1071D00061E0CE0180960E94268D009789F325EE0E
:1071E000FC0120831BA20E945089F82ECE018096BC
:1071F0000E9475BAFF2011F1A7E2EA2EA3E0FA2E51
:10720000F7018491882331F0FFEFEF1AFF0A0F9402
:107210000214F6CFD8018D918D01882319F00F94B7
:107220000214F8CF8AE00F94021410921A0D1092F3
:107230001B0D10921C0D10921D0D19C0F5E3EF2EC1
:10724000F3E0FF2EF7018491882331F0FFEFEF1A6E
:10725000FF0A0F940214F6CFD8018D918D01882377
:1072600019F00F940214F8CF8EE20F940214CE019D
:1072700001960E9497CC0C94CB418091770A8111A2
:107280000E94BEF8E0902D04F0902E0480E50E944C
:107290008BB9182F882319F00E9449B9182F8091B3
:1072A000780A882311F40C94CB41412F61E0C70187
:1072B0000E94D5AA83E50E94BAB9882381F00E9472
:1072C00028B9AB01BC0140931A0D50931B0D60937C
:1072D0001C0D70931D0D89E69CE00E943F8C8091EF
:1072E000780A882319F081E08093770A11110C94B1
:1072F000CB414DCE80912D0490912E0421E020931E
:10730000760A40E060E00E94D5AA0C94CB410E942E
:10731000BBC6ECE3CE2ED12CE12CF12CA7019601BB
:107320000F947D1E762E672ECA01B901A701960122
:107330000F947D1E6B017C01CA01B90128E130E088
:1073400040E050E00F947D1E4B015C01C9016DE6E9
:1073500071E00F94A3218E010F5F1F4F611571051E
:1073600099F06F927F92DF92CF929F928F929F932C
:107370008F937F936F9389E893E09F938F931F93ED
:107380000F930F943B1A12C00097B1F06F927F9247
:10739000DF92CF929F928F929F938F9389E793E092
:1073A0009F938F931F930F930F943B1A0FB6F894EC
:1073B000DEBF0FBECDBF36C081149104A104B1045D
:1073C00079F06F927F92DF92CF929F928F928DE6AB
:1073D00093E09F938F931F930F930F943B1AE6CFE5
:1073E000C114D104E104F10469F06F927F92DF923D
:1073F000CF9285E693E09F938F931F930F930F9403
:107400003B1AD4CF6F927F9281E693E09F938F9344
:107410001F930F930F943B1A0F900F900F900F90A4
:107420000F900F9060E0C8010E9452D6E7E4F6E2A8
:1074300084917F019FEFE91AF90A882321F00F94C4
:107440000214F701F5CFB8018DE993E00E94D977D6
:107450008AE00F9402149FC783E50E94BAB988237B
:1074600009F499C70E9438B9E82E80E50E94BAB99C
:10747000811112C081E0E11001C080E08093D1044D
:10748000882329F024982C9A0898109A84C7249A63
:107490002C98089A10987FC780E50E94BAB9882373
:1074A00031F00E9428B98B0177FF03C074C70DE04B
:1074B00010E0902FEAEAF3E088E28E0F2491921711
:1074C00021F031968E13FACFDAC7E8E8F4E284911E
:1074D0008F010F5F1F4F882321F00F940214F801D2
:1074E000F6CFE2EDF3E084918F010F5F1F4F882309
:1074F00009F451C70F940214F801F5CF0E947EAF32
:107500004AC70E9452C547C788E690E00E9435BA34
:10751000811141C780917B1483FD3DC783E50E94A3
:10752000BAB9882309F437C70E9458B90F941F20AD
:10753000709352046093510480E00E94F79B0E9474
:1075400058B920E030E040E752E40F94A21A181630
:107550003CF00E9452C560E08DEE93E00E9433D66D
:107560000E9458B92091AC123091AD124091AE12E8
:107570005091AF120F94012118160CF00CC784ED36
:1075800092E09F938F9381EE93E09F938F931F924E
:107590000E9437C50F900F900F900F900F90FBC671
:1075A0008EE40E94BAB9882309F4F5C60E9428B96E
:1075B00060935614709357148093581490935914F1
:1075C000EAC683E50E94BAB9882319F00E9438B947
:1075D00001C080E080937B14E7E4F6E284918F01A0
:1075E0000F5F1F4F882321F00F940214F801F6CF8C
:1075F000E0E1F4E084918F010F5F1F4F882321F0B9
:107600000F940214F801F6CF80917B148823A1F126
:1076100072E0C72E74E0D72EE12CF12C20E080918F
:107620007B1490E00E2C02C0959587950A94E2F7A2
:1076300080FF17C0BB24B394B20E222319F08CE252
:107640000F940214F60125913491F9018491890176
:107650000F5F1F4F882321F00F9402149801F5CF7C
:107660002B2DFFEFEF1AFF0A32E0C30ED11C45E0CD
:10767000E416F104A1F63FC0ECE0F4E084918F0140
:107680000F5F1F4F8823B9F10F940214F801F6CF52
:107690008AE50E948BB9882309F417C40E9458B95F
:1076A0006B017C0120E030E040E050EC0F940121C0
:1076B00087FDFEC320E030E040EA50E4C701B60198
:1076C0000F94A21A18160CF4F3C3C092F706D092C6
:1076D000F806E092F906F092FA0680E00E94DA6677
:1076E0006091F7067091F8068091F9069091FA067C
:1076F00042E00F94DB148AE00F9402144CC6809190
:107700007B1483FD48C683E50E94BAB9882309F437
:1077100042C60E9458B90F941F206739710514F0B2
:1077200066E970E07093500460934F040E94AC9B34
:1077300032C689E690E00E9435BA81110C948745E3
:10774000E7E1F4E084918F010F5F1F4F882321F060
:107750000F940214F801F6CF0F94F5118AE00F94FC
:1077600002140C94874583E50E94BAB9882309F472
:1077700012C60E9438B980935E148D3318F08CE3E2
:1077800080935E140E94ACC16B017C0120915E1459
:1077900030E0A8EEB3E00F94CB1EDC01CB018C0DE2
:1077A0009D1DAE1DBF1D80935A1490935B14A09332
:1077B0005C14B0935D14EFC58DE690E00E9435BA7D
:1077C0008111E9C580917B1483FDE5C583E50E94A5
:1077D000BAB960968FAF609781116EC682E50E943C
:1077E000BAB9811169C6D7C580917B1483FDD3C511
:1077F00083E50E94BAB968968FAF689781110C949F
:10780000004482E50E94BAB98111FAC7C4C580E577
:107810000E94BAB9882339F00E9428B962307105F4
:1078200008F0B9C502C060E070E0660F771FFB0189
:10783000E55BFB4F11821082AEC510923E04ABC5D2
:1078400081E080933E04A7C50F946A11A4C50E94ED
:107850000572A1C5EEE5F5E084918F010F5F1F4F22
:10786000882321F00F940214F801F6CFE0E5F5E04B
:1078700084918F010F5F1F4F882321F00F94021412
:10788000F801F6CFE9E3F5E084918F010F5F1F4F18
:10789000882321F00F940214F801F6CFE9E2F5E015
:1078A00084918F010F5F1F4F882321F00F940214E2
:1078B000F801F6CFE8E1F5E084918F010F5F1F4FEB
:1078C000882321F00F940214F801F6CFE7E0F5E0E9
:1078D00084918F010F5F1F4F882321F00F940214B2
:1078E000F801F6CFE8EFF4E084918F010F5F1F4FAE
:1078F000882321F00F940214F801F6CFE3EEF4E0B0
:1079000084918F010F5F1F4F882321F00F94021481
:10791000F801F6CFEDECF4E084918F010F5F1F4F7B
:10792000882321F00F940214F801F6CFE8EBF4E07D
:1079300084918F010F5F1F4F882321F00F94021451
:10794000F801F6CFEBE9F4E084918F010F5F1F4F50
:10795000882321F00F940214F801F6CFE3E8F4E055
:1079600084918F010F5F1F4F882309F414C50F9472
:107970000214F801F5CF85E40E948BB9882381F0C9
:107980000E9449B9882361F0E7E4F6E284918F010F
:107990000F5F1F4F882321F00F940214F801F6CFD8
:1079A00081E40E948BB9882381F00E9449B9882321
:1079B00061F0E4E5F6E084918F010F5F1F4F8823AB
:1079C00021F00F940214F801F6CF00912D041091CC
:1079D0002E04D8018D918D01882309F48CCE0F944B
:1079E0000214F7CF81E08093D10424982C9A089850
:1079F000109A0E943FD31092D104249A2C98089A8E
:107A00001098C9C41092D0041092CF04C4C483E566
:107A10000E94BAB9882319F00E9428B902C060E018
:107A200070E08B01112702301105CCF0E8E8F4E298
:107A300084918F010F5F1F4F882321F00F94021450
:107A4000F801F6CFE8E5F6E084918F010F5F1F4F54
:107A5000882309F4A0C40F940214F801F5CF88E438
:107A60000E94BAB98823A9F00E9428B96837710525
:107A70003CF06332B1E07B072CF062E271E002C0BF
:107A800068E770E0F801EE0FFF1FE352F94F7183D2
:107A9000608386E40E94BAB98823A9F00E9428B9BD
:107AA000F801EE0FFF1FEB52F94F718360836F3FB8
:107AB000710519F014F06FEF70E077FF02C060E01D
:107AC00070E07183608382E40E94BAB9882309F46C
:107AD00062C40E9428B96530710534F068387105B8
:107AE0002CF067E870E002C065E070E0000F111F45
:107AF000F801E752F94F718360834DC40E94AC6F67
:107B00004AC40E948A6F47C40E94BB6E44C4F501F8
:107B100081915F010E948BB9882311F10E9458B9AD
:107B20002B013C01D7012D913D914D915C910F941A
:107B3000DA1E9B01AC01F601608171818281938123
:107B40000F94DB1ED6016D937D938D939C931397B9
:107B5000F7014082518262827382812F0E94E2B4D7
:107B60001F5FF4E0CF0ED11C24E0E20EF11C1330B5
:107B700071F60E9438B80E94A8700DC40E942B6E46
:107B80000AC483E50E94BAB9882309F404C40E9498
:107B900028B97093700260936F02FDC30E94C56D97
:107BA000FAC30E94F66CF7C30E947A6CF4C30E9479
:107BB000256CF1C381E00E9423B4EDC386E50E94E9
:107BC0008BB9882321F087EA96E00E944CB183E5C7
:107BD0000E948BB9182F882319F00E9449B9182FD9
:107BE00083E50E948BB9882319F0812F0E94FFB290
:107BF000F090BF12111103C0E7E4F6E21AC0F110D1
:107C0000FBCFE8E8F4E284918F010F5F1F4F8823D8
:107C100021F00F940214F801F6CFE8E8F6E0849121
:107C20008F010F5F1F4F882339F30F940214F8015F
:107C3000F6CF84918F010F5F1F4F882321F00F949F
:107C40000214F801F6CFF11003C06EEE72E002C02C
:107C50006AEE72E08AE796E00E94D9778AE00F9494
:107C6000021499C352EDC52E54E0D52E6BE0E62EDA
:107C700067E0F62E7BE2272E77E0372E00E010E05B
:107C8000A22CA0946096AFAE6097D1018D911D019A
:107C9000882309F4A3C0F70140805180628073807B
:107CA000F801EF58FD4F2081318142815381F80165
:107CB000E15DFB4F60817181828193810F94DB1EB6
:107CC00020E030E040E05FE30F94071B9B01AC0134
:107CD000C301B2010F940121181644F4F801E056D3
:107CE000F84D85909590A590B49003C0812C912C6F
:107CF0005401F801ED5BFC4E2081318142815381BA
:107D0000C301B2010F94DA1E9B01AC01C501B4019D
:107D10000F94DA1E4B015C0120E030E040EA51ECA8
:107D20000F94012187FD2BC020E030E040EA51E4B0
:107D3000C501B4010F94A21A18160CF1D6012D91A9
:107D40003D914D915C91C501B4010F94DA1E9B01E8
:107D5000AC01C301B2010F94DB1EF7016083718394
:107D600082839383D6018D929D92AD92BC9213979C
:107D700060968FAD6097820D0E94E2B42FC0E8E854
:107D8000F4E284918F010F5F1F4F882321F00F943D
:107D90000214F801F6CFE2EEF6E084918F010F5F56
:107DA0001F4F882321F00F940214F801F6CF61E0F1
:107DB00084ED96E00E9433D60E94226588E290E02E
:107DC0009A83898388EC90E099A388A3BE016F5FB2
:107DD0007F4FCE0180960E944BAFDDC2B4E0CB0E48
:107DE000D11C0C5F1F4FE4E0EE0EF11C0C301105AE
:107DF00009F04BCF0E9438B80E94A87060E084EC74
:107E000096E00E9433D683E992E099A388A304E622
:107E100010E01A830983BE01605E7F4FCE01019698
:107E20000E944BAF8AEB92E099A388A31A8309833F
:107E3000BE01605E7F4FCE0101960E944BAFABC288
:107E40000E9439A4A8C20E94F5A2A5C283E50E949F
:107E50008BB9882319F00E9449B901C081E091E0F3
:107E600089270E94BD9E97C283E50E948BB9882313
:107E700009F491C20E9449B98093E2048CC2E7E4FC
:107E8000F6E284918F010F5F1F4F882321F00F943A
:107E90000214F801F6CFE8E1F7E084918F010F5F5B
:107EA0001F4F882309F4F4CB0F940214F801F5CF87
:107EB000E3E0F7E084918F010F5F1F4F882309F4FF
:107EC0001ACC0F940214F801F5CF4091F7065091A7
:107ED000F8066091F9067091FA0680E097E00E943A
:107EE000577209CC0E94B8AF882319F081E00E9434
:107EF000975C85E40E948BB9882319F00E9458B9D9
:107F000004C060E070E080E090EC2F966CAF7DAF35
:107F10008EAF9FAF2F978AE50E94BAB9882319F0D8
:107F20000E9458B904C060E070E080E291E42B96B2
:107F30006CAF7DAF8EAF9FAF2B9788E50E94BAB92B
:107F4000882319F00E9458B904C060E070E080E214
:107F500091E427966CAF7DAF8EAF9FAF279789E5F1
:107F60000E94BAB9882319F00E9458B904C060E091
:107F700070E082E993E423966CAF7DAF8EAF9FAF44
:107F8000239785E50E948BB9882319F00E9458B980
:107F900004C060E070E088EC92EC6BAF7CAF8DAF1A
:107FA0009EAF8CE40E948BB9882319F00E9458B9C7
:107FB00003C060E070E0CB0168A379A38AA39BA310
:107FC00082E40E94BAB9882321F00E9428B9F62ED3
:107FD00002C045E0F42ED090680A8091550D8111C1
:107FE00081C0CC24C394EF2C8E01055C1F4F9E01F1
:107FF000215C3F4FAE014D5B5F4FBE01695B7F4F20
:10800000CE01855B9F4F0E94CAC8882309F46AC0CD
:1080100081E08093171311E080911713882309F4EE
:108020004DC060E08F2D0F94D1128091BE0988233E
:1080300009F440C01093041340E050E0BA0184E416
:1080400098EE0E94FF5F80911713882321F081E052
:108050000F94360BF8CF109294061092950610925A
:108060009606109297061092BE090E94F79B0F94F5
:1080700074121093041340E050E0BA0183EB97EEC2
:108080000E94FF5F0E94ACC1DC01CB018853904588
:10809000AF4FBF4F8093940690939506A09396069A
:1080A000B09397061092BE091093171361E08F2DBD
:1080B0000F94D11281E00F94360BAECF80E090E0A8
:1080C000A8E4B2E489839A83AB83BC838091550D85
:1080D000882341F04F2DBE016F5F7F4FCE01809608
:1080E0000E9439CAF1E0DF1256C10E947EAF53C12F
:1080F0001F5F143069F0D7018D917D010E948BB90B
:108100008823B1F30E9428B9812F0E9431F8F0CF63
:1081100082E40E948BB9882329F00E9428B984E068
:108120000E9431F883E50E948BB9882309F433C19A
:1081300010E00E9428B9812F0E9431F81F5F15308E
:10814000C1F729C183E50E94BAB9882321F00E94B2
:1081500028B98B0102C000E010E080E50E94BAB9A6
:10816000882321F00E9428B9CB0102C080E090E072
:10817000B8010E9422F80FC183E50E948BB98111DA
:1081800006C023E0E22E23E0F22E10E00EC010E045
:108190000E9438B9682F812F0E940BF81F5F15309D
:1081A000B9F7EFCF1F5F143071F0F70181917F01B4
:1081B0000E948BB98823B1F30E9438B9682F812FB0
:1081C0000E940BF8EFCF82E40E948BB9882331F034
:1081D0000E9438B9682F84E00E940BF80E94A9F62B
:1081E000DAC083E50E94BAB9882309F44BC00E9423
:1081F00038B9813049F0823009F044C083E0E82E7C
:1082000083E0F82E10E023C093E0E92E93E0F92EEE
:1082100010E0D7018D917D010E94BAB9882339F011
:108220000E9438B94FEF682F812F0E9461F71F5FBE
:10823000143079F782E40E94BAB9882319F10E94B8
:1082400038B94FEF682F1BC01F5F143079F0F7016A
:1082500081917F010E94BAB98823B1F30E9438B995
:10826000482F6FEF812F0E9461F7EECF82E40E94CA
:10827000BAB9882339F00E9438B9482F6FEF84E0EB
:108280000E9461F70E94A9F686C0E8E8F4E28491B2
:108290008F010F5F1F4F882321F00F940214F80104
:1082A000F6CFE2E2F7E084918F010F5F1F4F882342
:1082B00009F471C00F940214F801F5CF81E08093A6
:1082C0007D021092BF0983E50E948BB9811103C022
:1082D0000F94610E60C00E9449B981115CC0F8CF53
:1082E000F0904004FF2021F1E7E4F6E284918F0151
:1082F0000F5F1F4F882321F00F940214F801F6CF6F
:1083000084E50F9402146F2D70E080E090E04AE065
:108310000F945B1480E20F94021402EF12E0D80174
:108320008D918D01882309F4E6C90F940214F7CFCB
:1083300010923913E7E4F6E284918F010F5F1F4F2B
:10834000882321F00F940214F801F6CF60913913BD
:1083500070E081E397E00E9474728AE00F94021447
:108360001AC0E7E4F6E284918F010F5F1F4F882364
:1083700021F00F940214F801F6CF609171147091FE
:10838000721483E497E00E94D97782E20F9402147A
:108390008AE00F9402140F94FF0DB9C341155105E3
:1083A00019F4AF0141505109812C912C0C94252CCA
:1083B00080E00E94FFB20E94A5BA83E50E948BB9BB
:1083C000882309F449C00E9449B921E0482FBE0121
:1083D0006F5F7F4FCE0180960F9400016B017C018F
:1083E0009B01AC010F948721811131C02CEA35EC3F
:1083F00047E257E368A179A18AA19BA10F94DB1EF4
:10840000AB01BC0187E992E00E943A722CEA35EC9C
:1084100047E257E369817A818B819C810F94DB1E4F
:10842000AB01BC0182E992E00E943A722CEA35EC81
:1084300047E257E3C701B6010F94DB1EAB01BC0155
:108440008DE892E00E943A728AE00F9402140E9432
:108450008CBA0E94A8709FCF81E0B7CF0E9428B944
:10846000AB01BC0140931A0D50931B0D60931C0D82
:1084700070931D0D89E69CE00E943F8C8CCF802F6D
:108480000E943CC36E2D802F0E947FC0F12CB7014B
:10849000802F0E94AEC00630110529F4F0924E04E0
:1084A000E0924D0478CF0830110509F074CFF092B6
:1084B0004C04E0924B046FCF0E9458B90F941F20D8
:1084C000709352046093510480E00E94F79B0E94D5
:1084D00058B920E030E040E752E40F94A21A181691
:1084E00044F00E9452C560E086E494E00E9433D6D6
:1084F00002C00E947EAF6091510470915204072E19
:10850000000C880B990B0F94A81A2091AC12309193
:10851000AD124091AE125091AF120F940121181676
:108520000CF066C184ED92E09F938F938AE394E010
:108530009F938F931F920E9437C50F900F900F90BB
:108540000F900F9081E080939E0267961CAE1DAE47
:108550001EAE1FAE67976F961CAE1DAE1EAE1FAE51
:108560006F9710E0A0961FAEA0975CE3A4965FAF54
:10857000A4978CE1A8968FAFA89796E4AC969FAF8E
:10858000AC97C12CD12C50E8E52E6FEBF62E812C48
:10859000912C54016091510470915204072E000CEB
:1085A000880B990B0F94A81A062F772E682E592E38
:1085B000262F372F482F592FB601C7010F94A21A23
:1085C0008823D9F02091AC123091AD124091AE12B7
:1085D0005091AF12602F772D862D952D0F94A21AF2
:1085E000182F111F1127111F6096AFAD6097AA2396
:1085F00041F0112331F011E0E9C00C2D7D2C6E2CDF
:108600005F2C0E94ACC16B017C01DC01CB016F9639
:108610002CAD3DAD4EAD5FAD6F97821B930BA40BA0
:10862000B50BB7FD3DC0D701C60188519C4FAF4F78
:10863000BF4F6F968CAF9DAFAEAFBFAF6F970F942C
:10864000F511E6E3F4E084911F019FEF291A390A3E
:10865000882321F00F940214F101F5CF81149104C5
:10866000A104B104B9F0D501C40188519C4FAF4FAA
:10867000BF4FBC01CD016C197D098E099F0928EE01
:1086800033E040E050E00F947D1ECA01B9010F9421
:10869000C11403C08FE30F9402148AE00F940214F4
:1086A00080E00F94360B0E9482BAA091AC126896BB
:1086B000AFAF68972090AD123090AE124090AF12DD
:1086C0002A2F322D432D542D602F772D862D952D59
:1086D0000F94DA1E9F7720E030E040E251E48114ED
:1086E0009104A104B10429F40F94A21A87FF07C0D2
:1086F00004C00F940121181614F4460157011123E8
:1087000009F44AC067962CAD3DAD4EAD5FAD67979D
:10871000211531054105510541F0D701C601821BE4
:10872000930BA40BB50BB7FD37C068962FAD6897B8
:10873000322D432D542DA0966FADA097A4967FADFA
:10874000A497A8968FADA897AC969FADAC970F94C1
:10875000DA1E20E030E040EC5FE30F94A21A87FDC0
:108760004ACFD701C601805A9541AF4FBF4F679698
:108770008CAF9DAFAEAFBFAF679768969FAD689760
:10878000A0969FAFA097A4962FAEA497A8963FAEB1
:10879000A897AC964FAEAC9780919E028823B1F01B
:1087A00081149104A104B10429F4C02ED72CE62C25
:1087B000F52CF0CEA8EECA1AA3E0DA0AE108F10817
:1087C000C818D908EA08FB08F7FCEFCF80919E0291
:1087D000882309F4E0CD60E0112329F08AE194E0D8
:1087E0000E9433D6D8CD88E294E00E9433D6D3CD10
:1087F0006096AFAC6097A110A5CE8FED92E094CEBD
:108800000E9458B90F941F206739710514F066E96A
:1088100070E07093500460934F040E94AC9B0E94E0
:1088200058B920E030E040EA50E40F9401211816D6
:1088300014F40E947EAF60914F0470915004072E93
:10884000000C880B990B0F94A81A2091AF0430915B
:10885000B0044091B1045091B2040F94A21A60E0A8
:1088600087FF03C086E794E002C089E694E00E9497
:1088700033D681E080939E028091391380932C043B
:1088800067961CAE1DAE1EAE1FAE67976F961CAEF0
:108890001DAE1EAE1FAE6F9760961FAE6097A0967E
:1088A0001FAEA097BCE3A496BFAFA497ECE1A89637
:1088B000EFAFA897F6E4AC96FFAFAC97C12CD12CE4
:1088C00030E8E32E4FEBF42E812C912C5401609173
:1088D0004F0470915004072E000C880B990B0F94D5
:1088E000A81A162F072F782E692E262F372F482FDC
:1088F000592FB601C7010F94A21A882331F1209194
:10890000AF043091B0044091B1045091B204612F92
:10891000702F872D962D0F94A21A881F8827881FE5
:1089200060968FAF609768962FAD6897222389F085
:10893000882379F080919E02882309F42CCD60E091
:108940008BE594E00E9433D626CD1C2D0D2D7E2C78
:108950006F2C0E94ACC16B017C01DC01CB016F96D6
:108960002CAD3DAD4EAD5FAD6F97821B930BA40B4D
:10897000B50BB7FD3DC0D701C60188519C4FAF4F25
:10898000BF4F6F968CAF9DAFAEAFBFAF6F970F94D9
:10899000F511E5E6F4E084912F019FEF491A590A99
:1089A000882321F00F940214F201F5CF8114910471
:1089B000A104B104B9F0D501C40188519C4FAF4F57
:1089C000BF4FBC01CD016C197D098E099F0928EEAE
:1089D00033E040E050E00F947D1ECA01B9010F94CE
:1089E000C11403C08FE30F9402148AE00F940214A1
:1089F00080E00F94360B0E9482BA2090AF04309032
:108A0000B0044090B1045090B2049101A201612FD2
:108A1000702F872D962D0F94DA1E9F7720E030E07F
:108A200040EA50E481149104A104B10429F40F94A4
:108A3000A21A87FF07C004C00F940121181614F46E
:108A4000460157016096AFAD6097AA2309F443C071
:108A500067962CAD3DAD4EAD5FAD679721153105E5
:108A60004105510541F0D701C601821B930BA40BB0
:108A7000B50BB7FD30C09101A201A0966FADA097D4
:108A8000A4967FADA497A8968FADA897AC969FADFE
:108A9000AC970F94DA1E20E030E040EC5FE30F94D7
:108AA000A21A87FD47CFD701C601805A9541AF4F23
:108AB000BF4F67968CAF9DAFAEAFBFAF6797A09625
:108AC0002FAEA097A4963FAEA497A8964FAEA897B6
:108AD000AC965FAEAC9780919E02882309F42ACFB2
:108AE00081149104A104B10429F4C12ED02EE72CE5
:108AF000F62CEDCE98EEC91A93E0D90AE108F108F8
:108B0000C818D908EA08FB08F7FE14CFEECFCA57F9
:108B1000DF4F0FB6F894DEBF0FBECDBFDF91CF9110
:108B20001F910F91FF90EF90DF90CF90BF90AF908B
:108B30009F908F907F906F905F904F903F902F907D
:108B400008950C9483E4EF92FF920F931F93CF93B9
:108B5000DF9300D01F92CDB7DEB710920F13809134
:108B6000241390912513A0912613B09127138130DF
:108B70009048A105B10540F01092241310922513DE
:108B800010922613109227131091241380918904B8
:108B90001816DCF4282F082E000C330B2150310955
:108BA000412F012E000C550B4217530774F01FEF95
:108BB000180F812F90E0A0E0B0E0809324139093F1
:108BC0002513A0932613B09327131092A11280911E
:108BD000AA12181714F41093AA128091AA12082E40
:108BE000000C990B0496212F012E000C330B8217D9
:108BF000930724F48CEF810F8093AA12E090AA12BD
:108C0000F12CE1101DC080911613811106C08091D6
:108C10002002882309F47AC109C01111F8CF0E94FB
:108C200028658091A112882391F378C181E0111108
:108C300080E024E048E059E06F2D0E9495D566C1A0
:108C400081E0E81228C080911613811106C080913E
:108C50002002882309F45AC111C01130C1F720E065
:108C600030E040E251E465E874E082E099E00F947E
:108C700092058091A112882351F350C185E894E0B8
:108C80000E945CD09C0181E0113009F080E000E09E
:108C90004CEF58E038C122E0E21228C08091161350
:108CA000811106C080912002882309F42FC111C0D0
:108CB0001230C1F720E030E048EC52E461E874E0A3
:108CC00082EF98E00F9492058091A112882351F3CE
:108CD00025C181E894E00E945CD09C0181E01230C3
:108CE00009F080E000E048EE58E00DC183E0E812B2
:108CF00028C080911613811106C08091200288231C
:108D000009F404C111C01330C1F720E030E048EC91
:108D100052E46DE774E08FED98E00F949205809136
:108D2000A112882351F3FAC08DE794E00E945CD031
:108D30009C0181E0133009F080E000E046ED58E04E
:108D4000E2C024E0E21236C080911613811106C001
:108D500080912002882309F4D9C011C01430C1F7D2
:108D600024E630E040E050E06DE674E08FEC98E0FF
:108D70000F9461068091A112882351F3CFC06091B6
:108D80006D0470916E0480916F04909170040F9443
:108D9000A61A69837A838B839C83CE0101960E94F5
:108DA0005CD09C0181E0143009F080E000E048ECE8
:108DB00058E0A9C085E0E81236C0809116138111F1
:108DC00006C080912002882309F4A0C011C015308C
:108DD000C1F724E630E040E050E061E774E081EC68
:108DE00098E00F9461068091A112882351F396C0F8
:108DF0006091710470917204809173049091740475
:108E00000F94A61A69837A838B839C83CE01019683
:108E10000E945CD09C0181E0153009F080E000E008
:108E20004AEB58E070C026E0E21236C0809116137B
:108E3000811106C080912002882309F467C011C007
:108E40001630C1F72AE030E040E050E065E774E01A
:108E500083EB98E00F9461068091A112882351F36F
:108E60005DC0609175047091760480917704909153
:108E700078040F94A61A69837A838B839C83CE012E
:108E800001960E945CD09C0181E0163009F080E0E0
:108E900000E04CEA58E037C087E0E81237C0809124
:108EA0001613811105C080912002882379F111C029
:108EB0001730C9F724E630E040E050E069E774E09D
:108EC00085EA98E00F9461068091A112882359F3F6
:108ED00025C06091790470917A0480917B0490910F
:108EE0007C040F94A61A69837A838B839C83CE01BA
:108EF00001960E945CD09C0181E0173009F080E06F
:108F000000E04EE958E06F2D0E940166F394E3946F
:108F100025E0F21276CE88E0809389040F900F90BE
:108F20000F900F90DF91CF911F910F91FF90EF90D5
:108F300008952F924F926F927F928F929F92AF924D
:108F4000BF92CF92DF92EF92FF920F931F93CF9336
:108F5000DF9310920F138091241390912513A09109
:108F60002613B091271381309048A105B10540F038
:108F70001092241310922513109226131092271387
:108F8000D091241380916C041816DCF4282F082E3D
:108F9000000C330B215031094D2F0D2E000C550BB9
:108FA0004217530774F0DFEFD80F8D2F90E0A0E049
:108FB000B0E08093241390932513A0932613B093CD
:108FC00027131092A1128091AA12D81714F4D093EB
:108FD000AA128091AA12082E000C990B04962D2F2C
:108FE0000D2E000C330B8217930724F48CEF8D0F9A
:108FF0008093AA12C091AA12412C63E0262E7FE52D
:10900000672E78E0772EE4E7CE2EE8E0DE2EF2E859
:10901000AF2EF8E0BF2EA9E88A2EA8E09A2EC11143
:109020001DC080911613811106C0809120028823F3
:1090300009F4AAC109C0D111F8CF0E942865809116
:10904000A112882391F3A8C181E0D11180E024E02E
:1090500047E958E0642D0E9495D596C1C13009F0CA
:109060003FC080911613811106C080912002882391
:1090700009F48AC116C0D130C1F7E12C10ECF12EF1
:1090800009E714E420E030E040E85FE36CE574E0D9
:1090900080E998E00F9433008091A112882329F38E
:1090A0007BC12F9287EE8F931F9281E08F938CE587
:1090B00094E09F938F93BF92AF929F928F924F9223
:1090C00081E0D13009F080E08F930E9470668DB707
:1090D0009EB70C960FB6F8949EBF0FBE8DBF54C1BD
:1090E000C23009F041C080911613811106C08091F1
:1090F0002002882309F448C116C0D230C1F7E12C00
:1091000010ECF12E09E714E420E030E040E85FE3E2
:1091100060E674E08BE798E00F9433008091A11231
:10912000882329F339C12F9287EE8F931F9281E014
:109130008F9380E694E09F938F93ADE6B8E0BF9362
:10914000AF93DF92CF924F9281E0D23009F080E06E
:109150008F930E9470668DB79EB70C960FB6F894E9
:109160009EBF0FBE8DBF10C1C33009F041C08091BA
:109170001613811106C080912002882309F404C1CE
:1091800016C0D330C1F7E12C10ECF12E09E714E43E
:1091900020E030E040E85FE364E674E086E698E0D3
:1091A0000F9433008091A112882329F3F5C02F92E8
:1091B00087EE8F931F9281E08F9384E694E09F93D4
:1091C0008F93A8E5B8E0BF93AF937F926F924F92D1
:1091D00081E0D33009F080E08F930E9470668DB7F4
:1091E0009EB70C960FB6F8949EBF0FBE8DBFCCC035
:1091F000C43009F043C080911613811106C08091DC
:109200002002882309F4C0C016C0D430C1F7E12C75
:1092100010ECF12E09E714E420E030E040E85FE3D1
:1092200068E674E081E598E00F9433008091A11224
:10923000882329F3B1C02F9287EE8F931F9281E08C
:109240008F9388E694E09F938F93A3E4B8E0BF9355
:10925000AF93AAE4B8E0BF93AF934F9281E0D430CC
:1092600009F080E08F930E9470668DB79EB70C96D0
:109270000FB6F8949EBF0FBE8DBF86C0C53009F0F3
:1092800041C080911613811106C08091200288236D
:1092900009F47AC015C0D530C1F7E12C10ECF12EDD
:1092A00009E714E420E030E0A90168E574E08EE30A
:1092B00098E00F9433008091A112882331F36CC0A1
:1092C0002F9287EE8F931F921F9288E594E09F93D1
:1092D0008F93A4E3B8E0BF93AF93A9E3B8E0BF9343
:1092E000AF934F9281E0D53009F080E08F930E94D8
:1092F00070668DB79EB70C960FB6F8949EBF0FBEE2
:109300008DBF42C0C63009F03FC080911613811155
:1093100005C0809120028823B9F115C0D630C9F765
:10932000E12C10ECF12E09E714E420E030E0A90173
:1093300064E574E08AE298E00F9433008091A11212
:10934000882339F329C02F9287EE8F931F921F92A3
:1093500084E594E09F938F93A6E1B8E0BF93AF9329
:10936000A0E2B8E0BF93AF934F9281E0D63009F00E
:1093700080E08F930E9470668DB79EB70C960FB6F3
:10938000F8949EBF0FBE8DBF4394CF5F95E0491206
:1093900046CE87E080936C04DF91CF911F910F91AF
:1093A000FF90EF90DF90CF90BF90AF909F908F9005
:1093B0007F906F904F902F9008950C94B0E5FF929E
:1093C0000F931F93CF93DF9310920F138091241369
:1093D00090912513A0912613B091271381309048C6
:1093E000A105B10540F0109224131092251310929C
:1093F000261310922713C09124138091530418163A
:10940000DCF4282F082E000C330B215031094C2F8F
:109410000C2E000C550B4217530774F0CFEFC80FFA
:109420008C2F90E0A0E0B0E080932413909325135C
:10943000A0932613B09327131092A1128091AA1221
:10944000C81714F4C093AA128091AA12082E000C17
:10945000990B04962C2F0C2E000C330B82179307BC
:1094600024F48CEF8C0F8093AA121091AA12D0E0F2
:10947000FF24F39411111AC080911613811106C0B4
:1094800080912002882309F4DEC009C0C111F8CF01
:109490000E9428658091A112882391F3DBC081E0AE
:1094A000C11180E024E041E158E0CAC01130A1F5CB
:1094B00080911613811106C080912002882309F43F
:1094C000C2C01BC0C130C1F7C0930F1310920B1361
:1094D00010920C1310920D1310920E1326EB3CEE0B
:1094E00042E251E061E574E08AE098E00F944105C2
:1094F0008091A112882301F3ADC080915104909115
:1095000052040E94ADD19C0181E0C13009F080E09D
:1095100000E043E058E06BC01230A1F580911613D3
:10952000811106C080912002882309F48CC01BC0E1
:10953000C230C1F7F0920F1310920B1310920C135C
:1095400010920D1310920E1329EB3CEE47E850E0F9
:109550006FE474E08FEF97E00F9441058091A112C2
:10956000882301F377C080914F04909150040E94AA
:10957000ADD19C0181E0C23009F080E000E04BEF0A
:1095800057E035C01330B9F580911613811106C02C
:1095900080912002882309F456C01BC0C330C1F754
:1095A000F0920F1310920B1310920C1310920D13D4
:1095B00010920E132FEF30E040E050E06BE474E0C7
:1095C0008FEE97E00F94AA008091A112882301F3F7
:1095D00041C080914B0490914C040E94ADD19C01FC
:1095E00081E0C33009F080E000E043EE57E06D2FEA
:1095F0000E94016628C0143031F580911613811144
:1096000005C0809120028823F1F013C0C430C9F74F
:1096100010924C0410924B0410924E0410924D0480
:109620000E94429C0E9422658091A112882349F3E6
:1096300011C081E0C43009F080E020E24AED57E03B
:109640006D2F0E9495D5DF5F1F5FD53009F012CFD7
:10965000D0935304DF91CF911F910F91FF90089504
:109660001F93CF93DF9310920F1380912413909147
:109670002513A0912613B091271381309048A1059E
:10968000B10540F010922413109225131092261366
:1096900010922713C091241380914A041816DCF409
:1096A000282F082E000C330B215031094C2F0C2E83
:1096B000000C550B4217530774F0CFEFC80F8C2FD7
:1096C00090E0A0E0B0E08093241390932513A09342
:1096D0002613B09327131092A1128091AA12C817D3
:1096E00014F4C093AA128091AA12082E000C990BB0
:1096F00004962C2F0C2E000C330B8217930724F4A6
:109700008CEF8C0F8093AA121091AA12D0E0111145
:109710001AC080911613811106C0809120028823FF
:1097200009F48DC009C0C111F8CF0E94286580914D
:10973000A112882391F38AC081E0C11180E024E066
:1097400041ED57E079C01130E9F480911613811191
:1097500006C080912002882309F471C00BC0C1307B
:10976000C1F784EB9DE40F941E008091A112882321
:1097700081F36CC081E0C13009F080E023E04AEC65
:1097800057E05AC01230E9F480911613811106C0D7
:1097900080912002882309F452C00BC0C230C1F767
:1097A00088EB9DE40F941E008091A112882381F321
:1097B0004DC081E0C23009F080E023E043EC57E087
:1097C0003BC01330E1F480911613811105C08091E4
:1097D00020028823A1F10BC0C330C9F78CEB9DE4B4
:1097E0000F941E008091A112882389F32FC081E07D
:1097F000C33009F080E023E04CEB57E01DC014308B
:10980000F1F480911613811105C080912002882304
:10981000B1F00BC0C430C9F780EC9DE40F941E007A
:109820008091A112882389F311C081E0C43009F02E
:1098300080E023E043EB57E06D2F0E9495D5DF5F7A
:109840001F5FD53009F063CFD0934A04DF91CF91E9
:109850001F91089562E08DE597E00C9448F261E075
:1098600086E597E00C9448F20F931F93CF93DF9314
:10987000082F709349046093480410920F1380914D
:10988000241390912513A0912613B09127138130B2
:109890009048A105B10540F01092241310922513B1
:1098A0001092261310922713C0912413809147041D
:1098B0001816DCF4282F082E000C330B2150310928
:1098C0004C2F0C2E000C550B4217530774F0CFEFA2
:1098D000C80F8C2F90E0A0E0B0E080932413909309
:1098E0002513A0932613B09327131092A1128091F1
:1098F000AA12C81714F4C093AA122091AA12022E19
:10990000000C330B2C5F3F4F8C2F0C2E000C990B4F
:109910002817390724F48CEF8C0F8093AA1210912A
:10992000AA12D0E091E0013049F1023009F44AC0B6
:1099300001116CC0111191C09923B1F01C16A4F053
:109940008091241390912513A0912613B091271391
:109950000196A11DB11D8093241390932513A0930C
:109960002613B0932713CF5F80912002882309F438
:10997000EEC021E041E06CEA77E06BC011116DC0F0
:109980009923B1F01C16A4F0809124139091251313
:10999000A0912613B09127130196A11DB11D8093AC
:1099A000241390932513A0932613B0932713CF5F0E
:1099B00080912002882309F4CAC021E041E065EAD1
:1099C00077E047C0111149C09923B1F01C16A4F0EB
:1099D0008091241390912513A0912613B091271301
:1099E0000196A11DB11D8093241390932513A0937C
:1099F0002613B0932713CF5F80912002882309F4A8
:109A0000A6C021E041E06EE977E023C0111125C036
:109A10009923B1F01C16A4F0809124139091251382
:109A2000A0912613B09127130196A11DB11D80931B
:109A3000241390932513A0932613B0932713CF5F7D
:109A400080912002882309F482C021E041E065E989
:109A500077E08D2F0F94E5047AC01130D9F480910E
:109A60001613811106C080912002882309F46FC06B
:109A700009C0C130C1F70E9428658091A1128823D6
:109A800091F36DC081E0C13009F080E024E04BE843
:109A900057E05AC01230E9F480911613811106C0C4
:109AA00080912002882309F452C00BC0C230C1F754
:109AB00088ED9DE40F941E008091A112882381F30C
:109AC0004EC081E0C23009F080E023E041E857E079
:109AD0003BC01330E1F480911613811105C08091D1
:109AE00020028823A1F10BC0C330C9F78DED9DE49E
:109AF0000F941E008091A112882389F330C081E069
:109B0000C33009F080E023E048E757E01DC014307F
:109B1000F1F480911613811105C0809120028823F1
:109B2000B1F00BC0C430C9F782EE9DE40F941E0063
:109B30008091A112882389F312C081E0C43009F01A
:109B400080E023E04DE657E06D2F0E9495D5DF5F62
:109B50001F5F90E0D53009F0E6CED0934704DF9147
:109B6000CF911F910F91089568E773EF80E07CCE4D
:109B70006FE27CE481E078CE6AE27CE482E074CE3D
:109B800067EE7DE483E070CE21E0209304136093C0
:109B9000430470934404809345049093460440E04A
:109BA00050E0BA0180914804909149040C94FF5F01
:109BB00060E070E080E291E4E7CF60E070E080E890
:109BC0009FE3E2CF6DEC7CEC8CEC9DE3DDCF8091EC
:109BD000161381110C94286560912413709125133C
:109BE00080912613909127136115710581059105C8
:109BF00071F10F94A81A20914304309144044091CC
:109C00004504509146040F94071B9B01AC016091E1
:109C10001707709118078091190790911A070F94F0
:109C2000DB1E6093170770931807809319079093B2
:109C30001A071092241310922513109226131092D3
:109C4000271383E00E9412F281E08093200280912A
:109C50002002882349F087E197E00E94FED0BC01F2
:109C600084E697E00C943D650895EF92FF921F9370
:109C7000CF93DF931F92CDB7DEB7182FE1E7F9E05E
:109C800084917F012FEFE21AF20A882331F0998341
:109C90000F940214F7019981F3CFE12FF92F8491EA
:109CA0007F019FEFE91AF90A882321F00F9402142B
:109CB000F701F5CFE8E5F9E084917F012FEFE21A93
:109CC000F20A882321F00F940214F701F5CF0F90C8
:109CD000DF91CF911F91FF90EF9008952F923F92C7
:109CE0004F925F926F927F928F929F92AF92BF92AC
:109CF000CF92DF92EF92FF920F931F93CF93DF9358
:109D0000CDB7DEB7CE5FD1090FB6F894DEBF0FBE78
:109D1000CDBF0E94B8AF81110C947D5CFE013196DD
:109D20008CE3DF011D928A95E9F70091BF12C352BF
:109D3000DF4F0883CD5DD0408AE40E948BB9882331
:109D400021F00E9414B30C947D5C86E50E94BAB9A0
:109D5000882349F00E9428B9C153DF4F7983688373
:109D6000CF5CD04006C0C153DF4F19821882CF5C50
:109D7000D040C153DF4F08811981CF5CD0400530FE
:109D8000110570F0E6E4FBE084918F010F5F1F4F37
:109D9000882311F40C947D5C0F940214F801F4CF25
:109DA00084E40E948BB9C152DF4F8883CF5DD040DD
:109DB000882339F00E9449B9C152DF4F8883CF5DB3
:109DC000D040C153DF4F08811981CF5CD0400330B0
:109DD00011056CF484E50E948BB9882379F00E9408
:109DE00049B9C252DF4F8883CE5DD0400CC011E02C
:109DF000C252DF4F1883CE5DD04005C0C252DF4F44
:109E00001882CE5DD04088E50E94BAB9882321F03F
:109E10000E9428B9162F01C012E089E50E94BAB944
:109E2000882321F00E9428B9062F01C002E080E5B6
:109E30000E94BAB9811103C0212E302E04C00E94A5
:109E400028B9262E362E21E0221518F0E1E1FBE09C
:109E500004C031E0331568F0F9CF84918F010F5FB2
:109E60001F4F882311F40C947D5C0F940214F801A9
:109E7000F4CF83E50E94BAB9882319F00E9458B93B
:109E800004C060E070E88BEB95E420E030E040E750
:109E900052E40F94B71F6093820270938302809301
:109EA000840290938502C0904313D0904413E090B5
:109EB0004513F09046138CE40E94BAB9811109C091
:109EC00020E030E040E151E4C701B6010F94DA1E12
:109ED00002C00E9458B90F941F206B017C01CF5221
:109EE000DF4F79836883C15DD040809043139090A9
:109EF0004413A0904513B090461382E50E94BAB96E
:109F0000811109C020E030E040E953E4C501B4010B
:109F10000F94DB1E02C00E9458B90F941F204B0102
:109F20005C01C154DF4F79836883CF5BD0404090A0
:109F30004713509048136090491370904A1386E479
:109F40000E94BAB9811109C020E030E040E151E43B
:109F5000C301B2010F94DA1E02C00E9458B90F94D7
:109F60001F20C554DF4F688379838A839B83CB5B33
:109F7000D040C554DF4F08811981CB5BD040C75218
:109F8000DF4F19830883C95DD0404090471350903C
:109F900048136090491370904A1382E40E94BAB942
:109FA000811109C020E030E840E953E4C301B20167
:109FB0000F94DB1E02C00E9458B90F941F20CB5291
:109FC000DF4F688379838A839B83C55DD040CB5202
:109FD000DF4F08811981C55DD040CD53DF4F198314
:109FE0000883C35CD040B6010D2C000C880B990B84
:109FF0000F94A81ACC51DF4F688379838A839B839F
:10A00000C45ED04040904313509044136090451379
:10A010007090461320E030E048ED51E4C301B201F6
:10A020000F94DA1E9B01AC01CC51DF4F688179811E
:10A030008A819B81C45ED0400F94A21A11E0C9545A
:10A04000DF4F1883C75BD04087FD10C0C40109975C
:10A05000CF52DF4F08811981C15DD0400817190721
:10A060002CF4C954DF4F1882C75BD040B401990C5F
:10A07000880B990B0F94A81A4B015C0120E030E08B
:10A0800040E953E4C301B2010F94DB1E9B01AC0114
:10A09000C501B4010F94012118167CF029E0C20E0D
:10A0A000D11C01E0C154DF4F88819981CF5BD04042
:10A0B000C816D9061CF400E001C001E0C554DF4F0A
:10A0C000A881B981CB5BD040BD01BB0F880B990B38
:10A0D0000F94A81AC851DF4F688379838A839B83C2
:10A0E000C85ED040C0904713D0904813E090491309
:10A0F000F0904A1320E030E040EA51E4C701B60195
:10A100000F94DA1E9B01AC01C851DF4F6881798141
:10A110008A819B81C85ED0400F94A21A11E087FD0E
:10A1200011C0CB52DF4F88819981C55DD04009971E
:10A13000C752DF4FE881F981C95DD040E817F907C0
:10A140000CF410E0CB52DF4F28813981C55DD0403F
:10A15000B901330F880B990B0F94A81A4B015C01BE
:10A1600020E030E047E953E4C701B6010F94DB1E5D
:10A170009B01AC01C501B4010F9401211816A4F094
:10A18000C554DF4F88819981CB5BD0400996FF246D
:10A19000F394CD53DF4FA881B981C35CD0408A17B7
:10A1A0009B0724F4F12C02C0FF24F394C954DF4F21
:10A1B000B881C75BD040B1110BC0002321F082E011
:10A1C0009BE053DD0AC0111108C0F1100BC013C091
:10A1D0008AE09BE04ADD0111F2CF112319F08AEFEA
:10A1E0009AE043DDFF2011F40C947D5C83EF9AE04C
:10A1F0003CDD0C947D5CC153DF4F08811981CF5C3D
:10A20000D040012BF9F0ECEDFAE084918F010F5F63
:10A210001F4F882321F00F940214F801F6CFC1528A
:10A22000DF4F1881CF5DD040112361F0E3ECFAE0FD
:10A2300084918F010F5F1F4F882321F00F94021428
:10A24000F801F6CF0E94BEF81092BF12C152DF4F44
:10A250000881CF5DD04001110AC00F948E0D8AEEA7
:10A2600096E00E940D870E9467CB0E9438B881E07B
:10A270000E9423B4882349F0C352DF4F1881CD5D7B
:10A28000D0401093BF120C947D5C0E94A5BA85E467
:10A290000E948BB9582E882319F00E9449B9582E74
:10A2A000022D10E0C351DF4F19830883CD5ED040EB
:10A2B000032D10E0C151DF4F19830883CF5ED040DA
:10A2C000239C80011124CB52DF4F19830883C55D85
:10A2D000D040832D80958170C553DF4F8883CB5C40
:10A2E000D040000F111F000F111FCD50DF4F1983F9
:10A2F0000883C35FD040CB52DF4F08811981C55D11
:10A30000D04093E0000F111F9A95E1F7CF50DF4F37
:10A3100019830883C15FD040C554DF4F198218826A
:10A32000CB5BD04066246A94762CC154DF4F088101
:10A330001981CF5BD040CF52DF4F28813981C15D79
:10A34000D040021B130BC154DF4F19830883CF5B2E
:10A35000D040CD53DF4F08811981C35CD040C75234
:10A36000DF4F28813981C95DD040021B130BCD53CB
:10A37000DF4F19830883C35CD040C953DF4F288166
:10A3800039814A815B81C75CD040CA01B9010F9411
:10A3900087218111E9C2C553DF4F0881CB5CD040D2
:10A3A000002369F0CF52DF4F2882C15DD04001E029
:10A3B000C752DF4F0883C95DD040412C0FC04424F1
:10A3C0004A94420C1FEFC752DF4F1883C95DD0403B
:10A3D0000FEFCF52DF4F0883C15DD04081E0C553FE
:10A3E000DF4F1881CB5CD0401827C553DF4F18834F
:10A3F000CB5CD040C3010196880F991F880F991F2D
:10A400000DE310E00C0F1D1F080F191FC954DF4F7B
:10A4100019830883C75BD040C351DF4F088119817E
:10A42000CD5ED04001501109CB50DF4F1983088316
:10A43000C55FD040C151DF4F08811981CF5ED04048
:10A4400001501109C950DF4F19830883C75FD040FD
:10A45000C554DF4F88819981CB5BD040092E000C19
:10A46000AA0BBB0BC750DF4F88839983AA83BB839A
:10A47000C95FD040CF52DF4F1881C15DD040411637
:10A4800009F461C2C154DF4F88819981CF5BD0400C
:10A49000CB50DF4F68817981C55FD0400F94B721E1
:10A4A000072E000C880B990B0F94A81A6B017C01E6
:10A4B000642D042C000C770B880B990B0F94A81AB1
:10A4C0009B01AC01C701B6010F94071B9B01AC01B6
:10A4D000CC51DF4F688179818A819B81C45ED040F5
:10A4E0000F94DB1E4B015C01CD53DF4F88819981B6
:10A4F000C35CD040C950DF4F68817981C75FD040CD
:10A500000F94B721072E000C880B990B0F94A81AF3
:10A510006B017C01C750DF4F688179818A819B8103
:10A52000C95FD0400F94A81A9B01AC01C701B601C6
:10A530000F94071B9B01AC01C851DF4F68817981E3
:10A540008A819B81C85ED0400F94DB1E6B017C0129
:10A5500020E030E0A901C501B4010F94A21A87FDE3
:10A5600005C020E030E040E05FE303C020E030E0E1
:10A57000A901C501B4010F94DB1E0F945020C355EF
:10A58000DF4F688379838A839B83CD5AD04020E054
:10A5900030E0A901C701B6010F94A21A87FD05C0DA
:10A5A00020E030E040E05FE303C020E030E0A901BC
:10A5B000C701B6010F94DB1E0F945020C755DF4F23
:10A5C000688379838A839B83C95AD0409FEF691A35
:10A5D000790AE42DEE0FFF0BC554DF4F0881198176
:10A5E000CB5BD040E00FF11FEE0FFF1F21EA30E000
:10A5F0002C0F3D1FE20FF31F71826082C153DF4FAA
:10A600002881CF5CD040452DBE0167557F4FCE01DC
:10A6100083559F4F0F940001C953DF4F688379839F
:10A620008A839B83C75CD0409B01AC010F94872138
:10A63000882341F0C352DF4F0881CD5DD0400093A5
:10A64000BF1281C1C953DF4F288139814A815B81A3
:10A65000C75CD040C052DF4F688179818A819B817D
:10A66000C05ED0400F94DB1EC052DF4F68837983F9
:10A670008A839B83C05ED040F301EE0FFF1FEE0F75
:10A68000FF1F2DE630E02C0F3D1FE20FF31FC953D3
:10A69000DF4F88819981AA81BB81C75CD0408083CC
:10A6A0009183A283B383C355DF4F88809980AA80AA
:10A6B000BB80CD5AD040C954DF4FA881B981C75B58
:10A6C000D0408D929D92AD92BC921397C755DF4FAB
:10A6D000C880D980EA80FB80C95AD040FD01CD50A6
:10A6E000DF4F08811981C35FD040E00FF11FC082A6
:10A6F000D182E282F382FD01CF50DF4F08811981C0
:10A70000C15FD040E00FF11F80E090E0A0E8BFE320
:10A7100080839183A283B383A501940169817A81A7
:10A720008B819C810F94DB1E69837A838B839C834E
:10A73000A70196016D817E818F8198850F94DB1E24
:10A740006D837E838F839887C953DF4F288139813A
:10A750004A815B81C75CD04069857A858B859C8501
:10A760000F94DB1E69877A878B879C87A5019401EC
:10A77000C501B4010F94071B9B01AC016D857E855B
:10A780008F8598890F94DB1E6D877E878F87988BC6
:10A79000A7019601C701B6010F94071B9B01AC01ED
:10A7A00069897A898B899C890F94DB1E698B7A8BE6
:10A7B0008B8B9C8BC953DF4F288139814A815B8108
:10A7C000C75CD040CA01B9010F94071B9B01AC01C3
:10A7D0006D897E898F89988D0F94DB1E6D8B7E8BA2
:10A7E0008F8B988FA7019601C501B4010F94071BA9
:10A7F0009B01AC01698D7A8D8B8D9C8D0F94DB1E36
:10A80000698F7A8F8B8F9C8FC953DF4F2881398155
:10A810004A815B81C75CD040C501B4010F94071B1E
:10A820009B01AC016D8D7E8D8F8D98A10F94DB1EE9
:10A830006D8F7E8F8F8F98A3C953DF4F2881398109
:10A840004A815B81C75CD040C701B6010F94071BEA
:10A850009B01AC0169A17AA18BA19CA10F94DB1E85
:10A8600069A37AA38BA39CA3E894B7F80DA1C35264
:10A87000DF4F0883CD5DD0401EA1C451DF4F188348
:10A88000CC5ED0400FA118A5C352DF4F2881CD5D0B
:10A89000D040C451DF4F3881CC5ED040A801C50103
:10A8A000B4010F94012118165CF0C352DF4F888069
:10A8B000CD5DD040C451DF4F9880CC5ED040580170
:10A8C0008DA29EA2AFA2B8A6E894F7F8A9A4BAA454
:10A8D0000BA51CA59501A801C701B6010F94012184
:10A8E000181614F065017801C9A6DAA6EBA6FCA635
:10A8F00020E030E040E85FE369AD7AAD8BAD9CAD20
:10A900000F94DB1E69AF7AAF8BAF9CAF80E00F94E2
:10A91000360BC752DF4F0881C95DD040400EC95485
:10A92000DF4F08811981C75BD0400C5F1F4FC954AE
:10A93000DF4F19830883C75BD040C352DF4F1882B3
:10A94000CD5DD04097CDC554DF4F08811981CB5BD9
:10A95000D0400F5F1F4FC554DF4F19830883CB5B77
:10A96000D040031508F409CD80E00E9423B4882369
:10A9700041F0C352DF4F1881CD5DD0401093BF121C
:10A98000B3C7C953DF4F288139814A815B81C75CD6
:10A99000D040CA01B9010F9487218111A5C789ACA4
:10A9A0009AACABACBCAC20E030E0A901C501B4016D
:10A9B0000F94A21A882309F408C2A50194016981A1
:10A9C0007A818B819C810F94B71FC954DF4F6883B4
:10A9D00079838A839B83C75BD04069837A838B8327
:10A9E0009C83A50194016D817E818F8198850F9450
:10A9F000B71FC554DF4F688379838A839B83CB5B02
:10AA0000D0406D837E838F839887A50194016985EB
:10AA10007A858B859C850F94B71FC154DF4F68835F
:10AA200079838A839B83CF5BD04069877A878B87C2
:10AA30009C87A50194016D857E858F8598890F94EB
:10AA4000B71F6B017C01C954DF4F288139814A81CE
:10AA50005B81C75BD040CA01B9010F94071B9B0102
:10AA6000AC01C701B6010F94DA1EC553DF4F6883EE
:10AA700079838A839B83CB5CD0406D877E878F8769
:10AA8000988BA501940169897A898B899C890F9497
:10AA9000B71F6B017C01C554DF4F288139814A8182
:10AAA0005B81CB5BD040CA01B9010F94071B9B01AE
:10AAB000AC01C701B6010F94DA1ECF52DF4F688395
:10AAC00079838A839B83C15DD040698B7A8B8B8B22
:10AAD0009C8BA50194016D897E898F89988D0F9437
:10AAE000B71F6B017C01C154DF4F288139814A8136
:10AAF0005B81CF5BD040CA01B9010F94071B9B015A
:10AB0000AC01C701B6010F94DA1E6D8B7E8B8F8B63
:10AB1000988FA5019401698D7A8D8B8D9C8D0F94F2
:10AB2000B71F6B017C01C554DF4F288139814A81F1
:10AB30005B81CB5BD040C954DF4F688179818A81CA
:10AB40009B81C75BD0400F94071B9B01AC01C701E1
:10AB5000B6010F94DA1ECD53DF4F688379838A8361
:10AB60009B83C35CD040698F7A8F8B8F9C8FA501AC
:10AB7000940169A17AA18BA19CA10F94B71F6B01CD
:10AB80007C01C154DF4F288139814A815B81CF5BD1
:10AB9000D040C554DF4F688179818A819B81CB5B2E
:10ABA000D0400F94071B9B01AC01C701B6010F9465
:10ABB000DA1E6B017C0169A37AA38BA39CA3A50178
:10ABC00094016D8D7E8D8F8D98A10F94B71F4B01D1
:10ABD0005C01C154DF4F288139814A815B81CF5BA1
:10ABE000D040C954DF4F688179818A819B81C75BDE
:10ABF000D0400F94071B9B01AC01C501B4010F9419
:10AC0000DA1E4B015C016D8F7E8F8F8F98A3CF5220
:10AC1000DF4F288139814A815B81C15DD040C553B6
:10AC2000DF4F688179818A819B81CB5CD0400F9412
:10AC3000071B2B013C01CD53DF4F288139814A810D
:10AC40005B81C35CD040CA01B9010F94071B9B0113
:10AC5000AC01C301B2010F94DA1EC752DF4F688303
:10AC600079838A839B83C95DD0402B013C01E894A2
:10AC700077F829A53AA54BA55CA56DA17EA18FA16A
:10AC800098A50F94DB1E2FEF36EE4BED5EE20F948E
:10AC9000071B9B01AC01C301B2010F94A21A181645
:10ACA0000CF093C0CD53DF4F288139814A815B81FD
:10ACB000C35CD040C701B6010F94071B2B013C01B8
:10ACC000CF52DF4F288139814A815B81C15DD040FD
:10ACD000C501B4010F94071B9B01AC01C301B20174
:10ACE0000F94DA1EC752DF4F288139814A815B8178
:10ACF000C95DD0400F94B71F2B013C016DA77EA703
:10AD00008FA798ABCD53DF4F288139814A815B8172
:10AD1000C35CD040C501B4010F94071B4B015C011B
:10AD2000C553DF4F288139814A815B81CB5CD0409C
:10AD3000C701B6010F94071B9B01AC01C501B4010B
:10AD40000F94DA1EC752DF4F288139814A815B8117
:10AD5000C95DD0400F94B71F6B017C0169AB7AAB22
:10AD60008BAB9CABC954DF4F288139814A815B8111
:10AD7000C75BD040C301B2010F94071B9B01AC011C
:10AD8000C154DF4F688179818A819B81CF5BD0403C
:10AD90000F94DB1E4B015C01C554DF4F28813981C4
:10ADA0004A815B81CB5BD040C701B6010F94071B82
:10ADB0009B01AC01C501B4010F94DB1EDC01CB018A
:10ADC000B0588DAB9EABAFABB8AFCDA4DEA4EFA4B3
:10ADD000F8A82601370177FA709477F8709489A85B
:10ADE0009AA8ABA8BCA88DA99EA9AFA9B8ADC95413
:10ADF000DF4F88839983AA83BB83C75BD040CB5244
:10AE0000DF4F08811981C55DD040B801110F880B53
:10AE1000990B0F94A81A9B01AC01C052DF4F6881B7
:10AE200079818A819B81C05ED0400F94B71FC55342
:10AE3000DF4F688379838A839B83CB5CD040C15387
:10AE4000DF4F08811981CF5CD040012B09F461C02C
:10AE5000EDEAFAE084918F010F5F1F4F882321F004
:10AE60000F940214F801F6CF48E0C301B2010F9429
:10AE7000DB14E8EAFAE084918F010F5F1F4F88230B
:10AE800021F00F940214F801F6CF48E0C501B40197
:10AE900090580F94DB14E3EAFAE084918F010F5F7E
:10AEA0001F4F882321F00F940214F801F6CFC954E4
:10AEB000DF4F688179818A819B81C75BD040905840
:10AEC00048E00F94DB148AE00F940214C153DF4F63
:10AED00008811981CF5CD04003301105D4F0EAE835
:10AEE000FAE084918F010F5F1F4F882321F00F94A8
:10AEF0000214F801F6CF48E0C553DF4F688179812D
:10AF00008A819B81CB5CD0400F94DB148AE00F9444
:10AF10000214C152DF4F1881CF5DD0401111D1C151
:10AF2000CB56DF4FC882D982EA82FB82C559D04016
:10AF3000C756DF4F88829982AA82BB82C959D04006
:10AF4000C12CD12C60E8E62E6FE3F62EC356DF4FFE
:10AF5000C882D982EA82FB82CD59D040CE018B567D
:10AF60009F4F0E94F0D4C757DF4FC882D982EA8230
:10AF7000FB82C958D040C357DF4F188219821A820A
:10AF80001B82CD58D040CF56DF4F488259826A820B
:10AF90007B82C159D040CE0187579F4F0E94F0D489
:10AFA000CB56DF4F88819981AA81BB81C559D0409A
:10AFB000C954DF4F88839983AA83BB83C75BD04082
:10AFC000C756DF4F488059806A807B80C959D0407E
:10AFD000C356DF4F88809980AA80BB80CD59D0406E
:10AFE000C757DF4F088119812A813B81C958D0405A
:10AFF000C554DF4F088319832A833B83CB5BD04042
:10B00000C357DF4F88819981AA81BB81CD58D04039
:10B01000C154DF4F88839983AA83BB83CF5BD04021
:10B02000CF56DF4FC880D980EA80FB80C159D0401D
:10B03000A7019601C301B2010F94071BCD53DF4F47
:10B04000688379838A839B83C35CD040C154DF4F7C
:10B05000288139814A815B81CF5BD040C501B40131
:10B060000F94071B9B01AC01CD53DF4F68817981A1
:10B070008A819B81C35CD0400F94DA1EC358DF4F96
:10B08000688379838A839B83CD57D040C554DF4F33
:10B09000288139814A815B81CB5BD040C501B401F5
:10B0A0000F94071B4B015C01A7019601C954DF4FA8
:10B0B000688179818A819B81C75BD0400F94071B8F
:10B0C0009B01AC01C501B4010F94DA1ECF57DF4FCD
:10B0D000688379838A839B83C158D040C154DF4FF2
:10B0E000288139814A815B81CF5BD040C954DF4FD1
:10B0F000688179818A819B81C75BD0400F94071B4F
:10B100006B017C01C554DF4F288139814A815B8105
:10B11000CB5BD040C301B2010F94071B9B01AC0174
:10B12000C701B6010F94DA1ECB57DF4F68837983CE
:10B130008A839B83C558D040CE0183589F4F0E947D
:10B14000F0D4C757DF4F088119812A813B81C95844
:10B15000D040C357DF4F488059806A807B80CD58EC
:10B16000D040CF56DF4F88809980AA80BB80C159DC
:10B17000D040C358DF4F88819981AA81BB81CD57C8
:10B18000D040C954DF4F88839983AA83BB83C75BB0
:10B19000D040CF57DF4F88819981AA81BB81C158A8
:10B1A000D040C554DF4F88839983AA83BB83CB5B90
:10B1B000D040CB57DF4F88819981AA81BB81C55888
:10B1C000D040C154DF4F88839983AA83BB83CF5B70
:10B1D000D040CB56DF4FC880D980EA80FB80C5596C
:10B1E000D040C756DF4F488159816A817B81C95958
:10B1F000D040C356DF4F88819981AA81BB81CD5948
:10B20000D0400093000A1093010A2093020A309361
:10B21000030A4092040A5092050A6092060A70924C
:10B22000070A8092080A9092090AA0920A0AB0922C
:10B230000B0AC954DF4F088119812A813B81C75B02
:10B24000D04000930C0A10930D0A20930E0A3093FD
:10B250000F0AC554DF4F088119812A813B81CB5BDE
:10B26000D0400093100A1093110A2093120A3093D1
:10B27000130AC154DF4F088119812A813B81CF5BBA
:10B28000D0400093140A1093150A2093160A3093A5
:10B29000170AC092180AD092190AE0921A0AF0927C
:10B2A0001B0A40931C0A50931D0A60931E0A709358
:10B2B0001F0A8093200A9093210AA093220AB09338
:10B2C000230AC252DF4F1881CE5DD040112309F40A
:10B2D0006CC2E7ECF9E084918F010F5F1F4F882368
:10B2E00021F00F940214F801F6CFCC24CA94C30CB9
:10B2F000DC2CC554DF4F1882CB5BD04000ECC1542E
:10B30000DF4F0883CF5BD04019E7CD53DF4F188361
:10B31000C35CD04004E4C252DF4F0883CE5DD0400E
:10B320008E010B561F4FCF54DF4F19830883C15B2B
:10B33000D0400C501109CD54DF4F19830883C35BF3
:10B34000D0400C501109CB54DF4F19830883C55BE3
:10B35000D040D7FC29C10D2D000F110BCF52DF4F6C
:10B3600019830883C15DD040C954DF4F1982188208
:10B37000C75BD040312CC954DF4FE881F981C75BEE
:10B38000D040CF52DF4F08811981C15DD040E00F1E
:10B39000F11F21EA30E02C0F3D1FE20FF31F008167
:10B3A00011817801EE0CFF1CEE0CFF1CEDE6F0E0C5
:10B3B000EC0FFD1FEE0DFF1D4080518062807380F9
:10B3C000C553DF4F288139814A815B81CB5CD040F6
:10B3D000C301B2010F94DA1E4B015C01E1E0F0E021
:10B3E000EC0FFD1FEE0DFF1D84AD95ADA6ADB7AD05
:10B3F000CB56DF4F88839983AA83BB83C559D0403E
:10B40000CB52DF4FE881F981C55DD040E00FF11FDD
:10B41000EE0FFF1FEE0FFF1F81E090E08C0F9D1FCE
:10B42000E80FF91F84AD95ADA6ADB7ADC757DF4F97
:10B4300088839983AA83BB83C958D040C358DF4F00
:10B44000188219821A821B82CD57D040CA54DF4F0E
:10B450009881C65BD0409F93CB54DF4FA881C55BDA
:10B46000D040AF93CC54DF4FB881C45BD040BF9382
:10B47000CD54DF4FE881C35BD040EF93CE54DF4F14
:10B48000F881C25BD040FF93CF54DF4F0881C15B8E
:10B49000D0400F932DB73EB7245231090FB6F89420
:10B4A0003EBF0FBE2DBFADB7BEB71196E0E0FAE0CC
:10B4B00084E201900D928A95E1F70E940BD4C35863
:10B4C000DF4F288139814A815B81CD57D040C3014C
:10B4D000B2010F94DA1E7B018C010FB6F894DEBF27
:10B4E0000FBECDBF9B01AC01C554DF4F6881CB5B64
:10B4F000D040C154DF4F7881CF5BD040CD53DF4F78
:10B500008881C35CD040C252DF4F9881CE5DD0406D
:10B510000F9401211816A4F4C554DF4FE882CB5BC9
:10B52000D040C154DF4FF882CF5BD040CD53DF4FC6
:10B530000883C35CD040C252DF4F1883CE5DD04039
:10B5400020E030E0A901C501B4010F94012187FD7D
:10B550000CC0E4ECF9E084918F010F5F1F4F88234A
:10B5600039F00F940214F801F6CF80E20F94021420
:10B5700045E0C501B4010F94DB143394C954DF4F87
:10B5800008811981C75BD0400C5F1F4FC954DF4F42
:10B5900019830883C75BD040321408F4ECCE8AE0EC
:10B5A0000F940214DA94D5CE8AE00F940214C1539A
:10B5B000DF4F08811981CF5CD0400430110509F0BC
:10B5C000F4C0EBE9F9E084918F010F5F1F4F811107
:10B5D0000CC03E0115E9610E711C2E0129E8420ED6
:10B5E000511C8E0103581F4F16C00F940214F8010E
:10B5F000EACF80E20F94021445E0C501B4010F9434
:10B60000DB14D394F4E0EF0EF11CD214A0F08AE026
:10B610000F940214CA94C7FCC4C02C2D220F330B04
:10B62000C153DF4F39832883CF5CD040E12CF12C0C
:10B63000D12C84E2382EC153DF4FE881F981CF5CF1
:10B64000D040EE0DFF1D81EA90E08C0F9D1FE80FAA
:10B65000F91F808191815C01AA0CBB1CAA0CBB1C48
:10B66000E1E0F0E0EC0FFD1FEA0DFB1D44AD55AD30
:10B6700066AD77ADD3014D935D936D937C93139736
:10B68000CB52DF4FE881F981C55DD040E80FF91F4B
:10B69000EE0FFF1FEE0FFF1F21E030E02C0F3D1FCC
:10B6A000E20FF31F84AD95ADA6ADB7ADF201808377
:10B6B0009183A283B383D8011D921D921D921C9287
:10B6C00013971F930F935F924F927F926F92EDB7F4
:10B6D000FEB7B4970FB6F894FEBF0FBEEDBFADB77F
:10B6E000BEB71196E0E0FAE0832D01900D928A95A5
:10B6F000E1F70E940BD4EDE6F0E0EC0FFD1FEA0D40
:10B70000FB1DD8012D913D914D915C91608171811E
:10B71000828193810F94DA1EC554DF4F2881CB5B61
:10B72000D040C154DF4F3881CF5BD040CD53DF4F85
:10B730004881C35CD040C252DF4F5881CE5DD040BB
:10B740000F94DA1E4B015C010FB6F894DEBF0FBEFA
:10B75000CDBF20E030E0A9010F94012187FD49CF42
:10B76000E8E9F9E084919F012F5F3F4F882309F4B6
:10B7700043CFC350DF4F2883CD5FD040C250DF4F4F
:10B780003883CE5FD0400F940214C350DF4F28811E
:10B79000CD5FD040C250DF4F3881CE5FD040F9013D
:10B7A000E1CF8AE00F94021408C0C153DF4F088133
:10B7B0001981CF5CD040012B21F089E799E00E94EC
:10B7C0004CB1C152DF4F1881CF5DD040111185C0FF
:10B7D0008CE0EBE0F7E0DE01A358BF4F01900D9243
:10B7E0008A95E1F781E08093BF12CE0183589F4F85
:10B7F0000E940D87C355DF4F288139814A815B81C3
:10B80000CD5AD04060910B0770910C0780910D07C5
:10B8100090910E070F94DA1E6B017C012DEB37E33C
:10B8200046E855EB0F94012187FD4BC02DEB37E324
:10B8300046E855E3C701B6010F94A21A18160CF496
:10B8400040C0C755DF4F288139814A815B81C95A81
:10B85000D04060910F07709110078091110790916F
:10B8600012070F94DA1E6B017C012DEB37E346E8DB
:10B8700055EB0F94012187FD24C02DEB37E346E8FB
:10B8800055E3C701B6010F94A21A1816D4F0C95394
:10B89000DF4F288139814A815B81C75CD04060914C
:10B8A00013077091140780911507909116070F9454
:10B8B000DA1ECB57DF4F688379838A839B83C55811
:10B8C000D0408CE0FE01E358FF4FABE0B7E00190C1
:10B8D0000D928A95E1F781E005C0C352DF4F888160
:10B8E000CD5DD0408093BF120E948CBA0E94A87098
:10B8F0008091BF1281110E9438B8C250DF4F0FB63D
:10B90000F894DEBF0FBECDBFDF91CF911F910F9195
:10B91000FF90EF90DF90CF90BF90AF909F908F906F
:10B920007F906F905F904F903F902F9008952F924F
:10B930003F924F925F926F927F928F929F92AF92BF
:10B94000BF92CF92DF92EF92FF920F931F93CF930C
:10B95000DF93CDB7DEB762970FB6F894DEBF0FBEA8
:10B96000CDBF082F11E01093D10424982C9A089889
:10B97000109A0E94BEF82091BF12298B80E00E948D
:10B98000FFB20E94A5BA1093D004011119C088E536
:10B990000E948BB9382E89E50E948BB9182F8AE551
:10B9A0000E948BB9282E311006C0111113C08823B4
:10B9B00069F0312E10C0112369F0312E082F0BC011
:10B9C0003324339411E02224239402C0382E182FFC
:10B9D00001E001C000E00E9473B4011105C0311004
:10B9E00003C0112309F414C120E030E040EA50E420
:10B9F00060914B1370914C1380914D1390914E13A5
:10BA00000F94DB1E60933C0D70933D0D80933E0DB3
:10BA100090933F0D20911307309114074091150723
:10BA2000509116070F94012118165CF419821A829E
:10BA30001B821C82BE016F5F7F4F8CE39DE00E94E2
:10BA40006CB401110CC0332009F40EC2111107C0EF
:10BA500080E00E9471CB002309F406C2CEC0109290
:10BA60000F071092100710921107109212071092F0
:10BA70000B0710920C0710920D0710920E070E94F0
:10BA800038B8E9EFF7E284918A8BEDEEF7E2C590E2
:10BA9000D590E590F490E1EFF7E285909590A59030
:10BAA000B490A5019401C701B6010F9401211816A5
:10BAB0002CF4A7019601C501B40104C0A5019401AD
:10BAC000C701B6010F94B71F6D877E878F87988B4C
:10BAD0008CEA682E87E2782EF30165917591859145
:10BAE000949120EB422E27E2522EF20125913591BE
:10BAF000459154910F94A21A87FF02C0F30101C02F
:10BB0000F20145905590659074902D853E854F8546
:10BB10005889CA01B9010F94071B20E030E040E8C2
:10BB20005FE30F94DB1E0F9446219B01AC01C30120
:10BB3000B2010F94071B69877A878B879C87EAEF8E
:10BB4000F7E294919D8720E030E040EC5FE3C5018F
:10BB5000B4010F94071B2B013C01AD856A2FAA0F7E
:10BB6000770B880B990B0F94A81A9B01AC01C301AA
:10BB7000B2010F94071B69837A838B839C8320E037
:10BB800030E040EC5FE3C701B6010F94071B6B0187
:10BB90007C01BA896B2FBB0F770B880B990B0F9425
:10BBA000A81A9B01AC01C701B6010F94071B6D8356
:10BBB0007E838F839887AE01475F5F4FBE016F5FC3
:10BBC0007F4FCE0105960E9468B41092F60610923F
:10BBD0000F0710921007109211071092120710927F
:10BBE0000B0710920C0710920D0710920E0701110F
:10BBF0002FCF31102DCF112359F081E00E9471CB4E
:10BC0000002309F437C18091CC04811104C007C01E
:10BC10002110F9CFB6C08091CD04811120C060E021
:10BC20008AE499E00E9433D6E7E4F6E284917F014A
:10BC30002FEFE21AF20A882321F00F940214F70181
:10BC4000F5CFEBE3F9E084917F019FEFE91AF90A60
:10BC5000882309F496C00F940214F701F4CF0E94D0
:10BC600038B840904313509044136090451370903F
:10BC7000461320E030E048E951E4C301B2010F94DB
:10BC8000DA1E4B015C016093340D7093350D809387
:10BC9000360D9093370D8091471390914813A091E2
:10BCA0004913B0914A138D879E87AF87B88B20E0E8
:10BCB00030E041E853E4BC01CD010F94DB1E6B0181
:10BCC0007C016093380D7093390D80933A0D9093F9
:10BCD0003B0D8091130790911407A0911507B09127
:10BCE000160780933C0D90933D0DA0933E0DB093AD
:10BCF0003F0DA3019201C501B4010F94DA1E4B015F
:10BD00005C012CE032E048ED51EC0F94012187FDFD
:10BD10008BC021E230E040E953E4C501B4010F9447
:10BD2000A21A18160CF480C02D853E854F855889BF
:10BD3000C701B6010F94DA1E6B017C012CE032E0E2
:10BD400040EA51EC0F94012187FD6EC021E230E002
:10BD500047E953E4C701B6010F94A21A18160CF470
:10BD600063C019821A821B821C82AE014F5F5F4F33
:10BD700068E37DE084E39DE00E9468B482E00E9475
:10BD800071CB0E9438B8002301F10E94BEF81092D6
:10BD900013071092140710921507109216070E94AD
:10BDA00038B81D821E821F82188680E090E0A0E2D3
:10BDB000B1E489839A83AB83BC83BE016B5F7F4F01
:10BDC000CE0101960E946CB402C02110DECF80919A
:10BDD000CF048093D00489890E94FFB20E948CBA5C
:10BDE00083E0809320020E94A8701092D104249ACC
:10BDF0002C98089A109862960FB6F894DEBF0FBE82
:10BE0000CDBFDF91CF911F910F91FF90EF90DF9009
:10BE1000CF90BF90AF909F908F907F906F905F90EA
:10BE20004F903F902F90089560E08AE299E00E9441
:10BE300033D6E7E4F6E284917F019FEFE91AF90A2D
:10BE4000882321F00F940214F701F5CFE8E1F9E01F
:10BE500084917F01AFEFEA1AFA0A882309F491CF9F
:10BE60000F940214F701F4CF112309F4D1CE81E02D
:10BE70000E9471CB2110C7CE0E9438B8A8CFCF93B3
:10BE8000DF93CDB7DEB727970FB6F894DEBF0FBEAE
:10BE9000CDBF0E94B8AF81113BC080E50E94BAB906
:10BEA000882319F00E9428B901C060E06F8383E500
:10BEB0000E94BAB9882319F00E9428B901C06CE029
:10BEC0006E8384E50E94BAB9882319F00E9428B9CC
:10BED00001C063E06D8382E50E94BAB9882319F03E
:10BEE0000E9458B904C060E070E080ED90E469837E
:10BEF0007A838B839C839E012B5F3F4FAE014F5F04
:10BF00005F4FBE016A5F7F4FCE0107960E9406CD4C
:10BF100027960FB6F894DEBF0FBECDBFDF91CF914D
:10BF20000895CF92DF92EF92FF9280E50E94BAB916
:10BF3000882329F00E9418B96B017C0103C0C12C31
:10BF4000D12C760183E50E94BAB9882361F00E9462
:10BF500058B920E030E04AE754E40F94071B0F94EF
:10BF600024206B017C010E94BEF880912102811186
:10BF700005C060E08FE099E00E9433D60E9482BA4B
:10BF80008091731490917414A0917514B0917614EB
:10BF9000C80ED91EEA1EFB1E0E94ACC1DC01CB01FB
:10BFA0008C199D09AE09BF09B7FF04C080E00F944A
:10BFB000360BF2CFFF90EF90DF90CF9008958091F5
:10BFC000AE048630D8F496E0899FF0011124E6573C
:10BFD000FB4F209180023091810231832083409178
:10BFE00024135091251360912613709127134283D7
:10BFF0005383648375838F5F8093AE04089520918B
:10C0000080023091810228173907D9F0909381027C
:10C01000809380024093241350932513609326133A
:10C02000709327138252904621F4109204131092B9
:10C03000AE0482E08093200281E08093A1121092EE
:10C04000101308954F925F926F927F928F929F92FA
:10C05000AF92BF92FF920F931F93CF93DF93CDB711
:10C06000DEB72A970FB6F894DEBF0FBECDBF109291
:10C070000F1380911613882349F00F94C90940E0EB
:10C0800050E0BA018EED90E0BADFC8C420916F0293
:10C090003091700240912413509125136091261322
:10C0A00070912713C901840F951F2436310524F49C
:10C0B000853691053CF416C02436310531F08436BE
:10C0C000910584F484E690E00DC04B305105610584
:10C0D000710514F00A9706C0463F5F4F6F4F7F4FC0
:10C0E0006CF40A969093700280936F02109224135E
:10C0F00010922513109226131092271380916F022D
:10C10000909170028A3091053CF0883E43E094079C
:10C110002CF087EE93E002C08AE090E090937002EA
:10C1200080936F020E94C0FFF82E0E94D4D58091A8
:10C13000FA09853198F4FF2049F080914B049091E1
:10C140004C04892B19F000E617E102C003E416E164
:10C1500023E14FE061E089E00E9493C38091FA09F6
:10C160008D3108F084C1883008F03FC08091BE094D
:10C17000F11002C0811139C06091510470915204D4
:10C18000072E000C880B990B0F94A81A20E030E0C2
:10C1900040E05FE30F94DB1E0F941F2064367105AF
:10C1A0002CF46A30710524F446E003C042E101C07A
:10C1B0004CE022E130E0241B310937FF02C02F5F41
:10C1C0003F4F359527953195219531092B5F209368
:10C1D000FD0927E02093FE09CB010E94ADD10F9409
:10C1E0007D0A80E496E10F94700A8091FA098D31FE
:10C1F000D0F58091FC098531B0F120E030E040E0DD
:10C200005FE36091AC127091AD128091AE1290918B
:10C21000AF120F94DB1E0F941F209B016436710533
:10C220000CF0F7C22A3031050CF0F1C246E022E1F1
:10C2300030E0241B310937FF02C02F5F3F4F359597
:10C2400027953195219531092B5F2093FD092CE12C
:10C250002093FE09CB010E94ADD10F947D0A80E4AA
:10C2600096E10F94700A8091FA09853140F580912A
:10C27000FC09813120F16091510470915204072E24
:10C28000000C880B990B0F94A81A2091AC123091D6
:10C29000AD124091AE125091AF120F9401211816B9
:10C2A0000CF0B9C21092E60902E022E041E16DE033
:10C2B00086EC99E00E947FBE81E08093E609809140
:10C2C000FA09883008F03FC08091B509F11002C02A
:10C2D000811139C060914F0470915004072E000CF9
:10C2E000880B990B0F94A81A20E030E040E05FE340
:10C2F0000F94DB1E0F941F20643671052CF46A30F6
:10C30000710524F446E003C042E101C04CE022E1A3
:10C3100030E0241B310937FF02C02F5F3F4F3595B6
:10C3200027953195219531092F5A2093FD0927E052
:10C330002093FE09CB010E94ADD10F947D0A80E4C9
:10C3400096E10F94700A8091FA098D31D0F58091B1
:10C35000FC098531B0F120E030E040E05FE360911E
:10C36000AF047091B0048091B1049091B2040F9425
:10C37000DB1E0F941F209B01643671050CF056C222
:10C380002A3031050CF050C246E022E130E0241B97
:10C39000310937FF02C02F5F3F4F35952795319503
:10C3A000219531092F5A2093FD092CE12093FE0994
:10C3B000CB010E94ADD10F947D0A80E496E10F94E9
:10C3C000700A8091FA09853140F58091FC0981312C
:10C3D00020F160914F0470915004072E000C880BDF
:10C3E000990B0F94A81A2091AF043091B00440919A
:10C3F000B1045091B2040F94012118160CF018C228
:10C400001092E60902E022E042E168E586EC99E05C
:10C410000E947FBE81E08093E6098091FA098C3109
:10C4200030F58091FC09843110F180914B0490919A
:10C430004C04019644E6489F9001499F300D112419
:10C4400037FF02C021503F4F832F932F990F990B35
:10C45000009769F028E62093FD092BE12093FE095F
:10C460000E94ADD10F947D0A85E20E948FC4809115
:10C47000FA09843328F48091FC098A3208F0E1C17A
:10C480008091FA09853328F48091FC09813308F002
:10C49000FEC18091770A882309F44BC08091FA0984
:10C4A000843308F046C08091FC09823308F441C00F
:10C4B00020916C0C222319F18091160D9091170D8B
:10C4C000A091180DB091190D0097A105B10509F4BF
:10C4D000E3C1BC01CD016D597F4F8F4F9F4F24E6C3
:10C4E00030E040E050E00F947D1E60911A0D709195
:10C4F0001B0D80911C0D90911D0D0F947D1E88E4E5
:10C50000289FB0011124072E000C880B990B0F9463
:10C51000A81A2AE037ED43E25CE30F94071B0F945F
:10C520002420262F02E042E367E386EC99E00E9494
:10C530007FBE8091FA09813308F060C08091FC09C8
:10C54000893208F45BC00E94BBC62B013C018CE31E
:10C55000882E912CA12CB12CC301B201A50194010C
:10C560000F947D1ECA01B901A50194010F947D1E8F
:10C57000CA01962E872E59018E010F5F1F4F41E889
:10C58000441641E5540641E06406710408F486C18E
:10C59000B90128E130E040E050E00F947D1E290110
:10C5A0003A018F929F92C50168E170E00F94A32138
:10C5B0009F938F935F924F9280E89BE09F938F931E
:10C5C0001F930F930F943B1A0FB6F894DEBF0FBE64
:10C5D000CDBF9AE0491651046104710408F08DC181
:10C5E00097E0892F880F980F9195955A9093FD09A0
:10C5F00080E38093FE09C8010F947D0AE091C00991
:10C60000F091C10984818111CEC060910B077091B6
:10C610000C0780910D0790910E070F941F20CB01FE
:10C620000E9446D1BC018FEB94E00F9419226091D7
:10C630000F077091100780911107909112070F94C6
:10C640001F20CB010E9446D1BC018AEB94E00F94DD
:10C6500019222CEA35EC47E257E3609113077091F9
:10C66000140780911507909116070F94DB1E20E0A8
:10C6700030E048EC52E40F94071B0F941F204B014D
:10C680005C0197FD19C090E1891697E29906A10413
:10C69000B104E4F0C501B40120E137E240E050E02C
:10C6A0000F949F1ECA01B9012AE030E040E050E03B
:10C6B0000F949F1E605D0BC0B094A09490948094E2
:10C6C000811C911CA11CB11C6DE201C060E2609351
:10C6D0001A1328EE821623E09206A104B10494F006
:10C6E000C501B40128EE33E040E050E00F949F1EF6
:10C6F000CA01B9012AE030E040E050E00F949F1EEB
:10C70000605D01C060E260931B13C501B40124E6C3
:10C7100030E040E050E00F949F1E9AE0492E512CEB
:10C72000612C712CCA01B901A30192010F949F1EC3
:10C73000605D60931C13C501B401A30192010F94C5
:10C740009F1E4B015C01672B682B692B79F08EE2F1
:10C7500080931D13CA01B901A30192010F949F1E7A
:10C76000605D60931E1380E3880D15C0CA01B90196
:10C77000A30192010F949F1E662339F08EE28093ED
:10C780001D13605D60931E1305C080E280931E132D
:10C7900080931D1380E280931F136AE173E183EBA2
:10C7A00094E00F9419228091FA098632A8F48091BE
:10C7B000FC098E3188F008E020E84EE160E086EC6C
:10C7C00099E00E947FBE8091FA09863228F4809118
:10C7D000FC098F3108F093C08091FA09823328F464
:10C7E0008091FC098C3208F0FAC08091FA098F33ED
:10C7F00008F014C18091FC09883308F40FC110922D
:10C80000FD098EE38093FE090E9466C507C14CE0D6
:10C810000ECD42E10CCD02E022E041E16DE086EC7C
:10C8200099E00E947FBE4BCD4CE0AFCD42E1ADCD53
:10C8300002E022E042E168E586EC99E00E947FBEDA
:10C84000ECCD07E028E04AE26AE286EC99E00E943B
:10C850007FBE05E022E04CE262E386EC99E00E94B4
:10C860007FBE6AE08AE20E94E7C36091C8097091C6
:10C87000C90982E38093E2098BE28093E30922EE07
:10C8800039E042E386EC99E00E94BDBCF9CD6AE450
:10C8900086E30E94E7C3FDCD20E031CE44E6A41636
:10C8A000B104C0F48F929F92C50168E170E00F94CB
:10C8B000A3219F938F9386E79BE09F938F931F9372
:10C8C0000F930F943B1A0FB6F894DEBF0FBECDBF87
:10C8D00095E087CE8F929F923F932F938EE69BE0B9
:10C8E0009F938F931F930F930F943B1A0FB6F89457
:10C8F000DEBF0FBECDBF96E074CE98E072CE109230
:10C90000E60983E08093FD0985E28093FE09FF201C
:10C9100029F08EE396E10F94700A0DC080912B07E9
:10C92000811102C08FE305C08091CC048111F1CF49
:10C9300080E20E948FC48BE08093FD0915E2109382
:10C94000FE098FEB94E00F947D0A8BE28093FD0942
:10C950001093FE09FF2029F08CE396E10F94700AF2
:10C960000DC080912C07811102C08FE305C080911A
:10C97000CD048111F1CF80E20E948FC483E38093C4
:10C98000FD0915E21093FE098AEB94E00F947D0AED
:10C9900083E58093FD091093FE09FF2029F08AE3C7
:10C9A00096E10F94700A0DC080912D07811102C08D
:10C9B0008FE305C08091CE048111F1CF80E20E9407
:10C9C0008FC48BE58093FD0985E28093FE0983EB9C
:10C9D00094E00F947D0A81E08093E609FDCE84E027
:10C9E0000F942B0A83E08093FD0912E31093FE0954
:10C9F00086E00F945C0A0E94D4D58CE08093FD09F8
:10CA00001093FE0980916F02909170020E94ADD147
:10CA10000F947D0A85E20E948FC4E7CE2A960FB656
:10CA2000F894DEBF0FBECDBFDF91CF911F910F9164
:10CA3000FF90BF90AF909F908F907F906F905F908E
:10CA40004F90089540E050E0BA0182E290E6D7CAE4
:10CA5000E091AE04EE2381F0E150E093AE0486E075
:10CA6000E89FF0011124E657FB4F42815381648116
:10CA7000758180819181C3CAE5CFAF92BF92CF9279
:10CA8000DF92EF92FF920F931F93CF93DF935C019E
:10CA90007B0120E030E0F501E20FF31FE491EE238B
:10CAA00019F02F5F3F4FF7CFF701CF018E199F0984
:10CAB00041914111FACF04E110E0081B110933271D
:10CAC000021713071CF0DD24D39402C082E0D82E95
:10CAD0008091C70990E06D2D70E06F5F7F4F0F94DC
:10CAE000B721C62EC6E0C60F8091FA09C81750F0CC
:10CAF0008091FC0990E02C2F30E02B5031098217F7
:10CB000093079CF5D0E0E114F104C1F18AE30E949F
:10CB10008FC482E0D8120FC0CC0D8091FA09C817DB
:10CB200068F12091FC0930E08C2F90E00B972817DA
:10CB300039071CF423C0DD2309F1802F880F080F6B
:10CB4000000F0093FD09C093FE0980E20E948FC48C
:10CB5000C701DF91CF911F910F91FF90EF90DF9070
:10CB6000CF90BF90AF900D947D0A1092FD09C093B5
:10CB7000FE09C5010F94700AD1E0C5CFDF91CF91B6
:10CB80001F910F91FF90EF90DF90CF90BF90AF90EB
:10CB900008950F934CE0849F402D112421E0240F31
:10CBA000209337138CE0840F80933813E091FA09B7
:10CBB000F0E090E002968E179F070CF1822F90E034
:10CBC0002091FC0930E082179307CCF4662371F0C2
:10CBD00081E08093E6094D5F0BE020E860E086ECA1
:10CBE00099E00E947FBE1092E60903C081E0809325
:10CBF000E609809138131092FD098093FE090F9188
:10CC00000895CF92DF92EF92FF920F93CF93DF932D
:10CC1000982F862F6A017901692FBBDF9091FA095D
:10CC200080913813891708F453C09091FC098091C2
:10CC30003713981708F44CC0002359F060E070E0F7
:10CC4000F701E60FF71FE491EE2351F06F5F7F4F7E
:10CC5000F7CFD701BD016E197F098D918111FACFF0
:10CC6000C62FD4E1D61BF6018491882339F00F94A6
:10CC7000450AD81BFFEFCF1ADF0AF5CF8AE30E94DF
:10CC80008FC4DD2329F080E20E948FC4D150F9CFF8
:10CC9000809138136AEFC69F602D1124605860930D
:10CCA000FD098093FE09C701002349F0DF91CF9170
:10CCB0000F91FF90EF90DF90CF900D94700ADF916D
:10CCC000CF910F91FF90EF90DF90CF900D947D0A60
:10CCD000DF91CF910F91FF90EF90DF90CF9008956B
:10CCE0000F93CF93DF93CDB7DEB7ED85FE856081DF
:10CCF0007181828193810F941F20CB010E94ADD15D
:10CD000000E09C0149855A8568858F817ADFDF9133
:10CD1000CF910F9108959CE0899F802D112421E0EF
:10CD2000280F20933713845F809338136091FA099A
:10CD300070E0482F50E04E5F5F4F46175707CCF129
:10CD400030E04091FC0950E02417350794F59EE34C
:10CD50009093FD098093FE0985E40F945C0A80910D
:10CD600039138F5C0F945C0A80E20F945C0A609127
:10CD7000AC127091AD128091AE129091AF120F94DF
:10CD80001F20CB010E94ADD10F947D0A8FE20F943A
:10CD90005C0A0E94C0FF811104C08091BE0981110C
:10CDA00008C080915104909152040E94ADD10D941D
:10CDB0007D0A08958F929F92AF92BF92CF92DF9299
:10CDC000EF92FF92CF93C82F8090000290900102C3
:10CDD000A0900202B0900302A5019401C501B40124
:10CDE0000F948721C090F706D090F806E090F906DE
:10CDF000F090FA0681112AC0C11128C08091BF129B
:10CE0000882321F1A5019401C701B6010F94DA1E10
:10CE10002091230730912407409125075091260740
:10CE20000F94071B0F940C2188279927861B970BBB
:10CE30002091CE04222351F06091B7127091B81264
:10CE4000860F971F9093B8128093B712C09200027A
:10CE5000D0920102E0920202F0920302CF91FF9081
:10CE6000EF90DF90CF90BF90AF909F908F900895FC
:10CE700088E893E190939A128093991280916F00C1
:10CE80008D7F80936F009091480A8091490A98178E
:10CE900019F00E94ABDDF7CF1092620D1092610D78
:10CEA00080916F00826080936F008FB7F89410922A
:10CEB00000131092011310920213109203138FBFEC
:10CEC0000E94BEF80F948E0D8AEE96E00E940D87A8
:10CED0000E9467CB0C9438B82F923F924F925F928A
:10CEE0006F927F928F929F92AF92BF92CF92DF927A
:10CEF000EF92FF920F931F93CF93DF93CDB7DEB7DF
:10CF0000C254D1090FB6F894DEBF0FBECDBF85E481
:10CF10000E94BAB9882321F00E9428B98B0102C06F
:10CF200000E010E083E40E94BAB9882329F00E944F
:10CF300028B97AA769A704C025E030E03AA729A755
:10CF400085E50E948BB98F8F882319F00E9449B91B
:10CF50008F8F17FD07C0C12CD12C86E1E82E83E40A
:10CF6000F82E06C0C12CD12CBCE8EB2EB2E4FB2E6F
:10CF700083E50E94BAB9882321F00E9458B96B0159
:10CF80007C010115110511F410922C040E94ACC112
:10CF90002B013C01C8010196029728F4ABE0AA2EB0
:10CFA000A3E0BA2E26C00EE113E0D8018D918D01C9
:10CFB000882319F00F940214F8CF8AE0CE5BDF4F7C
:10CFC0000FB6F894DEBF0FBECDBFDF91CF911F919A
:10CFD0000F91FF90EF90DF90CF90BF90AF909F9018
:10CFE0008F907F906F905F904F903F902F900D9417
:10CFF0000214F50181915F01882319F00F94021446
:10D00000F8CF8AE00F9402140E94429C0F3FFFEF7A
:10D010001F0761F487E68093B80627E630E040E01A
:10D0200050E029833A834B835C830BC08FE7809366
:10D03000BA068FE790E0A0E0B0E089839A83AB83E3
:10D04000BC83C701B6010F941F20072E000C880B6C
:10D05000990B0F94A81A6B8B7C8B8D8B9E8B81E028
:10D0600080939E020F3F9FEF190729F48EEC90E00A
:10D07000A0E0B0E004C08FEF90E0A0E0B0E09C0141
:10D08000AD0123513109410951092FA738AB49ABF3
:10D090005AAB9C01AD0124513109410951092BAB17
:10D0A0003CAB4DAB5EAB9C01AD01559547953795BB
:10D0B00027952FAB38AF49AF5AAF9C01AD01215036
:10D0C0003109410951092BAF3CAF4DAF5EAF8980AB
:10D0D0009A80AB80BC8049A25AA26BA27CA24BA6CC
:10D0E0005CA66DA67EA61F8A30E4388F4CE1498F7E
:10D0F00056E45A8F1B8E1C8E1D8E1E8E1F86188A1C
:10D10000198A1A8A1B861C861D861E86C12CD12C64
:10D1100076011DA21EA21FA218A681E088A31A866E
:10D120001986212C312C22961FAE229723961FAEF2
:10D13000239780919E02882309F4EEC10E94ACC11E
:10D140006D837E838F8398878091A806882309F456
:10D15000C2C00E94069D0F3F9FEF190779F42090EF
:10D16000AF043090B004A091B1042296AFAF2297E3
:10D17000B091B2042396BFAF23970EC02090AC129B
:10D180003090AD12E091AE122296EFAF2297F0915F
:10D19000AF122396FFAF2397910122964FAD2297AE
:10D1A00023965FAD23976B8D7C8D8D8D9E8D0F9417
:10D1B000A21A87FF0AC02B8E3C8E22962FAD229793
:10D1C0002D8F23963FAD23973E8F910122964FAD31
:10D1D000229723965FAD23976F89788D898D9A8DDD
:10D1E0000F940121181654F42F8A388E22964FADD1
:10D1F0002297498F23965FAD23975A8F88A12B8959
:10D200003C894D895E89B101882309F446C0229684
:10D210008FAD229723969FAD23970F940121181667
:10D220000CF059C04D815E816F8178854419550994
:10D2300066097709DB01CA0188589341A109B10940
:10D24000B7FD49C089819A81AB81BC818819990950
:10D25000AA09BB09B595A795979587950F3FEFEF5D
:10D260001E0719F48093B80602C08093BA064DA336
:10D270005EA36FA378A7FB89FB8F2C892C8F3D8938
:10D280003D8F4E894E8F8D819E81AF81B88589A358
:10D290009AA3ABA3BCA318A21EC022968FAD22975F
:10D2A00023969FAD23970F94A21A87FF14C08D81F8
:10D2B0009E81AF81B88529A13AA14BA15CA1821BB7
:10D2C000930BA40BB50BAC01BD0148585341610948
:10D2D000710977FF40C120E030E040EA51E46B89FA
:10D2E0007C898D899E890F94DB1E9B01AC01B10165
:10D2F00022968FAD229723969FAD23970F940121FD
:10D3000018166CF4E5E5FAE184918F010F5F1F4F69
:10D31000882309F480C20F940214F801F5CF80E34A
:10D3200098EFAFEFBFEF2BA53CA54DA55EA5821BE7
:10D33000930BA40BB50B2D813E814F815885820F35
:10D34000931FA41FB51FB7FD0DC00F94F5118AE000
:10D350000F9402148D819E81AF81B8858BA79CA705
:10D36000ADA7BEA78D819E81AF81B885880F991F1B
:10D37000AA1FBB1F29A13AA14BA15CA1821B930B41
:10D38000A40BB50B84199509A609B70981389F44E8
:10D39000A241B10568F0E7E3FAE184918F010F5FE4
:10D3A0001F4F882309F437C20F940214F801F5CFF8
:10D3B00049855A8589A59AA5841795070CF0A9C0B7
:10D3C000EAEDF9E184915F019FEFA91AB90A882378
:10D3D00021F00F940214F501F5CF0F3FAFEF1A07BC
:10D3E00029F02BEBA22E23E0B22E04C097E0A92E49
:10D3F00093E0B92EB50188EC99E10E94D977B70185
:10D40000A60184EC99E10E9457728AE00F940214FD
:10D41000B50182EB99E10E94D9774B855C856D85DA
:10D420007E858EEA99E10E9457728AE00F94021479
:10D43000B5018CE999E10E94D9774F8558896989AE
:10D440007A8988E999E10E9457728AE00F94021460
:10D45000BF8DBB2309F4DFC10F3F1F4F69F5C09299
:10D46000C506D092C606E092C706F092C8062CEA1E
:10D4700035EC47E25EE36B857C858D859E850F9458
:10D48000071B6093C1067093C2068093C3069093F6
:10D49000C4062CEA35EC47E25EE36F85788989891A
:10D4A0009A890F94B71F6093BD067093BE06809350
:10D4B000BF069093C006AFC1C092D106D092D206EB
:10D4C000E092D306F092D4062CEA35EC47E25EE314
:10D4D0006B857C858D859E850F94071B6093CD069B
:10D4E0007093CE068093CF069093D0062CEA35EC4D
:10D4F00047E25EE36F85788989899A890F94B71F1F
:10D500006093C9067093CA068093CB069093CC06AD
:10D5100082C10E94A3FC0DCE80919E0281117BC12D
:10D52000CE5BDF4F0FB6F894DEBF0FBECDBFDF91ED
:10D53000CF911F910F91FF90EF90DF90CF90BF9010
:10D54000AF909F908F907F906F905F904F903F90A3
:10D550002F900C94429C49855A85141615060CF0A0
:10D560001DC14DA05EA06FA078A4480E591E6A1E72
:10D570007B1E2DA13EA14FA158A5281B390B4A0B9C
:10D580005B0BCA01B901A50194010F946E1EA301A2
:10D5900092010F949F1E89809A80AB80BC80820E7E
:10D5A000931EA41EB51E34E183169104A104B10498
:10D5B0000CF41EC18FA598A9A9A9BAA98816990625
:10D5C000AA06BB060CF022C12FA938AD49AD5AAD51
:10D5D000281539054A055B057CF489829A82AB825D
:10D5E000BC828BAD9CADADADBEAD88199909AA09C1
:10D5F000BB094C015D0104C089829A82AB82BC8266
:10D60000E1ECFAE184919F012F5F3F4F882361F0A5
:10D610002FAF21963FAF21970F9402142FAD219683
:10D620003FAD2197F901EECF69817A818B819C8191
:10D630000F94C114ECEBFAE184919F012F5F3F4FEF
:10D64000882361F02FAF21963FAF21970F940214EA
:10D650002FAD21963FAD2197F901EECFC501B40161
:10D660000F94C1144F89588D698D7A8D85EB9AE19D
:10D670001ED74B8D5C8D6D8D7E8D8EEA9AE117D70E
:10D68000A985BA8513970CF489C0C501B4010F941C
:10D69000A81A20E030E040E850E40F94071B6B012B
:10D6A0007C012F89388D498D5A8D6B8D7C8D8D8DA8
:10D6B0009E8D0F94DA1E2BED3FE049E450E40F9469
:10D6C000071B20E030E040E05FE30F94071B9B0165
:10D6D000AC01C701B6010F94B71F6B017C01C301F8
:10D6E000B2010F94A81A2FE632E143E85AE30F94EF
:10D6F000071B2B013C01B701A60188EA9AE1D7D6A6
:10D70000B301A20182EA9AE1D2D62AE939E949E1D4
:10D710005FE3C701B6010F94071B6B017C019B01FE
:10D72000AC010F94DB1EA30192010F94B71F6B870E
:10D730007C878D879E87A3019201C701B6010F9454
:10D74000071B20E030E040E05EE30F94071B6F878B
:10D75000788B898B9A8BE2E9FAE184913F01BFEFE4
:10D760006B1A7B0A882321F00F940214F301F5CF82
:10D77000B701A6018CE89AE19AD64B855C856D8548
:10D780007E8586E89AE193D64F85588969897A899A
:10D7900080E89AE18CD68AE00F94021489819A81FC
:10D7A000AB81BC81880D991DAA1DBB1DB595A795A0
:10D7B000979587950F3FEFEF1E0719F48093B806F2
:10D7C00002C08093BA0629853A852F5F3F4F3A877A
:10D7D00029873B893F8B4C89488F5D89598F8E897A
:10D7E0008A8F4D805E806F80788491E098A373CD9E
:10D7F00084E1882E912CA12CB12C24E130E040E072
:10D8000050E029833A834B835C83FACE8BA89CA893
:10D81000ADA8BEA8E2CECE5BDF4F0FB6F894DEBF58
:10D820000FBECDBFDF91CF911F910F91FF90EF9071
:10D83000DF90CF90BF90AF909F908F907F906F9030
:10D840005F904F903F902F900895CF93DF9383E5A3
:10D850000E948BB9C82F882371F00E9458B90F9489
:10D860001F2070936A026093690221E0672B09F020
:10D8700020E02093B01280E50E948BB9882359F0F4
:10D880002091690230916A02232B11F00E9449B95C
:10D890008093B0122CC0C1112AC0E7E4F6E2849153
:10D8A000EF012196882321F00F940214FE01F7CF97
:10D8B0008091B012811103C067E473E002C06BE98C
:10D8C00073E085E899E10E94D977609169027091CF
:10D8D0006A0284E799E108D6E0E7F9E18491EF0173
:10D8E0002196882321F00F940214FE01F7CFDF91D7
:10D8F000CF910895CF93DF9380E50E948BB9882361
:10D9000051F00E9458B96093C5067093C606809383
:10D91000C7069093C80689E40E948BB9882381F0DA
:10D920000E9458B92CEA35EC47E25EE30F94071BDE
:10D930006093C1067093C2068093C3069093C40699
:10D9400084E40E948BB9882381F00E9458B92CEAA4
:10D9500035EC47E25EE30F94B71F6093BD0670930A
:10D96000BE068093BF069093C006E7E4F6E284917A
:10D97000EF012196882321F00F940214FE01F7CFC6
:10D980004091C5065091C6066091C7067091C806C1
:10D990008CE699E18CD52CEA35EC47E25EE36091A8
:10D9A000C1067091C2068091C3069091C4060F947F
:10D9B000B71FAB01BC0188E699E15CD52CEA35ECD8
:10D9C00047E25EE36091BD067091BE068091BF069E
:10D9D0009091C0060F94071BAB01BC0184E699E14E
:10D9E00049D58AE0DF91CF910D940214CF93DF9354
:10D9F00085E40E94BAB9811110C080E50E948BB9FC
:10DA0000882391F00E9458B96093D1067093D20692
:10DA10008093D3069093D40607C00E9438B9882318
:10DA200061F3E8E8F4E26AC089E40E948BB98823D4
:10DA300081F00E9458B92CEA35EC47E25EE30F947E
:10DA4000071B6093CD067093CE068093CF0690930C
:10DA5000D00684E40E948BB9882381F00E9458B9D3
:10DA60002CEA35EC47E25EE30F94B71F6093C906DA
:10DA70007093CA068093CB069093CC06E7E4F6E257
:10DA80008491EF012196882321F00F940214FE0166
:10DA9000F7CF4091D1065091D2066091D306709194
:10DAA000D40680E699E103D52CEA35EC47E25EE343
:10DAB0006091CD067091CE068091CF069091D006F0
:10DAC0000F94B71FAB01BC018CE599E1D3D42CEACC
:10DAD00035EC47E25EE36091C9067091CA06809119
:10DAE000CB069091CC060F94071BAB01BC0188E5D7
:10DAF00099E1C0D410C00F940214FE018491EF018B
:10DB000021968111F8CFC2EFD2E08991882319F0D4
:10DB10000F940214FACF8AE0DF91CF910D94021492
:10DB2000CF93DF9300D01F92CDB7DEB783E50E947D
:10DB3000BAB9882319F00E9428B902C064E071E0E4
:10DB40007C836B8380E50E94BAB9882339F00E94F8
:10DB500028B9693883E1780730F402C068EE73E0D1
:10DB60007A83698304C088E893E19A838983BE013C
:10DB70006D5F7F4FCE0101960E944BAF0F900F90CB
:10DB80000F900F90DF91CF910895CF92DF92EF9297
:10DB9000FF92CF93DF9380E50E948BB98823C9F170
:10DBA0000E9428B96B017C0183E50E94BAB98823E1
:10DBB00021F00E9428B9EB0102C0CFEFDFEF9E01F8
:10DBC0002F5F3F4F2330310520F5D7FC22C00E9444
:10DBD000BEF8CF3F8FEFD80729F0219771F4C1E04D
:10DBE000D0E00DC08C2D0E9457C031E020E0892B81
:10DBF00009F030E0C32FD22F02C0C0E0D0E08C2D5E
:10DC00000E9457C08C179D0721F080E00F94360BBF
:10DC1000F6CFDF91CF91FF90EF90DF90CF900895F6
:10DC2000CF93DF938DED90E00E9435BA811110C043
:10DC300083E50E94BAB9882359F0C0912C04D0E042
:10DC40000E9428B9CC0FDD1FC359DD4F798368834B
:10DC5000DF91CF910895CF93DF93E7E4F6E28491CB
:10DC6000EF012196882321F00F940214FE01F7CFD3
:10DC700083E50E948BB9882321F00E9449B98093E3
:10DC80008602E8E4F9E18491EF012196882321F0EE
:10DC90000F940214FE01F7CF80918602811103C018
:10DCA000E4E4F9E102C0E0E4F9E18491EF012196B6
:10DCB000882321F00F940214FE01F7CFE8E3F9E185
:10DCC0008491EF012196882321F00F940214FE0124
:10DCD000F7CF40912F04509130046091310470913E
:10DCE000320486E399E1E3D3409133045091340444
:10DCF000609135047091360483E399E1D8D3409163
:10DD00003704509138046091390470913A0480E3EB
:10DD100099E1CDD3E8E2F9E18491EF0121968823DE
:10DD200021F00F940214FE01F7CF4091710250913F
:10DD30007202609173027091740286E299E1B7D326
:10DD4000409175025091760260917702709178024D
:10DD500083E299E1ACD34091790250917A026091CB
:10DD60007B0270917C0280E299E1A1D38AE0DF918D
:10DD7000CF910D94021483E50E948BB9882351F052
:10DD80000E9458B9609358047093590480935A04C0
:10DD900090935B0484E50E948BB9882351F00E9424
:10DDA00058B960935404709355048093560490932B
:10DDB000570482E40E948BB9882351F00E9418B95D
:10DDC0006093E1067093E2068093E3069093E40685
:10DDD00088E50E948BB9882351F00E9458B960935E
:10DDE000630D7093640D8093650D9093660D89E5C6
:10DDF0000E948BB9882351F00E9458B96093670D37
:10DE00007093680D8093690D90936A0D8AE50E9466
:10DE10008BB9882351F00E9458B960936B0D7093B1
:10DE20006C0D80936D0D90936E0D85E40E948BB9FF
:10DE3000882351F00E9458B960936F0D7093700D54
:10DE40008093710D9093720D089583E50E948BB9B4
:10DE50008823D1F00E9458B9AB01BC0140938504DE
:10DE600050938604609387047093880440937D04E4
:10DE700050937E0460937F047093800488EF98E150
:10DE800016D38AE00F94021480E50E948BB9882390
:10DE900091F00E9458B9AB01BC01409385045093A6
:10DEA000860460938704709388048BED98E1FFD219
:10DEB0008AE00F94021482E50E948BB9882391F0C6
:10DEC0000E9458B9AB01BC01409381045093820475
:10DED00060938304709384048CEB98E1E8D28AE029
:10DEE0000F94021484E50E948BB9882391F00E945C
:10DEF00058B9AB01BC0140937D0450937E046093FC
:10DF00007F04709380048EE998E1D1D28AE00D9469
:10DF100002140895FF920F931F93CF93DF930CE5A4
:10DF200014E0C3E0D3E0FC2E84E0F80E89910E9457
:10DF30008BB9882339F00E9458B9F8016083718346
:10DF4000828393830C5F1F4FFC12F0CFDF91CF9140
:10DF50001F910F91FF900895FF920F931F93CF93FE
:10DF6000DF930DE614E0C3E0D3E0FC2E84E0F80E6E
:10DF700089910E948BB9882349F00E9458B90F9467
:10DF80002420F80160837183828393830C5F1F4F89
:10DF9000FC12EECFDF91CF911F910F91FF900C9467
:10DFA00083E4CF93DF9388EC90E00E9435BA81112F
:10DFB00042C084E40E948BB98823C9F10E9458B9F9
:10DFC000C1E020E030E0A9010F94A21A811101C044
:10DFD000C0E0C093E906CC2351F1C0912C04D0E0FD
:10DFE0000E9458B9CC0FDD1FCC0FDD1FCB51D94F8C
:10DFF000688379838A839B8320E030E0A901609164
:10E00000E5067091E6068091E7069091E8060F9488
:10E01000A21A81110CC080E090E0A0E4B0E48093EB
:10E02000E5069093E606A093E706B093E806DF9135
:10E03000CF910D94490DDF91CF910895CF92EF923A
:10E040000F931F93CF93DF93CDB7DEB764970FB6CF
:10E05000F894DEBF0FBECDBF8CE40E948BB988233D
:10E0600019F00E9458B904C060E070E080E090ECC4
:10E070006D877E878F87988B8AE50E94BAB988233F
:10E0800019F00E9458B903C060E070E0CB0120E0B5
:10E0900030E040E251E40F94DB1E69877A878B877A
:10E0A0009C8788E50E94BAB9882319F00E9458B964
:10E0B00003C060E070E0CB0120E030E040E251E4DA
:10E0C0000F94DB1E6D837E838F83988789E50E9482
:10E0D000BAB9882319F00E9458B903C060E070E013
:10E0E000CB0120E030E047E953E40F94DB1E20E051
:10E0F00030E040E251E40F94DA1E69837A838B8327
:10E100009C83198A1A8A1B8A1C8A8091550D811159
:10E1100012C0C12CE12C8E010F5E1F4F9E012F5F9C
:10E120003F4FAE014B5F5F4FBE01675F7F4FCE0138
:10E130000D960E94CAC864960FB6F894DEBF0FBE53
:10E14000CDBFDF91CF911F910F91EF90CF900895A8
:10E150004F925F926F927F928F929F92AF92BF92F7
:10E16000CF92DF92EF92FF92CF93DF93EBE9F8E14A
:10E170008491EF012196882321F00F940214FE016F
:10E18000F7CF60910B0770910C0780910D0790916C
:10E190000E0742E00F94DB14E7E9F8E18491EF0108
:10E1A0002196882321F00F940214FE01F7CF60918D
:10E1B0000F0770911007809111079091120742E0AC
:10E1C0000F94DB14E3E9F8E18491EF0121968823B1
:10E1D00021F00F940214FE01F7CF609113077091A4
:10E1E0001407809115079091160742E00F94DB14F5
:10E1F000EFE8F8E18491EF012196882321F00F9454
:10E200000214FE01F7CF60911707709118078091F3
:10E21000190790911A0742E00F94DB148FB7F89416
:10E220004090FB065090FC066090FD067090FE0644
:10E230008090FF0690900007A0900107B090020721
:10E24000C0900307D0900407E0900507F090060700
:10E250008FBFE5E8F8E18491EF012196882321F052
:10E260000F940214FE01F7CFC301B2010F94C11441
:10E27000E1E8F8E18491EF012196882321F00F94E1
:10E280000214FE01F7CFC501B4010F94C114EDE7EC
:10E29000F8E18491EF012196882321F00F94021474
:10E2A000FE01F7CFC701B6010F94C1148AE0DF91D8
:10E2B000CF91FF90EF90DF90CF90BF90AF909F9065
:10E2C0008F907F906F905F904F900D9402144F92BB
:10E2D0005F926F927F92AF92BF92CF92DF92EF9256
:10E2E000FF920F931F93CF9383E0A82E83E0B82E65
:10E2F0000BE117E0C0E0F50181915F010E948BB94D
:10E30000882309F46DC0C33009F063C00E9458B976
:10E310006B017C0120E030E040EA51E40F94A21A46
:10E3200087FF4EC0A70196016091270770912807CB
:10E330008091290790912A070F94B71F2B013C0168
:10E340009B01AC0160916F0D7091700D8091710D0A
:10E350009091720D0F94071B60936F0D7093700D69
:10E360008093710D9093720DA301920160916804E6
:10E370007091690480916A0490916B040F94071B5B
:10E38000609368047093690480936A0490936B04AB
:10E390006091870D7091880D8091890D90918A0D03
:10E3A0000F94A61AA30192010F94071B0F94242027
:10E3B0006093870D7093880D8093890D90938A0DDB
:10E3C000C0922707D0922807E0922907F0922A07E7
:10E3D00007C00E9458B9F8016083718382839383D8
:10E3E000CF5F0C5F1F4FC43009F085CFCF911F91D5
:10E3F0000F91FF90EF90DF90CF90BF90AF907F9004
:10E400006F905F904F900C94B0E583E50E948BB9BC
:10E41000882391F00E9458B920E030E04AE754E4A4
:10E420000F94071B0F942420609377147093781433
:10E430008093791490937A140895CF92DF92EF929B
:10E44000FF92CF93DF936A017B01FC018491EF017E
:10E450002196882321F00F940214FE01F7CF4AE0A1
:10E46000C701B601DF91CF91FF90EF90DF90CF9081
:10E470000D945B14CF92DF92EF92FF92CF93DF93D4
:10E480006A017B01FC018491EF012196882321F030
:10E490000F940214FE01F7CF42E0C701B601DF91ED
:10E4A000CF91FF90EF90DF90CF900D94DB14CF923F
:10E4B000DF92EF92FF92CF93DF936A017B01FC0121
:10E4C0008491EF012196882321F00F940214FE011C
:10E4D000F7CF42E0C701B601DF91CF91FF90EF90F7
:10E4E000DF90CF900D94DB140F931F93CF93DF93A6
:10E4F0008B01FC018491EF012196882321F00F9478
:10E500000214FE01F7CFB801110F880B990BDF91B0
:10E51000CF911F910F910D94C114CF93DF931F9250
:10E520001F92CDB7DEB7789484B5826084BD84B580
:10E53000816084BD85B5826085BD85B5816085BDFE
:10E5400080916E00816080936E00109281008091B6
:10E55000810082608093810080918100816080933E
:10E560008100809180008160809380008091B10063
:10E5700084608093B1008091B00081608093B0008E
:10E5800080919100826080939100809191008160E0
:10E5900080939100809190008160809390008091A1
:10E5A000A10082608093A1008091A100816080938E
:10E5B000A1008091A00081608093A0008091210142
:10E5C00082608093210180912101816080932101EB
:10E5D0008091200181608093200180917A00846085
:10E5E00080937A0080917A00826080937A00809193
:10E5F0007A00816080937A0080917A0080688093AD
:10E600007A001092C1006F98779A82E08093C000E0
:10E610001092C50087E08093C4008091C1008061A2
:10E620008093C1008091C10088608093C100809177
:10E63000C10080688093C1008091C1008F7D80936C
:10E64000C1001092C404E4E4FCE184918F010F5FE7
:10E650001F4F882321F00F940214F801F6CFE7E44E
:10E66000F6E284918F010F5F1F4F882321F00F94F2
:10E670000214F801F6CF14B710FF0DC0EBE3FCE174
:10E6800084917F019FEFE91AF90A882321F00F9402
:10E690000214F701F5CF11FF0DC0EAE2FCE184910D
:10E6A0007F019FEFE91AF90A882321F00F940214E1
:10E6B000F701F5CF12FF0DC0E8E1FCE184917F0185
:10E6C0009FEFE91AF90A882321F00F940214F70149
:10E6D000F5CF13FF0DC0E7E0FCE184917F019FEFD0
:10E6E000E91AF90A882321F00F940214F701F5CFF3
:10E6F00015FF0CC0E6EFFBE184918F010F5F1F4F08
:10E70000882321F00F940214F801F6CF14BEEFEE27
:10E71000FBE184918F010F5F1F4F882321F00F943D
:10E720000214F801F6CF80E20F940214E8EEFBE148
:10E7300084918F010F5F1F4F882321F00F940214E3
:10E74000F801F6CF8AE00F940214E7E4F6E2849130
:10E750008F010F5F1F4F882321F00F940214F801DF
:10E76000F6CFE8EDFBE184918F010F5F1F4F882307
:10E7700021F00F940214F801F6CFE4ECFBE1849150
:10E780008F010F5F1F4F882321F00F940214F801AF
:10E79000F6CFEBE8FBE184918F010F5F1F4F8823D9
:10E7A00021F00F940214F801F6CFE7E4F6E2849129
:10E7B0008F010F5F1F4F882321F00F940214F8017F
:10E7C000F6CFE4E7FBE184918F010F5F1F4F8823B1
:10E7D00021F00F940214F801F6CFE7E4F6E28491F9
:10E7E0008F010F5F1F4F882321F00F940214F8014F
:10E7F000F6CF8091281590912915BE016F5F7F4F4C
:10E80000009719F0681B790B02C06E52754185E6BE
:10E810009BE16ADE60EF74E08EE49BE165DE8AE0F6
:10E820000F94021481E08093DE048093DF048093D0
:10E83000E0048093E1040E9439A48CE0E2EDF4E06E
:10E84000ABE0B7E001900D928A95E1F70E9438B8ED
:10E8500080910101806480930101809101018061B8
:10E8600080930101809101018860809301016D9A7C
:10E870008091010180628093010188E00E948CB147
:10E880008091010188608093010186E00E948CB133
:10E890006C9A82E00E948CB187ED80937A0010928E
:10E8A0007E0010927D0080917E00816080937E00CA
:10E8B00080917E00846080937E0080E888BD809196
:10E8C0006E00846080936E006AEF70E080E090E0FC
:10E8D0000E9474C185E090E09093CA048093C904BB
:10E8E00060E080910602909107020E94729920E0F8
:10E8F00030E040EA50E40F94A21A87FF0AC08091EA
:10E9000006029091070240979093070280930602B7
:10E91000E7CF81E391E0909309028093080260E0E1
:10E920008091C7049091C8040E94729920E030E859
:10E9300048E953E40F940121181654F48091C70458
:10E940009091C80440969093C8048093C704E7CF81
:10E9500080910402909105020E94679C20E030E0C3
:10E9600040EA50E40F94A21A87FF0AC08091040283
:10E970009091050240979093050280930402E8CF9E
:10E980008091C5049091C6040E94679C20E030E00D
:10E9900046E153E40F940121181654F48091C50404
:10E9A0009091C60440969093C6048093C504E8CF26
:10E9B00098E288E10FB6F894A895809360000FBEA6
:10E9C000909360001FB7F8948091CB04811124C00C
:10E9D000E0E0F7E28491E6E4F7E29491E82FF0E0DA
:10E9E000EE0FFF1FEF54F94DA591B491EC91E9237F
:10E9F00021F461E085E30E947FC085E30E943CC36F
:10EA00008CB580618CBD8CB580648CBD84E30E9424
:10EA10003CC383E30E943CC38091CB048F5F80930F
:10EA2000CB041FBF579AB5E6EB2EB3E0FB2E10E0E8
:10EA3000F70161917F0170E0812F0E9431F81F5F23
:10EA40001530B1F7999A989A809107018068809360
:10EA500007019A9A80910701806480930701809151
:10EA6000070180628093070180910701886080938D
:10EA70000701809107018061809307018091070160
:10EA80008260809307018091070184608093070171
:10EA9000AAE6EA2EA3E0FA2E10E0F70161917F01C9
:10EAA000812F0E940BF81F5F1530B9F780910A0182
:10EAB000826080930A0180910A01816080930A013B
:10EAC00080910A01846080930A0180910A01806428
:10EAD00080930A0180910A01806880930A010F9A4D
:10EAE000179A0E9A169A0D9A159A0C9A149A0B9ACE
:10EAF000139A26982E9A25982D9A24982C9A0A983B
:10EB0000129A0998119A3F98479A0898109A389A39
:10EB10004098179A1092CC04399A4198169A1092FC
:10EB2000CD043A9A4298159A1092CE043B9A439893
:10EB3000149A3C9A4498809180008C7F8093800046
:10EB400080918100877E8860809381008091800021
:10EB50008F738093800080918100887F8260809392
:10EB6000810080E090E49093890080938800109267
:10EB700085001092840080916F00826080936F0006
:10EB800081E08093D00478940E944ADD1092D104F1
:10EB90006C9A0E94F8FF64EC79E080E090E00E94BB
:10EBA000E3D180910A02811118C064EC79E080E021
:10EBB00090E00E94E3D181E08093D0048093CF0461
:10EBC00060E6862E7DE0772EE2E6CE2EECE1DE2EAC
:10EBD000F0E0AF2EF0E0BF2EB0C010920A022091FC
:10EBE000C60930E07901F8E3EF1AF108F7FE04C036
:10EBF000790187E3E81AF108F594E7942E51310979
:10EC000036952795F22E0E9475C509EC1AE123E18D
:10EC100047E06CE08E2D0E9493C384E00F942B0A92
:10EC20000091C60910E002571109169507956091E9
:10EC3000C70962514BE453E08F2D0E940EC46091CE
:10EC4000C709665041E553E0802F0E940EC40E9420
:10EC50005BC38111DACFA9CF8091F60680FD57C141
:10EC60008091F60684FD53C190E2F92E8091F6065C
:10EC700081FD69C18091F60685FD65C100E2809144
:10EC8000F60682FD7BC18091F60686FD77C110E213
:10EC90008091F60683FF36C16091FB047091FC04FD
:10ECA0008091FD049091FE040F94A81A2091EB042A
:10ECB0003091EC044091ED045091EE040F94071B49
:10ECC000AB01BC0187E79CE1F2DB90E58AE09A8327
:10ECD0000F9402141F929A819F931F921F931F9269
:10ECE0000F931F92FF92DF92CF921F920E9437C51F
:10ECF0001092F6060FB6F894DEBF0FBECDBF80911E
:10ED0000E204882391F01092770A89E69CE00E9441
:10ED1000418D89E69CE00E94728D1092760A1092D5
:10ED2000750A0E9438670E94429C80E00F94360B5F
:10ED3000A114B10421F00E9400002AE0922E8091DB
:10ED40008006843010F40E94B4B58091220D88238F
:10ED5000F1F00E94ACC100911E0D10911F0D209189
:10ED6000200D3091210DDC01CB01801B910BA20BFA
:10ED7000B30BB7FD0CC01092220D8091780A81115F
:10ED8000C3C00E9404AE8091780A8111BDC08091F9
:10ED90008006882309F498C08091750A882309F4B5
:10EDA00080C000917F06809E8001112401501B4F7E
:10EDB00069EA7CE1C8010F94211A892BF9F089E6F0
:10EDC0009CE00E94418D89E69CE00E94728D109229
:10EDD000760A1092750AE6E9FCE184918F010F5FD3
:10EDE0001F4F882341F00F940214F801F6CF809151
:10EDF000760A811156C00F94FF0D55C0F80101909D
:10EE00000020E9F731977F01E01AF10A1092690CAE
:10EE10006EE470E0C8010F940E222C01009729F4D3
:10EE2000F7013197E00FF11F0EC060E270E00F9420
:10EE30000E228C010F5F1F4F6AE270E0C2010F9437
:10EE40000E22FC013197718292821382F8010190A7
:10EE50000020E9F73197AF01401B510BB80189E65B
:10EE60009CE00E94358E8091690C882309F4BFCF05
:10EE7000E8E8F4E284918F010F5F1F4F882321F0AF
:10EE80000F940214F801F6CFEBE4FCE184918F01BA
:10EE90000F5F1F4F882309F4AACF0F940214F801C3
:10EEA000F5CF0E942D2B80918006882369F0815038
:10EEB0008093800680917F068F5F843018F4809362
:10EEC0007F0602C010927F068091F606882309F41F
:10EED0002CCFE7E4F6E284918F010F5F1F4F882368
:10EEE00021F00F940214F801F6CFE7E8FCE18491D9
:10EEF0008F010F5F1F4F882309F4AECE0F940214C9
:10EF0000F801F5CF90E2E2CE0E9453AD40CF609180
:10EF1000F3047091F4048091F5049091F6040F9439
:10EF2000A81A2091E3043091E4044091E504509143
:10EF3000E6040F94071BAB01BC0183E89CE1B7DA40
:10EF400088E5F82E93CE6091F7047091F8048091D3
:10EF5000F9049091FA040F94A81A2091E7043091D3
:10EF6000E8044091E9045091EA040F94071BAB01B7
:10EF7000BC018FE79CE19BDA09E581CE6091FB043F
:10EF80007091FC048091FD049091FE040F94A81AE6
:10EF90002091EB043091EC044091ED045091EE048B
:10EFA0000F94071BAB01BC018BE79CE180DA1AE5EB
:10EFB0006FCE0F931F93CF93DF931F921F92CDB706
:10EFC000DEB7FC0184918F010F5F1F4F811102C0DA
:10EFD0008B0108C069837A830F940214F801698158
:10EFE0007A81F0CFF80181918F01882319F00F9475
:10EFF0000214F8CF0F900F90DF91CF911F910F91D6
:10F0000008954F925F926F927F92AF92BF92CF928C
:10F01000DF92EF92FF920F931F93CF93DF930097AE
:10F0200009F456C0FC01208121FD52C0EB018C0186
:10F0300047A050A461A472A4AFA0B8A4C9A4DAA444
:10F040009501A601C301B2010F94A21A87FF40C027
:10F05000A3019201C301B2010F94071B2B013C01D4
:10F06000F80183A994A9A5A9B6A9BC01CD0190581E
:10F070009B01AC010F94DB1EF80127A530A941A923
:10F0800052A90F94071B9B01AC01C301B2010F945D
:10F09000DA1E0F9446217B018C019B01AC01B50166
:10F0A000C6010F94A21A87FF02C07501860197015D
:10F0B000A801B501C6010F94A21A882349F0A7013F
:10F0C000B8014FA358A769A77AA788818160888370
:10F0D000DF91CF911F910F91FF90EF90DF90CF9034
:10F0E000BF90AF907F906F905F904F9008952F9258
:10F0F0003F924F925F926F927F928F929F92AF92C8
:10F10000BF92CF92DF92EF92FF920F931F93CF9314
:10F11000DF93CDB7DEB768970FB6F894DEBF0FBEAA
:10F12000CDBF1C015B018A01DC01D7966D917D91F9
:10F130008D919C91DA970F94A61A6B017C01F501D1
:10F1400020813181428153810F94071B0F94A11FAD
:10F150000F94242069877A878B879C87D8012D910B
:10F160003D914D915C91C701B6010F94071B0F941F
:10F17000A11F0F9424206D877E878F87988B298508
:10F180003A854B855C85283731054105510540F4AA
:10F1900088E790E0A0E0B0E089879A87AB87BC87DA
:10F1A0002D853E854F855889283731054105510504
:10F1B00040F488E790E0A0E0B0E08D879E87AF87BD
:10F1C000B88B91012D5B3F4FD9018D919D910D9091
:10F1D000BC91A02D8D839E83AF83B887BC01CD01E8
:10F1E0000F94A81A69837A838B839C8369857A85B7
:10F1F0008B859C850F94A61A698B7A8B8B8B9C8B45
:10F2000020E030E0A90169817A818B819C810F9493
:10F21000A21A882339F1A7019601C701B6010F94FC
:10F22000071B4B015C0129893A894B895C89CA011A
:10F23000B9010F94071B9B01AC01C501B4010F94E8
:10F24000DA1E4B015C0129813A814B815C81CA0144
:10F25000B9010F94DB1E9B01AC01C501B4010F94F1
:10F26000B71F03C060E070E0CB010F94A11F0F94A3
:10F270001F202B013C016D817E818F8198859095A7
:10F280008095709561957F4F8F4F9F4F0F94A81A6F
:10F290004B015C016D857E858F8598890F94A61A38
:10F2A0006D837E838F83988720E030E0A901C501BC
:10F2B000B4010F94A21A882349F12D813E814F8118
:10F2C0005885CA01B9010F94071B6D8B7E8B8F8BFC
:10F2D000988FA7019601C701B6010F94071B9B01E8
:10F2E000AC016D897E898F89988D0F94DA1E6B0130
:10F2F0007C01A5019401C501B4010F94DB1E9B01A3
:10F30000AC01C701B6010F94B71F03C060E070E005
:10F31000CB010F945020F10182889388A488B5888E
:10F3200075016401C418D508E608F7080F941F207A
:10F33000C61AD70AE80AF90AF7FE6BC020E030E0E7
:10F34000A90169817A818B819C810F94A21A8823FB
:10F3500009F447C029813A814B815C81CA01B90116
:10F360000F94DB1E6B017C01C501B4010F94A61A3A
:10F370009B01AC01C701B6010F94071B6B017C0117
:10F3800029893A894B895C89CA01B9010F94071B05
:10F390009B01AC01C701B6010F94DA1E6B017C0121
:10F3A0002D813E814F815885CA01B9010F94071BF9
:10F3B0009B01AC01C701B6010F94DB1E6B017C0100
:10F3C00020E030E040E850E469817A818B819C81C3
:10F3D0000F94071B9B01AC01C701B6010F94B71F27
:10F3E00003C060E070E0CB010F94A11F0F941F20B9
:10F3F0002B013C0197FF03C0412C512C32014814D2
:10F4000059046A047B0410F024013501C12CD12C6D
:10F4100076018FB7F894D1019C9193FD22C0F10140
:10F42000468A578A608E718EC40CD51CE61CF71C68
:10F430005A96CD92DD92ED92FC925D9729853A85A0
:10F440004B855C85DB962D933D934D935C93DE97C6
:10F45000FF962D853E854F855889208331834283D1
:10F4600053838FBF68960FB6F894DEBF0FBECDBF33
:10F47000DF91CF911F910F91FF90EF90DF90CF9090
:10F48000BF90AF909F908F907F906F905F904F90C4
:10F490003F902F900895CF93DF931F92CDB7DEB7A3
:10F4A000698341E050E0BE016F5F7F4F04960E9488
:10F4B000358E0F90DF91CF9108952F923F924F920A
:10F4C0005F926F927F928F929F92AF92BF92CF92F4
:10F4D000DF92EF92FF920F931F93CF93DF93CDB7FD
:10F4E000DEB7C557D1090FB6F894DEBF0FBECDBF4A
:10F4F0003B014A015901EFA6FBAA0BAF21961FAFB2
:10F5000021973C2C20911B0730911C0740911D072F
:10F5100050911E07DC016D917D918D919C910F940E
:10F52000071B0F940C21AE966CAF7DAF8EAF9FAFD3
:10F53000AE9720911F0730912007409121075091ED
:10F540002207F30160817181828193810F94071BEF
:10F550000F940C21E2966CAF7DAF8EAF9FAFE29718
:10F5600020912307309124074091250750912607C9
:10F57000D4016D917D918D919C910F94071B0F94F7
:10F580000C21E6966CAF7DAF8EAF9FAFE6972091D2
:10F590002707309128074091290750912A07F50144
:10F5A00060817181828193810F94071B0F940C21DC
:10F5B0006A966CAF7DAF8EAF9FAF6A978091380A25
:10F5C0009091390AA0913A0AB0913B0AAE96CCAC20
:10F5D000DDACEEACFFACAE97C81AD90AEA0AFB0A5A
:10F5E00080913C0A90913D0AA0913E0AB0913F0A59
:10F5F000E2968CAC9DACAEACBFACE297881A990A8F
:10F60000AA0ABB0A8091400A9091410AA091420A3D
:10F61000B091430AE6960CAD1DAD2EAD3FADE69719
:10F62000081B190B2A0B3B0B0FAB18AF29AF3AAFD6
:10F6300080917B1483FF0EC06A962CAD3DAD4EAD1C
:10F640005FAD6A972093440A3093450A4093460A77
:10F650005093470A8091440A9091450AA091460A26
:10F66000B091470A6A964CAC5DAC6EAC7FAC6A97C1
:10F67000481A590A6A0A7B0A09F495C08091B012A7
:10F68000811141C06091690270916A02072E000CDD
:10F69000880B990B0F94A81A9B01AC016091AC12D6
:10F6A0007091AD128091AE129091AF120F94A21A88
:10F6B00087FF29C06A968CAD9DADAEADBFAD6A9790
:10F6C0008093440A9093450AA093460AB093470A50
:10F6D000E7E4F6E284918F010F5F1F4F882321F04A
:10F6E0000F940214F801F6CFECECFCE184918F0149
:10F6F0000F5F1F4F882321F00F940214F801F6CFFB
:10F70000412C512C32014BA65CA66DA67EA677FE3D
:10F710000BC000271127980104191509260937097C
:10F720000BA71CA72DA73EA760912707709128075C
:10F730008091290790912A070F941F209B01AC010B
:10F74000A8ECB0E00F94BB1E2BA53CA54DA55EA573
:10F7500062177307840795074CF56A968CAD9DADCB
:10F76000AEADBFAD6A978093440A9093450AA093CB
:10F77000460AB093470AE7E4F6E284918F010F5FEF
:10F780001F4F882321F00F940214F801F6CFEDEA01
:10F79000FCE184918F010F5F1F4F882321F00F94AC
:10F7A0000214F801F6CF412C512C3201D701C601C9
:10F7B0008827B7FD83959927AA27BB27282EB7FE50
:10F7C00003C0E82FE2602E2E0FA918AD29AD3AAD87
:10F7D00037FF03C0122D1460212E77FE03C0222DA7
:10F7E0002860222E032D10E0C301B2010F94A81A45
:10F7F000F801EE0FFF1FEE0FFF1FEA57F94F2081B0
:10F800003181428153810F94071B2B013C01000F72
:10F81000111FF801E359FD4F60817181072E000C23
:10F82000880B990B0F94A81A9B01AC01C301B2017C
:10F830000F94071B2AE037ED43E25CE30F94071BAC
:10F840002B013C0120E030E0A9010F9401211816A2
:10F850004CF420E030E040E05FE3C301B2010F94DC
:10F86000DB1E08C0A301920160E070E080E09FE32E
:10F870000F94DA1E0F941F206CAF7DAF8EAF9FAF39
:10F880008091480A8F5F8F706F968FAF6F978091CE
:10F89000490A6F960FAD6F97801304C080E00F94F4
:10F8A000360BF5CFE091480A0E2F10E01CA70BA7EE
:10F8B0001FE4E19FF0011124E557F24F108222A2CC
:10F8C000D701C601F7FE07C088279927DC018C19EC
:10F8D0009D09AE09BF0982839383A483B5838FE416
:10F8E0000BA51CA5809FF001819FF00D1124E55709
:10F8F000F24FD501C401B7FE07C088279927DC0164
:10F9000088199909AA09BB0986839783A087B187BB
:10F910008FE40BA51CA5809FF001819FF00D1124A1
:10F92000E557F24F8FA998ADA9ADBAADB7FF07C0A3
:10F93000B095A095909581959F4FAF4FBF4F82870F
:10F940009387A487B5878FE40BA51CA5809FF00142
:10F95000819FF00D1124E557F24F2CAD3DAD4EAD1A
:10F960005FAD26873787408B518B428153816481FD
:10F9700075810681178120853185041715072607B3
:10F98000370714F48A019B018FE4ABA5BCA58A9FBD
:10F99000F0018B9FF00D1124E557F24F828593857E
:10F9A000A485B58580179107A207B30764F48CADD1
:10F9B0009DADAEADBFAD80179107A207B30764F44C
:10F9C000D901C8010DC00CAD1DAD2EAD3FAD08175E
:10F9D00019072A073B0724F08CAD9DADAEADBFAD36
:10F9E0002FE40BA51CA5209FF001219FF00D1124F1
:10F9F000E557F24F828B938BA48BB58B0697A105AD
:10FA0000B10510F40C94F386DF01A95BBF4F809120
:10FA10004B0490914C0411969C938E931296809176
:10FA20004D0490914E048D939C933182452B462B2F
:10FA3000472B09F017988FE40BA51CA5809FF001B8
:10FA4000819FF00D1124E557F24F86819781A085A3
:10FA5000B185892B8A2B8B2B09F016988FE40BA587
:10FA60001CA5809FF001819FF00D1124E557F24FF6
:10FA700082859385A485B585892B8A2B8B2B09F0EC
:10FA800015982CAD3DAD4EAD5FAD232B242B252B12
:10FA9000B1F080918506882319F081508093850606
:10FAA000311004C0149880E2809385062090580499
:10FAB0003090590400915A0410915B0408C02090C2
:10FAC000540430905504009156041091570491014C
:10FAD000A8016FA57BA98BAD21969FAD21970F94AF
:10FAE000A21A87FD02C00C94EB86C701B6010F94E1
:10FAF000A81A2091E3043091E4044091E504509168
:10FB0000E6040F94071B6FA778AB89AB9AAB698BA0
:10FB10007A8B8B8B9C8BC501B4010F94A81A209112
:10FB2000E7043091E8044091E9045091EA040F940D
:10FB3000071B4B015C016D8B7E8B8F8B988F6FA9A0
:10FB400078AD89AD9AAD0F94A81A2091EB0430914D
:10FB5000EC044091ED045091EE040F94071B6B01EF
:10FB60007C01698F7A8F8B8F9C8F2091EF0430916D
:10FB7000F0044091F1045091F204C301B2010F94DA
:10FB8000071B6D8F7E8F8F8F98A32FE44BA55CA5ED
:10FB9000249FF001259FF00D1124E557F24F42807C
:10FBA00053806480758056E04516510461047104E9
:10FBB000E4F44680578060847184A6E04A165104BC
:10FBC0006104710494F44284538464847584B6E0BF
:10FBD0004B1651046104710444F4DC01CB01BF777E
:10FBE00087A790ABA1ABB2AB34C02FA538A949A968
:10FBF0005AA9CA01B9010F94071B2B013C01A501A9
:10FC00009401C501B4010F94071B9B01AC01C30112
:10FC1000B2010F94DB1E4B015C01A7019601C701E5
:10FC2000B6010F94071B9B01AC01C501B4010F94F1
:10FC3000DB1E0F9446212FE44BA55CA5249FF00109
:10FC4000259FF00D1124E557F24F67A770AB81ABEC
:10FC500092AB8FE4ABA5BCA58A9FF0018B9FF00D02
:10FC60001124E557F24F27A530A941A952A960E018
:10FC700070E080E89FE30F94B71F26966CAF7DAFCE
:10FC80008EAF9FAF26979B01AC01B101C8010F94C5
:10FC9000071B6B017C010E947BBA2B968FAF2B97C1
:10FCA000A701960160E074E284E799E40F94B71F1E
:10FCB0000F940C214B015C012B968FAD2B9782503A
:10FCC000863008F044C08091E1069091E206A09150
:10FCD000E306B091E40688169906AA06BB06B8F5B5
:10FCE00088199909AA09BB09BC01CD01660F771FC4
:10FCF000881F991F2B96BFAD2B970B2F10E020E08C
:10FD000030E0A90198010F947D1ECA01B9010F943A
:10FD1000A61A0F940C21680D791D8A1D9B1D0F9446
:10FD2000A61A9B01AC0160E074E284E799E40F94A9
:10FD3000B71F6B017C019B01AC0160E074E284E7BA
:10FD400099E40F94B71F0F940C214B015C012FB75E
:10FD5000F8948091001390910113A0910213B09137
:10FD60000313880E991EAA1EBB1E80920013909248
:10FD70000113A0920213B09203132FBF8FE4EBA5DF
:10FD8000FCA58E9F80018F9F100D11240557124FE7
:10FD9000D8019F962D913D914D915C91D297A3965C
:10FDA0002CAF3DAF4EAF5FAFA397A7019601A396CF
:10FDB0006CAD7DAD8EAD9FADA3970F94071B2A96BA
:10FDC0006CAF7DAF8EAF9FAF2A97F80163A374A38A
:10FDD00085A396A322893389448955892FAB38AFEF
:10FDE00049AF5AAFCA01B9010F94A61A6FA778ABF1
:10FDF00089AB9AABA70196010F94071B0F94A11F23
:10FE00000F94242062966CAF7DAF8EAF9FAF629748
:10FE1000F80167AB70AF81AF92AF8E010F5E1F4FDD
:10FE200022961FAF0EAF22970051110966961FAFA1
:10FE30000EAF66970CE514E06C961FAF0EAF6C9793
:10FE40008E010F5D1F4F1AA709A766960EAD1FAD55
:10FE5000669764961FAF0EAF6497212C312C10E883
:10FE60001BAB0FE30BAF2296AEADBFAD22976D91EA
:10FE70007D918D919D912296BFAFAEAF2297A70144
:10FE800096010F94071B6496EEADFFAD64976193E6
:10FE90007193819391936496FFAFEEAF64974B019A
:10FEA0005C01E894B7F86C96AEADBFAD6C974D9021
:10FEB0005D906D907D906C96BFAFAEAF6C97A301D7
:10FEC0009201C501B4010F9401211816A4F4A501F3
:10FED0009401C301B2010F94B71F5B018C019B0118
:10FEE000AC01B1018BA99BAD0F94012118161CF434
:10FEF00015010BAB1BAF22960EAD1FAD229729A5A6
:10FF00003AA50217130709F0AECF20E030E040E831
:10FF10005FE3B1018BA99BAD0F94A21A87FF4BC081
:10FF20007E0131E1E30EF11C66960EAD1FAD6697C2
:10FF300091014BA95BADD8016D917D918D919C9103
:10FF40000F94071BF80161937193819391938F0133
:10FF5000EE15FF0569F78FE42BA53CA5829F800174
:10FF6000839F100D11240557124F91014BA95BADD2
:10FF70002A966CAD7DAD8EAD9FAD2A970F94071B71
:10FF8000D80193966D937D938D939C9396976296EB
:10FF90006CAD7DAD8EAD9FAD62970F94A61A9101A9
:10FFA0004BA95BAD0F94071B0F942420F80167AB9E
:10FFB00070AF81AF92AF26962CAD3DAD4EAD5FAD2B
:10FFC00026976FA578A989A99AA90F94071B6BABEF
:10FFD0007CAB8DAB9EAB8FE40BA51CA5809FF00185
:10FFE000819FF00D1124E557F24F82809380A48009
:10FFF000B58081149104A104B10409F5868197812B
:020000021000EC
:10000000A085B185892B8A2B8B2BC9F4828593859A
:10001000A485B585892B8A2B8B2B89F420918104AB
:100020003091820440918304509184046BA97CA98F
:100030008DA99EA90F94071B0F94A11F27C22CAD59
:100040003DAD4EAD5FAD232B242B252B49F06091A8
:10005000850470918604809187049091880408C07B
:1000600060917D0470917E0480917F049091800462
:100070002BA93CA94DA95EA90F94071B0F94A11FA2
:100080000F9424206B017C018091770D9091780D65
:10009000A091790DB0917A0D0FA918AD29AD3AADA7
:1000A00080179107A207B30708F4E2C081149104F6
:1000B000A104B10441F120917B0D30917C0D409160
:1000C0007D0D50917E0D2C153D054E055F05D8F434
:1000D0006FA978AD89AD9AAD0F946E1E2B013C01CE
:1000E000A7019601C501B4010F946E1E461657066E
:1000F0006806790640F4C301B201A50194010F948A
:100100007D1E69017A018FE40BA51CA5809FF0017B
:10011000819FF00D1124E557F24F86809780A084CF
:10012000B18481149104A104B10441F120917F0DA7
:100130003091800D4091810D5091820D2C153D051F
:100140004E055F05D8F46FA978AD89AD9AAD0F94CF
:100150006E1E2B013C01A7019601C501B4010F944D
:100160006E1E461657066806790640F4C301B201B2
:10017000A50194010F947D1E69017A018FE40BA5FE
:100180001CA5809FF001819FF00D1124E557F24FCF
:1001900082849384A484B58481149104A104B1045D
:1001A00041F12091830D3091840D4091850D509146
:1001B000860D2C153D054E055F05D8F46FA978AD69
:1001C00089AD9AAD0F946E1E2B013C01A7019601DB
:1001D000C501B4010F946E1E4616570668067906CF
:1001E00040F4C301B201A50194010F947D1E690181
:1001F0007A018FE40BA51CA5809FF001819FF00D73
:100200001124E557F24F86849784A088B188811421
:100210009104A104B10409F43DC12091870D3091EE
:10022000880D4091890D50918A0D2C153D054E0584
:100230005F0508F02FC16FA978AD89AD9AAD0F9415
:100240006E1E2B013C01A7019601C501B4010F945C
:100250006E1E461657066806790608F01BC1C301D4
:10026000B201A50194010F947D1E69017A0112C1AA
:1002700081149104A104B104A9F160917B0D7091E6
:100280007C0D80917D0D90917E0D6C157D058E0508
:100290009F0540F50F94A61A2FA538A949A95AA978
:1002A0000F94071B2B013C01C501B4010F94A81A40
:1002B0004B015C01C701B6010F94A61AA501940178
:1002C0000F94071BA30192010F940121181654F4F7
:1002D000A5019401C301B2010F94B71F0F9424200C
:1002E0006B017C018FE40BA51CA5809FF001819F11
:1002F000F00D1124E557F24F4680578060847184D9
:100300004114510461047104A9F160917F0D709151
:10031000800D8091810D9091820D6C157D058E056B
:100320009F0540F50F94A61A2FA538A949A95AA9E7
:100330000F94071B4B015C01C301B2010F94A81A73
:100340002B013C01C701B6010F94A61AA30192012B
:100350000F94071BA50194010F940121181654F462
:10036000A3019201C501B4010F94B71F0F9424207B
:100370006B017C018FE40BA51CA5809FF001819F80
:10038000F00D1124E557F24F428453846484758440
:100390004114510461047104A9F16091830D7091BD
:1003A000840D8091850D9091860D6C157D058E05CF
:1003B0009F0540F50F94A61A2FA538A949A95AA957
:1003C0000F94071B4B015C01C301B2010F94A81AE3
:1003D0002B013C01C701B6010F94A61AA30192019B
:1003E0000F94071BA50194010F940121181654F4D2
:1003F000A3019201C501B4010F94B71F0F942420EB
:100400006B017C018FE40BA51CA5809FF001819FEF
:10041000F00D1124E557F24F86849784A088B188A7
:1004200081149104A104B104A9F16091870D709128
:10043000880D8091890D90918A0D6C157D058E0532
:100440009F0540F50F94A61A2FA538A949A95AA9C6
:100450000F94071B2B013C01C501B4010F94A81A8E
:100460004B015C01C701B6010F94A61AA5019401C6
:100470000F94071BA30192010F940121181654F445
:10048000A5019401C301B2010F94B71F0F9424205A
:100490006B017C018FE42BA53CA5829F8001839F8B
:1004A000100D11240557124FF801ED5BFF4FC0826C
:1004B000D182E282F382C701B6010F94A61A6B01C2
:1004C0007C012BA93CA94DA95EA90F94B71F6E967C
:1004D0006CAF7DAF8EAF9FAF6E97D801D3966D9303
:1004E0007D938D939C93D69720E030E040E85BE4C9
:1004F000C701B6010F94071B20E034E244EF59E432
:100500000F94B71F0F941F20F801668F778F80A379
:1005100091A3F3A1FCAFD8019496BC91BFABF801B5
:10052000F5A1FFA7D8019696BC91BBAB03E61DE0F1
:10053000A6961FAF0EAFA6972E0111E1410E511CDA
:1005400033E6232E3DE0332E66966EAC7FAC669785
:100550000CAD0BAF1FA921961FAF21972396FFAFBC
:1005600023972796BFAF279710E0D3018D909D90DA
:10057000AD90BD903D01E894B7F8F101C190D190E4
:10058000E190F1901F01A7019601C501B4010F94FC
:1005900001211816E4F5112379F12CAD3FA94FA5DF
:1005A0005BA9C701B6010F94071B6B017C012BAD42
:1005B00021963FAD219723964FAD239727965FADA8
:1005C0002797C501B4010F94071BA70196010F944B
:1005D00001211816DCF4A5019401C701B6010F949E
:1005E000B71F6BAF21967FAF219723968FAF2397CD
:1005F00027969FAF27970AC0CBAE2196DFAE2197F3
:100600002396EFAE23972796FFAE279711E0641449
:10061000750409F0AACF2B960FAD2B97023008F482
:1006200076C13090240A2090250A1091260A009164
:10063000270A27E137EB41ED58E3632D722D812F17
:10064000902F0F94012118160CF061C121E0A4969F
:100650002FAFA4972CAD3FA94FA55BA9632D722D99
:10066000812F902F0F9401211816A4F0A4961FAE8D
:10067000A4972CAD3FA94FA55BA9632D722D812FA7
:10068000902F0F94B71FAA966CAF7DAF8EAF9FAF20
:10069000AA9714C0232D322D412F502F6CAD7FA966
:1006A0008FA59BA90F94B71FAA966CAF7DAF8EAF95
:1006B0009FAFAA973CAC2FA81FA50BA948E25AE010
:1006C00064965FAF4EAF649780E090E0A0E8BFE330
:1006D0002E968CAF9DAFAEAFBFAF2E972F961FAEAD
:1006E0002F976496AEADBFAD6497CD90DD90ED9041
:1006F000FD906496BFAFAEAF64976696EEADFFAD6A
:10070000669781909190A190B1906696FFAFEEAF01
:100710006697A496FFADA497FF2361F0AA962CAD2F
:100720003DAD4EAD5FADAA97C701B6010F94071B53
:100730006B017C012F962FAD2F972223C1F02E96AF
:100740002CAD3DAD4EAD5FAD2E97C701B6010F94F8
:10075000071B6B017C012E962CAD3DAD4EAD5FAD00
:100760002E97C501B4010F94071B4B015C01A50135
:100770009401C701B6010F94012120E030E0A901E6
:1007800018162CF5C501B4010F94012118164CF070
:1007900020E030E0A901C701B6010F94A21A87FF3B
:1007A00005C0A5019401C701B60124C0240135018B
:1007B00077FA709477F87094A3019201C701B6019B
:1007C0000F94012118165CF52601370128C0C501D8
:1007D000B4010F94A21A87FD09C020E030E0A901FE
:1007E000C701B6010F94012118164CF4A701960118
:1007F000C501B4010F94DA1E2B013C0110C0260183
:10080000370177FA709477F87094A5019401C301C9
:10081000B2010F940121181614F024013501A69697
:10082000AEADBFADA697CD90DD90ED90FD90A696B4
:10083000BFAFAEAFA697A7019601C301B2010F9457
:1008400001211816ECF4A3019201C701B6010F941F
:10085000B71F9B01AC012E966CAD7DAD8EAD9FADEB
:100860002E970F94071B2E966CAF7DAF8EAF9FAF68
:100870002E972F96BFAD2F97BF5F2F96BFAF2F97A5
:100880006496EEADFFAD6497E853FA4009F029CFC6
:100890002F963FAD2F97332381F02E962CAD3DAD93
:1008A0004EAD5FAD2E97632D722D812F902F0F943B
:1008B000071B362E272E182F092F24EA30E74DE785
:1008C0005FE3632D722D812F902F0F94071B6B0117
:1008D0007C019B01AC016091810670918206809140
:1008E0008306909184060F94012118163CF5A70108
:1008F00096016BAD21967FAD219723968FAD2397FF
:1009000027969FAD27970F9401211816BCF48FE40A
:100910000BA51CA5809FF001819FF00D1124E557C8
:10092000F24F8081846080833BAC21962FAC21976D
:1009300023961FAD239727960FAD27978FE42BA5FE
:100940003CA5829FF001839FF00D1124E557F24FE3
:10095000832D922DA12FB02F83A794A7A5A7B6A76B
:100960006E966CAD7DAD8EAD9FAD6E9790589B0130
:10097000AC010F94DB1EA3962CAD3DAD4EAD5FAD2B
:10098000A3970F94071B9B01AC016BE077ED83E20B
:100990009BE30F94DA1E0F9446216B017C019B01AF
:1009A000AC01632D722D812F902F0F94A21A87FD19
:1009B00004C03C2C2D2C1E2D0F2D8FE44BA55CA5C7
:1009C000849FF001859FF00D1124E557F24F832D90
:1009D000922DA12FB02F87A390A7A1A7B2A7B08077
:1009E0009601A7016CAD7FA98FA59BA90F94A21AB0
:1009F000181614F481E001C083E09FE4ABA5BCA508
:100A00009A9F90019B9F300D1124F901E557F24FF9
:100A10007F01B82AB08280E1FE013196A8E2BAE0F7
:100A200001900D928A95E1F78CAD9FA9AFA5BBA966
:100A30008093240A9093250AA093260AB093270A4C
:100A40008BAD21969FAD21972396AFAD2397279627
:100A5000BFAD27978093810690938206A09383066B
:100A6000B09384062CAD3FA94FA55BA9BC01CD0175
:100A70000F94B71F6DA37EA38FA398A72CAD3FA99A
:100A80004FA55BA9632D722D812F902F0F94B71F57
:100A900069A37AA38BA39CA3AE014B5D5F4FBE01FC
:100AA0006F5D7F4FC7010E9477786F960FAD6F978C
:100AB0000093480AAE962CAD3DAD4EAD5FADAE97FE
:100AC0002093380A3093390A40933A0A50933B0AEC
:100AD000E2968CAD9DADAEADBFADE29780933C0A82
:100AE00090933D0AA0933E0AB0933F0AE6960CAD60
:100AF0001DAD2EAD3FADE6970093400A1093410A1D
:100B00002093420A3093430A6A962CAD3DAD4EAD18
:100B10005FAD6A972093440A3093450A4093460A92
:100B20005093470A0E947BBA843048F41091490AD6
:100B3000F12C00E080E090E02FE4E22E9EC0409097
:100B4000490A8091480A83508F70F82EA12CB12C4D
:100B500000E010E09FE4592EF41441F30115110553
:100B600021F0D8018C9182FDE1CF8FEF8F0D8F7036
:100B7000F82E589EC0011124FC01E557F24FFCA746
:100B8000EBA70115110509F474C0A114B10409F40F
:100B900070C0D8019B967C909B979C96CC909C971C
:100BA0009D96DC909D979E96EC909E97272D3C2DD0
:100BB0004D2D5E2D97966D917D918D919C919A977B
:100BC0000F94A21A882309F454C0F801608061FCD4
:100BD00042C0D50197968D909D90AD90BC909A970C
:100BE000A5019401672D7C2D8D2D9E2D0F94A21AA9
:100BF00018168CF5A5019401C501B4010F94071BCB
:100C00004B015C01F80183A994A9A5A9B6A9BC016F
:100C1000CD0190589B01AC010F94DB1ED8019F962B
:100C20002D913D914D915C91D2970F94071B9B01A3
:100C3000AC01C501B4010F94DA1E0F9446211B01CB
:100C40005C019B01AC01672D7C2D8D2D9E2D0F9499
:100C5000A21A87FF04C0272C3C2CAD2CBE2CC1014E
:100C6000D501F80187A390A7A1A7B2A7862D81601F
:100C7000808358010BA51CA56FCF2091480A12173D
:100C800091F0E19E90011124A9014557524F6A014C
:100C90006F2D702F0E9401781F5F1F708F2D902F76
:100CA000FC2C0D2DEACF6F2D702F0E940178F09053
:100CB000490A00E010E08FE4E82E4F2D0F2C000CC5
:100CC000550B8091480A90E04817590709F44DC028
:100CD000E49EC001E59E900D1124DC01A557B24FA2
:100CE0006D0101151105D9F1F801808180FD03C066
:100CF0008C9180FF34C0D80193968D909D90AD90DB
:100D0000BC909697E49EF001E59EF00D1124E55706
:100D1000F24FA501940167A170A581A592A50F943A
:100D2000B71F69A37AA38BA39CA3A5019401F80123
:100D300067A170A581A592A50F94B71F6DA37EA38F
:100D40008FA398A7AE014F5D5F4FBE016B5D7F4FD4
:100D5000C8010E947778D8018C918E7F8C9381E0B6
:100D60008F0D8F70F82E8601A8CF0115110569F13E
:100D7000F801C3A0D4A0E5A0F6A0A70196016DECF0
:100D80007CEC8CE49DE30F94B71F69A37AA38BA33B
:100D90009CA3A7019601D80197966D917D918D91A5
:100DA0009C919A970F94B71F6DA37EA38FA398A7CA
:100DB000AE014F5D5F4FBE016B5D7F4FC8010E946A
:100DC0007778F80180818E7F808380916F008260C8
:100DD00080936F0008C02FA43BA80BAD21961FADD8
:100DE00021970C94757DCB58DF4F0FB6F894DEBF7A
:100DF0000FBECDBFDF91CF911F910F91FF90EF906C
:100E0000DF90CF90BF90AF909F908F907F906F902A
:100E10005F904F903F902F9008952F923F924F9266
:100E20005F926F927F928F929F92AF92BF92CF927A
:100E3000DF92EF92FF920F931F93CF93DF93CDB783
:100E4000DEB7EC970FB6F894DEBF0FBECDBF209192
:100E5000BF12222309F437C11C010091040A10912A
:100E6000050A2091060A3091070A4090080A50901E
:100E7000090A60900A0A70900B0A49AA5AAA6BAA3A
:100E80007CAA80900C0A90900D0AA0900E0AB09057
:100E90000F0A4091100A5091110A6091120A709144
:100EA000130A8091140A9091150AA091160AB09124
:100EB000170A8DAB9EABAFABB8AFC090180AD090FD
:100EC000190AE0901A0AF0901B0A80911C0A90916E
:100ED0001D0AA0911E0AB0911F0A4090200A50904E
:100EE000210A6090220A7090230A49AE5AAE6BAE76
:100EF0007CAE4090000A5090010A6090020A709007
:100F0000030A49825A826B827C828D829E82AF82E2
:100F1000B886C986DA86EB86FC860D871E872F8702
:100F2000388B498B5A8B6B8B7C8B8D8B9E8BAF8BCD
:100F3000B88F89A99AA9ABA9BCA9898F9A8FAB8FC1
:100F4000BC8F4DA85EA86FA878AC4D8E5E8E6F8E5C
:100F500078A289AD9AADABADBCAD89A39AA3ABA382
:100F6000BCA32091431330914413409145135091F9
:100F70004613D1016D917D918D919C910F94DA1E54
:100F800020E030E048E951E40F94DB1E6DA77EA716
:100F90008FA798AB20914713309148134091491384
:100FA00050914A13F10164817581868197810F9474
:100FB000DA1E20E030E041E853E40F94DA1E69A71E
:100FC0007AA78BA79CA720914B1330914C1340918B
:100FD0004D1350914E13D10118966D917D918D91C5
:100FE0009C911B970F94DA1E6DA37EA38FA398A7E5
:100FF000CE0185969F938F9304969F938F9304962B
:101000009F938F93EDB7FEB7B4970FB6F894FEBFDA
:101010000FBEEDBFADB7BEB7119684E2FE013196AB
:1010200001900D928A95E1F70E940BD420E030E008
:1010300048E951E46DA57EA58FA598A90F94DA1E05
:10104000209143133091441340914513509146131E
:101050000F94DB1ED1016D937D938D939C93139719
:1010600020E030E041E853E469A57AA58BA59CA572
:101070000F94DB1E20914713309148134091491380
:1010800050914A130F94DB1EF101648375838683AC
:10109000978320914B1330914C1340914D135091F5
:1010A0004E136DA17EA18FA198A50F94DB1ED101D7
:1010B00018966D937D938D939C931B970FB6F89420
:1010C000DEBF0FBECDBFEC960FB6F894DEBF0FBEED
:1010D000CDBFDF91CF911F910F91FF90EF90DF90E7
:1010E000CF90BF90AF909F908F907F906F905F90C8
:1010F0004F903F902F900895CF92DF92EF92FF9202
:101100000F931F93CF93DF93CDB7DEB72C970FB616
:10111000F894DEBF0FBECDBF2091BF12222309F489
:10112000B0C08A017B016C012091431330914413BC
:101130004091451350914613FC0160817181828179
:1011400093810F94DA1E20E030E048E951E40F94D7
:10115000DB1E69877A878B879C87209147133091A4
:1011600048134091491350914A13F70160817181EE
:10117000828193810F94DA1E20E030E041E853E44D
:101180000F94DA1E6D837E838F83988720914B1393
:1011900030914C1340914D1350914E13F8016081E2
:1011A0007181828193810F94DA1E69837A838B83A4
:1011B0009C83CE0101969F938F9304969F938F9368
:1011C00004969F938F938DB79EB784970FB6F8942C
:1011D0009EBF0FBE8DBFADB7BEB7119684E2E0E0F3
:1011E000FAE001900D928A95E1F70E940BD420E07D
:1011F00030E048E951E469857A858B859C850F94B8
:10120000DA1E2091431330914413409145135091BD
:1012100046130F94DB1EF6016083718382839383F0
:1012200020E030E041E853E46D817E818F81988534
:101230000F94DB1E209147133091481340914913BE
:1012400050914A130F94DB1EF701608371838283F0
:10125000938320914B1330914C1340914D13509137
:101260004E1369817A818B819C810F94DB1EF8017A
:1012700060837183828393830FB6F894DEBF0FBEC1
:10128000CDBF2C960FB6F894DEBF0FBECDBFDF9159
:10129000CF911F910F91FF90EF90DF90CF90089525
:1012A000CF93809136098823A9F140912E0950915E
:1012B0002F0960913009709131092EE237E0809159
:1012C00037099091380969D4C82F811102C0C0E054
:1012D00022C04091320950913309609134097091D4
:1012E0003509411551056105710589F02EE237E098
:1012F000809137099091380950D4882341F3109296
:101300003209109233091092340910923509109263
:10131000360901C0C1E08C2FCF910895CF92DF92A2
:10132000EF92FF92CF936B017C01C42F80912E0925
:1013300090912F09A0913009B09131098C159D052C
:10134000AE05BF05C1F0ACDF811102C080E017C05F
:101350002EE237E0B701A601809137099091380954
:1013600002D6882399F3C0922E09D0922F09E092D9
:101370003009F092310981E0C11180933609CF9193
:10138000FF90EF90DF90CF9008954F925F926F9211
:101390007F928F929F92AF92BF92CF92DF92EF9205
:1013A000FF920F931F93CF93DF93EC016A017B01B0
:1013B00028013901423051056105710510F480E0C2
:1013C00064C089859A85AB85BC850196A11DB11D38
:1013D00084179507A607B70790F38F89803149F4E2
:1013E0008D2C9E2CAF2CBB248B899C89AD89BE890A
:1013F0000FC0803221F78B889C88AD88BE88DB01C6
:10140000CA0157E0B695A795979587955A95D1F754
:10141000880E991EAA1EBB1E41E0C501B4017EDFE5
:10142000882369F29F89903161F4DD24EE24FF2442
:101430009601220F331FF901E25DF84F518240827D
:1014400011C0E894C7F8DD24EE24FF249601220F92
:10145000331F220F331FF901E25DF84F40825182A2
:10146000628273829A89923080F04D815E816F81B1
:101470007885840E951EA61EB71E80923209909222
:101480003309A0923409B0923509DF91CF911F91B1
:101490000F91FF90EF90DF90CF90BF90AF909F9013
:1014A0008F907F906F905F904F900895CF92DF92D2
:1014B000EF92FF920F931F93CF93DF93FC018185EF
:1014C0009285A385B4850196A11DB11D841795074A
:1014D000A607B70710F480E061C08789803149F41E
:1014E000BB27A72F962F852FC388D488E588F68839
:1014F0000FC0803281F783899489A589B6896A01F2
:101500007B01C7E0F694E794D794C794CA95D1F7C6
:101510008C0D9D1DAE1DBF1DE9016A017B018F0170
:1015200040912E0950912F09609130097091310935
:1015300084179507A607B70799F4F80187898031C2
:10154000B1F4B701A601552766277727440F551F29
:10155000FA01E25DF84F80819181A0E0B0E019C00E
:1015600040E0BC01CD01DADE8111E7CFB4CFB70195
:10157000A6014F77552766277727440F551F440F3D
:10158000551FFA01E25DF84F80819181A281B381FC
:10159000BF7088839983AA83BB8381E0DF91CF9159
:1015A0001F910F91FF90EF90DF90CF9008954F9291
:1015B0005F926F927F92AF92BF92CF92DF92EF9243
:1015C000FF920F931F93CF93DF9300D01F92CDB75D
:1015D000DEB78C0149835A836B837C835901C12C0C
:1015E000D12C7601412C82E0582E612C712C49813E
:1015F0005A816B817C819E012F5F3F4FC80156DF6E
:10160000882341F1D301C201F801058404C0880F89
:10161000991FAA1FBB1F0A94D2F7C80ED91EEA1E33
:10162000FB1E49815A816B817C818789803139F425
:1016300081E0483F5F4F6105710538F4D8CF81E004
:10164000483F5F4F6F4F7F4090F2F501C082D182DB
:10165000E282F3820F900F900F900F90DF91CF9165
:101660001F910F91FF90EF90DF90CF90BF90AF90C0
:101670007F906F905F904F9008953F924F925F924E
:101680006F927F928F929F92AF92BF92CF92DF9292
:10169000EF92FF920F931F93CF93DF93CDB7DEB7F7
:1016A0002C970FB6F894DEBF0FBECDBF5C01DC01F6
:1016B00059968D909C905A97F40181859285A385C7
:1016C000B4859C01AD012F5F3F4F4F4F5F4F29877E
:1016D0003A874B875C87D5011496CD90DD90ED90CD
:1016E000FC901797C114D104E104F10439F0BFEF65
:1016F000CB1ADB0AEB0AFB0A312C07C0F401C080CD
:10170000D180E280F38033243394260137011D8297
:101710001E821F821886F40181859285A385B48577
:101720002D813E814F815885281739074A075B076D
:1017300008F061C089859A85AB85BC858C159D05AF
:10174000AE05BF0550F482E0C82ED12CE12CF12C5F
:1017500092E0492E512C612C712C9E012F5F3F4F3E
:10176000B701A601C401A2DE882309F444C089811F
:101770009A81AB81BC81892B8A2B8B2B41F026016E
:1017800037019FEF491A590A690A790A05C0C4143A
:10179000D504E604F70491F02D813E814F815885F0
:1017A0002F5F3F4F4F4F5F4F2D833E834F835887AF
:1017B0003FEFC31AD30AE30AF30AADCF0FEF1FEFCF
:1017C0002FEF3FE0B301A201C401DFDDF82E882333
:1017D00091F0D50114964D915D916D917C91179783
:1017E000411551056105710541F093018201C40164
:1017F000CCDD811102C0F12C29C0D50114964D9287
:101800005D926D927C921797332051F0D301C20103
:101810000196A11DB11DF40180839183A283B3833E
:10182000F50185899689A789B08D892B8A2B8B2B09
:1018300069F4D50155964D925D926D927C925897C0
:1018400011968C911197806811968C938F2D2C9600
:101850000FB6F894DEBF0FBECDBFDF91CF911F91C1
:101860000F91FF90EF90DF90CF90BF90AF909F903F
:101870008F907F906F905F904F903F9008958F92E0
:101880009F92AF92BF92CF92DF92EF92FF920F930F
:101890001F93CF93DF93EC018B81811102C080E015
:1018A00076C009891A892B893C89041715072607F0
:1018B0003707A8F36A017B01823029F4C886D986EC
:1018C000EA86FB860DC0C114D104E104F10451F491
:1018D0001C821D821E821F82188619861A861B860C
:1018E00081E055C088849984AA84BB84E98DFA8DEF
:1018F000258530E0275F3F4FB501A40141505109D4
:1019000061097109022E04C0769567955795479530
:101910000A94D2F7D701C6010197A109B10904C001
:10192000B695A795979587952A95D2F78417950729
:10193000A607B70720F089288A288B2849F44D8903
:101940005E896F89788D4C835D836E837F8304C04D
:10195000841B950BA60BB70B4C015D018E010C5F30
:101960001F4F81149104A104B10409F4A7CF4C8145
:101970005D816E817F819801898D9A8D97DD91E0DF
:10198000891A9108A108B1088111EBCF88CFDF91A6
:10199000CF911F910F91FF90EF90DF90CF90BF906C
:1019A000AF909F908F9008950F931F93CF93DF93E5
:1019B000FC012381222311F080E043C08B01EC0164
:1019C000FB018789803131F18032B1F783E08B836D
:1019D000F801428D538D648D758D4D8B5E8B6F8BB1
:1019E000788F9E012F5E3F4FC801E1DD882321F3F0
:1019F0001A8F098F81E089831C821D821E821F82BB
:101A0000188619861A861B861C861D861E861F86CA
:101A1000188A17C082E08B831D8A1E8A1F8A188E3F
:101A2000FB01808D918DA0E0B0E025E0880F991F2B
:101A3000AA1FBB1F2A95D1F7898B9A8BAB8BBC8BC6
:101A4000D7CFDF91CF911F910F910895CF93DF935F
:101A5000EC0141E0611101C040E06C857D858E851F
:101A60009F855CDC882341F0888920E2829FC00149
:101A70001124825D984F02C080E090E0DF91CF9109
:101A80000895CF93DF93EC018B81882329F189811D
:101A900087FF1FC061E0CE01D9DFFC01892BE1F097
:101AA0008081853EC9F08B81823040F489899A8992
:101AB000AB89BC89848F958FA68FB78F8D899E89BE
:101AC000AF89B88D938F828FB58BA48B89818F77E7
:101AD0008983DF91CF91E4CB81E0888380E0DF913F
:101AE000CF910895CF93DF93EC01CBDF1B82DF9181
:101AF000CF910895CF93DF93EB01FC012381211156
:101B000002C080E027C02250223020F48FE2888378
:101B100019821FC060E09ADF009799F3FC0190E002
:101B200080E02EE23081303269F0883029F4DE0125
:101B3000A90FB11D2C939F5F3081DE01A90FB11D4C
:101B40003C939F5F8F5F31968B3061F7C90FD11D3A
:101B5000188281E0DF91CF9108950F931F93CF9367
:101B6000DF938B010E94ACC1EB010F948B138F3F6D
:101B700049F00E94ACC16C1B7D0B60177107A8F384
:101B800080E001C081E0DF91CF911F910F91089516
:101B900061E0FC0180810C947FC00F931F93CF9371
:101BA000DF93EC0189018C81833039F089E0440FA7
:101BB000551F661F771F8A95D1F79A01AB0168E11F
:101BC000CE010F949213882311F086E032C08EEF7D
:101BD0008EBD80E090E00DB407FEFDCFF801E80F68
:101BE000F91F20812EBD0DB407FEFDCF21812EBD32
:101BF0000296811522E0920771F70DB407FEFDCF22
:101C00008FEF0F9486138FEF0F9486130F948B131F
